:100000000C9479220C94A8220C94A8220C94A82277
:100010000C94A8220C94A8220C94A8220C94A82238
:100020000C94A8220C94A8220C94A8220C94A82228
:100030000C94A8220C94FF520C94A8220C94A82291
:100040000C94A8220C94A8220C94A8220C94A82208
:100050000C94A8220C94A8220C94A8220C94A822F8
:100060000C94A8220C94BEDD0C94A8220C94EADD1A
:100070000C94A8220C9458A70C94A8220C94A822A3
:100080000C94A8220C94A8220C94A8220C94A822C8
:100090000C94A8220C94A8220C94A8220C94A822B8
:1000A0000C94A8220C94A8220C94A8220C94A822A8
:1000B0000C94A8220C94A8220C94A8220C94144FFF
:1000C0000C94A8220C94A8220C94A8220C94A82288
:1000D0000C94A8220C94A8220C94A8220C94A82278
:1000E0000C94A822EE4717481C48F84721486B4853
:1000F0006B48F8473F486B48444849484E48534886
:100100002B4830483548F8473A486B48F34726486B
:1001100058485D4861486B486B4865485072657047
:100120006172696E6720666F7220736C6565703AE4
:1001300049276D20636F6D706C6574696E6720610F
:100140006E792020717565756564206D6F766573B5
:100150002E004368616E67696E672046696C616D49
:10016000656E743A202049276D20636F6D706C6551
:1001700074696E6720616E7920207175657565649C
:10018000206D6F7665732E00494E56414C494420D0
:10019000544F4F4C3A2020202020202049207265C7
:1001A0006365697665642061204C65667420202053
:1001B000546F6F6C20636F6D616E642C2062757478
:1001C000204920206F6E6C792068617665206F6E03
:1001D0006520546F6F6C2E00494E56414C494420A7
:1001E000434F4D4D414E443A202020204920726516
:1001F000636569766564206120636F6D6D616E640F
:10020000666F7220612068656174656420706C613E
:1002100074652C20627574204920646F6E277420E9
:1002200068617665206F6E65004920736177206193
:1002300020676C6974636820696E206D795344206F
:10024000636172642E204966207468697320697343
:1002500020746865206669727374206572726F72AB
:100260002C2074727974686973206D6F64656C20DA
:10027000616761696E2E20202000492074696D65D8
:1002800064206F7574207768696C65202020617424
:1002900074656D7074696E6720746F206865617431
:1002A00020206D792065787472756465722E00491E
:1002B0002074696D6564206F7574207768696C655A
:1002C000202020617474656D7074696E6720746F8E
:1002D000206865617420206D7920706C6174666F90
:1002E000726D2E00507265706172696E6720666F64
:1002F0007220736C6565703A49276D20636F6F6C6F
:10030000696E67206D792020202020206865617447
:1003100065727320616E6420676F696E6720746F09
:100320006D79207761697420706F736974696F6E7D
:100330002E004368616E67696E672046696C616D67
:10034000656E743A202049276D20676F696E6720BB
:10035000746F206D792077616974706F7369746947
:100360006F6E2E0052657374617274696E672074CB
:100370006865204275696C6400546869732069730C
:10038000206E6F74207468652078336720766572FC
:1003900073696F6E204920776F726B20626573748A
:1003A00020776974682E20466F722068656C702013
:1003B0007365653A206D616B6572626F742E636F51
:1003C0006D2F68656C70202020004920616D2061D0
:1003D000205265706C696361746F722E20205468BE
:1003E0006973206275696C6420697320666F72207E
:1003F0002020616E6F7468657220626F742E2053C6
:1004000065653A2020206D616B6572626F742E63A2
:100410006F6D2F68656C7000546865205265706C54
:100420006963617430720049276D2043616E6365B2
:100430006C6C696E672E2020202020506C656173E3
:100440006520576169742E002000486561746572EB
:10045000732073687574646F776E20202020647534
:100460006520746F20696E616374697669747920A0
:100470002020004578747275646572204F7665722D
:1004800068656174212020536F66747761726520FE
:1004900054656D70204C696D6974205265616368A4
:1004A00065642120506C65617365202020202053F5
:1004B000687574646F776E206F7220526573746113
:1004C00072740048656174696E67204661696C7575
:1004D000726521202020204D792065787472756422
:1004E00065727320617265206E6F746865617469EE
:1004F0006E672070726F7065726C792E20202043B9
:100500006865636B206D7920636F6E6E65637469D7
:100510006F6E730048656174696E67204661696C2F
:1005200075726521202020204D79206578747275C0
:100530006465727320617265202020206C6F73697E
:100540006E672074656D70657261747572652E20BA
:10055000436865636B206D7920636F6E6E656374AD
:10056000696F6E7300486561746572204572726FC1
:1005700072212020202020202049276D20726561D3
:1005800064696E67206F7574206F66202072616EDB
:1005900067652074656D7065726174757265732E20
:1005A00020436865636B206D7920636F6E6E6563B1
:1005B00074696F6E7300486561746572204572726C
:1005C0006F7221202020202020204D792074656D1D
:1005D00070657261747572652072656164736172B1
:1005E00065206661696C696E672120506C65617376
:1005F0006520436865636B206D7920636F6E6E655F
:100600006374696F6E73009302690000006900EE05
:10061000016900000069002601B801000000002007
:10062000065500000055002D085500000055004DEE
:100630000A550000005500400CAB000000AB002D37
:10064000095500000055002D085500000055004DCB
:100650000AAB000000550000000001C00D5500006D
:100660000055002D08560100000000C00D20015368
:1006700011BC005B12B10100000000C00DC80000F9
:10068000001400C00DC80000001400910E9001007D
:100690000014005A10900100001400C00D20030047
:1006A000000000C805C80000001400C805C800000C
:1006B000001400C805C80000001400DD04B00400E8
:1006C0000014007505C800000014007505C800007E
:1006D0000014007505C800000014009704B0040061
:1006E000000000B807550000005500B909AB000034
:1006F00000AB007D06550000005500C80555000000
:10070000005500B807AB000000AB00C8055500005D
:10071000005500DD04550000005500C805550000D7
:10072000005500B8075500000055007D0656010031
:100730000000003F03550000005500FA0C55000072
:100740000055003F03550000005500B90955000051
:100750000055003F035500000055002D09550000CD
:100760000055003F03550000005500EA0A550000FF
:100770000055003F03550000005500B909AB0000CB
:10078000000000534420436172642052656D6F760F
:1007900065640024F404D9201BC40C5C0E9804C4C6
:1007A000095F0265077101F405F900FB04B3004815
:1007B000048700C10369005803550003034500BEC8
:1007C000023A008402310053022A00290225000463
:1007D000022000E4011C00C8011900AF01170098B5
:1007E0000114008401130071011000610110005117
:1007F000010E0043010D0036010B002B010B002000
:10080000010B00150109000C01090003010800FBA0
:10081000000800F3000800EB000700E4000600DE1B
:10082000000600D8000600D2000600CC000500C774
:10083000000500C2000500BD000400B9000400B5B9
:10084000000400B1000400AD000400A9000400A5EC
:10085000000300A20003009F0004009B0003009817
:100860000003009500020093000300900003008D38
:100870000002008B00030088000200860002008452
:10088000000300810002007F0002007D0002007B67
:100890000002007900020077000100760002007477
:1008A00000020072000100710002006F0002006D82
:1008B0000001006C0002006A00010069000200678C
:1008C0000001006600010065000100640002006292
:1008D00000010061000100600001005F0002005D96
:1008E0000001005C0001005B0001005A000100599A
:1008F000000100580001005700010056000100559A
:100900000001005400010053000000530001005298
:1009100000010051000100500001004F0001004E95
:100920000000004E0001004D0001004C0001004B92
:100930000000004B0001004A00010049000100488E
:10094000000000480001004700010046000000468A
:100950000001004500000045000100440001004383
:10096000000000430001004200000042000100417D
:1009700000000041000100400001003F0000003F76
:100980000001003E0000003E0001003D0000003D6F
:100990000001003C0000003C0000003C0001003B66
:1009A0000000003B0001003A0000003A000100395D
:1009B0000000003900010038000000380000003855
:1009C000000100370000003700010036000000364B
:1009D0000000003600010035000000350000003541
:1009E0000001003400000034000000340001003336
:1009F000000000330000003300010032000000322C
:100A00000000003200010031000000310000003120
:100A10000001003000000030000000300001002F15
:100A20000000002F0000002F0000002F0001002E0A
:100A30000000002E0000002E0001002D0000002DFF
:100A40000000002D0000002D0001002C0000002CF3
:100A50000000002C0000002C0001002B0000002BE7
:100A60000000002B0000002B0001002A0000002ADB
:100A70000000002A0000002A0001002900000029CF
:100A800000000029000000290000002900010028C2
:100A900000000028000000280000002800000028B6
:100AA00000010027000000270000002700000027A9
:100AB000000000270001002600000026000000269C
:100AC000000000260000002600010025000000258F
:100AD0000000002500000025000000250000002582
:100AE0000001002400000024000000240000002475
:100AF0000000002400010023000000230000002368
:100B00000000002300000023000000230000002359
:100B1000000100220000002200000022000000224C
:100B2000000000220000002200010021000000213E
:100B30000000002100000021000000210000002131
:100B40000000002100010020000000200000002023
:100B50000000002000000020000000200000002015
:100B6000000000200001001F0000001F0000001F07
:100B70000000001F0000001F0000001F0000001FF9
:100B80000001001E0000001E0000001E0000001EEC
:100B900000000024F4D43050C38E20C2A24017823B
:100BA0008B7011127A910D816CD90AA861E108C786
:100BB000586607615143061E4B5D05C145A7041ADF
:100BC000411104093D9803713931034036DB026558
:100BD000339102D4305402802E1D02632CEE017535
:100BE0002AC501B028A001102781018F2564012B9F
:100BF000244B01E0223401AC211F018D200D018026
:100C00001FFC00841EED00971DDF00B81CD200E61B
:100C10001BC600201BBC00641AB200B219A8000A4F
:100C200019A0006A189900D117910040178B00B5E0
:100C300016840031167E00B31579003A157300C78B
:100C4000146F0058146A00EE1366008813630025C1
:100C5000135E00C7125B006C12570015125400C1DE
:100C600011510070114F0021114B00D61049008D19
:100C70001047004610440002104200C00F400080A0
:100C80000F3E00420F3C00060F3B00CB0E38009396
:100C90000E37005C0E3500270E3400F30D3200C114
:100CA0000D3100900D3000600D2E00320D2D00052D
:100CB0000D2C00D90C2B00AE0C2900850C29005CF2
:100CC0000C2700350C27000E0C2600E80B2400C46E
:100CD0000B2400A00B23007D0B23005A0B210039AD
:100CE0000B2100180B2000F80A1F00D90A1E00BBB8
:100CF0000A1E009D0A1D00800A1D00630A1C004791
:100D00000A1B002C0A1B00110A1A00F7091A00DD41
:100D1000091900C4091900AB091900920917007BD1
:100D2000091800630917004C09160036091600203F
:100D30000916000A091500F5081500E0081400CC92
:100D4000081400B8081400A4081400900813007DCB
:100D50000812006B081300580812004608120034ED
:100D6000081100230811001208110001081100F0F9
:100D7000071000E0071000D0071000C0071000B0F7
:100D8000070F00A107100091070E0083070F0074E2
:100D9000070F0065070E0057070E0049070E003BBE
:100DA000070D002E070E0020070D0013070D00068B
:100DB000070D00F9060C00ED060D00E0060C00D44E
:100DC000060C00C8060C00BC060C00B0060C00A403
:100DD000060B0099060C008D060B0082060B0077AF
:100DE000060B006C060B0061060A0057060B004C50
:100DF000060A0042060A0038060A002E060A0024E7
:100E0000060A001A060A001006090007060A00FD75
:100E1000050900F4050900EB050900E2050900D900
:100E2000050900D0050900C7050900BE050900B580
:100E3000050800AD050800A50509009C05080094FB
:100E40000508008C050800840508007C050800746E
:100E50000508006C050700650508005D05070056DC
:100E60000508004E05070047050700400508003843
:100E7000050700310507002A050700230507001CA8
:100E8000050600160507000F050700080506000205
:100E9000050700FB040600F5040700EE040600E861
:100EA000040600E2040700DB040600D5040600CFB8
:100EB000040600C9040600C3040600BD040600B70A
:100EC000040600B1040500AC040600A6040600A058
:100ED0000405009B04060095040500900406008AA2
:100EE00004050085040500800406007A04050075E9
:100EF000040500700405006B04050066040500612C
:100F00000405005C04050057040500520405004D6B
:100F100004050048040500430405003E0404003AAB
:100F200004050035040500300404002C04050027E6
:100F3000040400230405001E0404001A040400161F
:100F4000040500110404000D040400090405000454
:100F500004040000040400FC030400F8030400F48B
:100F6000030400F0030400EC030400E8030400E4BD
:100F7000030400E0030400DC030400D8030400D4ED
:100F8000030400D0030400CC030400C8030300C51D
:100F90000303009502000000506C656173652077C3
:100FA0006169742E2E2E00840369010000140083F1
:100FB000048800000014008C000000000000000005
:100FC00030F8FFFF00000000000000008E0000006D
:100FD0000000000000000000000000000000000011
:100FE0000057290400188304DC0500001400901F3A
:100FF000891F9502000000506C6561736520776160
:1010000069740084036901000014008304880000EF
:101010000014008C000000000000000030F8FFFF0A
:1010200000000000000000008E0000000000000032
:10103000000000000000000000000000005729042C
:1010400000188304DC05000014008CE537000094D0
:101050001B000000000000000000000000000095E0
:101060000000000046696E64207468652034206BBF
:101070006E6F6273206F6E2000950100000074682F
:101080006520626F74746F6E206F662074686520CF
:101090002020009501000000706C6174666F726D15
:1010A00020616E64207469676874656E009507003E
:1010B0000000666F7572206F722066697665207415
:1010C00075726E732E00950000000049276D206731
:1010D0006F696E6720746F206D6F76652020200029
:1010E0009501000000746865206578747275646508
:1010F0007220746F202020202000950100000076CF
:101100006172696F757320706F736974696F6E7344
:10111000202020009507000000666F722061646A3D
:101120007573746D656E742E009500000000496E35
:10113000206561636820706F736974696F6E2C201D
:10114000202000950100000077652077696C6C20F5
:101150006E65656420746F202020202000950100BA
:10116000000061646A7573742032206B6E6F627365
:10117000206174202020009507000000746865201D
:1011800073616D652074696D652E00950000000027
:101190004E6F7A7A6C657320617265206174207479
:1011A000686520200095010000007269676874205E
:1011B000686569676874207768656E2020200095EF
:1011C00001000000796F752063616E206A75737489
:1011D00020736C69646520610095070000007368E6
:1011E000656574206F6620706170657200950000FF
:1011F00000006265747765656E20746865206E6FA7
:101200007A7A6C652020009501000000616E6420F0
:1012100074686520706C6174652E20202020202069
:1012200000950100000047726162206120736865CB
:101230006574206F662020202020009507000000A4
:10124000706170657220746F2061737369737420AC
:1012500075732E009502000000506C656173652067
:1012600077616974009502000000506C65617365D8
:101270002077616974008EE6370000951B0000D06E
:1012800007000000000000000000009AE9030018B9
:101290008E00000000CAE4FFFFD00700000000003D
:1012A00000000000002A0D3B00188E00000000C95D
:1012B000E4FFFF0000000000000000000000009AB2
:1012C000E9030018950000000041646A75737420FA
:1012D0007468652066726F6E742074776F00950174
:1012E0000000006B6E6F627320756E74696C207005
:1012F000617065722020200095010000006A7573FE
:101300007420736C69646573206265747765656EBB
:10131000200095070000006E6F7A7A6C6520616E80
:101320006420706C617465009502000000506C656B
:101330006173652077616974008E00000000CAE463
:10134000FFFFD007000000000000000000009AE945
:101350000300188E000000007A1A0000D007000079
:10136000000000000000000051812800188E0000DD
:1013700000007A1A000000000000000000000000D9
:1013800000009AE9030018950000000041646A75A6
:10139000737420746865206261636B2074776F20BA
:1013A0000095010000006B6E6F627320756E7469AA
:1013B0006C20706170657220202000950100000093
:1013C0006A75737420736C696465732062657477E1
:1013D00065656E200095070000006E6F7A7A6C6577
:1013E00020616E6420706C617465009502000000DD
:1013F000506C656173652077616974008E00000030
:10140000007A1A0000D00700000000000000000071
:10141000009AE90300188EC624000000000000D0E6
:101420000700000000000000000000A82F220018A4
:101430008EC6240000000000000000000000000034
:1014400000000000009AE903001895000000004128
:10145000646A7573742074686520726967687420A3
:1014600074776F0095010000006B6E6F62732075DA
:101470006E74696C20706170657220202000950187
:101480000000006A75737420736C69646573206270
:1014900065747765656E200095070000006E6F7AB1
:1014A0007A6C6520616E6420706C617465009502D1
:1014B000000000506C656173652077616974008E6F
:1014C000C624000000000000D0070000000000005B
:1014D000000000009AE90300188E3ADBFFFF0000CD
:1014E0000000D007000000000000000000008B7C1E
:1014F0003700188E3ADBFFFF0000000000000000FC
:1015000000000000000000009AE9030018950000A8
:10151000000041646A75737420746865206C6566A8
:10152000742074776F200095010000006B6E6F626D
:101530007320756E74696C20706170657220202054
:101540000095010000006A75737420736C6964650E
:1015500073206265747765656E2000950700000052
:101560006E6F7A7A6C6520616E6420706C61746550
:10157000009502000000506C656173652077616919
:1015800074008E3ADBFFFF00000000D0070000006F
:10159000000000000000009AE90300188E0000001F
:1015A0000000000000D00700000000000000000064
:1015B0000045BE1B00188E00000000000000000067
:1015C00000000000000000000000009AE90300187D
:1015D0009500000000436865636B207468617420A7
:1015E0007061706572202020200095010000006A63
:1015F00075737420736C69646573206265747765B4
:10160000656E200095070000006E6F7A7A6C652089
:10161000616E6420706C61746500891F9502000022
:1016200000506C656173652077616974008403699B
:10163000010000140083048800000014008C0000E6
:1016400000000000000030F8FFFF00000000000074
:1016500000008E00000000000000000000000000FC
:101660000000000000000057290400188304DC0576
:10167000000014008CE5370000941B0000000000FF
:101680000000000000000000009500000000466916
:101690006E64207468652034206B6E6F6273206FF7
:1016A0006E2000950100000074686520626F7474FC
:1016B0006F6E206F66207468652020200095010001
:1016C0000000706C6174666F726D20616E642074CE
:1016D00069676874656E009507000000666F757233
:1016E000206F722066697665207475726E732E00A5
:1016F000950000000049276D20676F696E672074B0
:101700006F206D6F76652020200095010000007429
:10171000686520657874727564657220746F202026
:10172000202020009501000000766172696F7573BA
:1017300020706F736974696F6E73202020009507A5
:10174000000000666F722061646A7573746D656E67
:10175000742E009500000000496E206561636820CA
:10176000706F736974696F6E2C20202000950100E2
:10177000000077652077696C6C206E656564207465
:101780006F202020202000950100000061646A7510
:1017900073742032206B6E6F62732061742020207E
:1017A0000095070000007468652073616D65207402
:1017B000696D652E0095000000004E6F7A7A6C65A9
:1017C0007320617265206174207468652020009523
:1017D0000100000072696768742068656967687451
:1017E000207768656E202020009501000000796F49
:1017F000752063616E206A75737420736C6964650B
:1018000020610095070000007368656574206F66AD
:101810002070617065720095000000006265747749
:1018200065656E20746865206E6F7A7A6C6520201D
:10183000009501000000616E642074686520706C82
:101840006174652E202020202020009501000000DA
:10185000477261622061207368656574206F66203D
:101860002020202000950700000070617065722024
:10187000746F206173736973742075732E00950201
:10188000000000506C656173652077616974009594
:1018900002000000506C6561736520776169740017
:1018A0008EE5370000941B0000D007000000000008
:1018B00000000000009AE90300188E11060000CA1B
:1018C000E4FFFFD00700000000000000000000DA85
:1018D000DF3700188E12060000CAE4FFFF00000088
:1018E0000000000000000000009AE90300189500C5
:1018F00000000041646A7573742074686520667224
:101900006F6E742074776F0095010000006B6E6F2E
:10191000627320756E74696C20706170657220202E
:10192000200095010000006A75737420736C69646F
:101930006573206265747765656E20009507000009
:10194000006E6F7A7A6C6520616E6420706C6174D1
:1019500065009502000000506C6561736520776139
:101960006974008E11060000C9E4FFFFD007000073
:1019700000000000000000009AE90300188E110624
:1019800000007B1A0000D0070000000000000000EB
:10199000000051812800188E110600007A1A0000FC
:1019A0000000000000000000000000009AE90300B1
:1019B00018950000000041646A75737420746865AE
:1019C000206261636B2074776F2000950100000036
:1019D0006B6E6F627320756E74696C2070617065D8
:1019E000722020200095010000006A757374207336
:1019F0006C69646573206265747765656E20009517
:101A0000070000006E6F7A7A6C6520616E6420704A
:101A10006C617465009502000000506C656173652F
:101A20002077616974008E120600007A1A0000D0D7
:101A300007000000000000000000009AE903001801
:101A40008E2A27000000000000D0070000000000E0
:101A50000000000000CFF91F00188E2A27000000A8
:101A60000000000000000000000000000000009ADC
:101A7000E9030018950000000041646A7573742042
:101A80007468652072696768742074776F009501C7
:101A90000000006B6E6F627320756E74696C20704D
:101AA000617065722020200095010000006A757346
:101AB0007420736C69646573206265747765656E04
:101AC000200095070000006E6F7A7A6C6520616EC9
:101AD0006420706C617465009502000000506C65B4
:101AE0006173652077616974008E2927000000000A
:101AF0000000D007000000000000000000009AE98C
:101B00000300188EF9E4FFFF00000000D00700007A
:101B1000000000000000000017F03100188EF9E40A
:101B2000FFFF0000000000000000000000000000B7
:101B300000009AE9030018950000000041646A75EE
:101B4000737420746865206C6566742074776F20E8
:101B50000095010000006B6E6F627320756E7469F2
:101B60006C207061706572202020009501000000DB
:101B70006A75737420736C69646573206265747729
:101B800065656E200095070000006E6F7A7A6C65BF
:101B900020616E6420706C61746500950200000025
:101BA000506C656173652077616974008EF9E4FF9C
:101BB000FF00000000D0070000000000000000004F
:101BC000009AE90300188E1106000000000000D002
:101BD00007000000000000000000000BF8180018CB
:101BE0008E11060000000000000000000000000050
:101BF00000000000009AE90300189500000000436F
:101C00006865636B20746861742070617065722010
:101C10002020200095010000006A75737420736C09
:101C200069646573206265747765656E2000950749
:101C30000000006E6F7A7A6C6520616E6420706CB3
:101C400061746500891F99000000006E6F7A7A6CDC
:101C50006543616C6962726174696F6E0096000021
:101C6000860084033E01000014008304A6000000E7
:101C700014008C000000000000000030F8FFFF009E
:101C8000000000000000008B0000000000000000C9
:101C9000000000000000000000000000A60000009E
:101CA0008304DC0500001400901F8CE537000094CD
:101CB0001B00000000000000000000000000008B7E
:101CC000D1D6FFFF28E5FFFF60EA0000000000001A
:101CD00000000000800000009101149100149104A4
:101CE0001491031488001F026E008D0064005802D6
:101CF00088000302E60088010302E6008700640012
:101D0000580287016400580291017F91007F91047D
:101D10007F91037F8B43E6FFFFB8E9FFFF68010077
:101D2000000000000000000000800000008B43E67F
:101D3000FFFFB8E9FFFF68010000E4FFFFFF0000BC
:101D400000000C0300008B43E6FFFFB8E9FFFFF043
:101D5000000000D0FFFFFF000000003E0000008BED
:101D600043E6FFFFB8E9FFFFF0000000B3FFFFFF0D
:101D700000000000850100008B8DD7FFFFB8E9FF50
:101D8000FFF00000004FFEFFFF000000004A0300CC
:101D9000008B43E6FFFF6EEDFFFFF00000007FFECB
:101DA000FFFF00000000C70000008B43E6FFFF6E4E
:101DB000EDFFFFF000000063FEFFFF000000008564
:101DC0000100008B3BDBFFFF6EEDFFFFF00000002A
:101DD000FEFCFFFF000000004C0300008B43E6FF09
:101DE000FF25F1FFFFF00000002EFDFFFF000000C7
:101DF00000CB0000008B43E6FFFF25F1FFFFF00062
:101E0000000012FDFFFF00000000850100008B3B79
:101E1000DBFFFF25F1FFFFF0000000ADFBFFFF003F
:101E20000000004C0300008B43E6FFFFDCF4FFFFE3
:101E3000F0000000DDFBFFFF00000000CB00000011
:101E40008B43E6FFFFDCF4FFFFF0000000C1FBFF67
:101E5000FF00000000850100008B3BDBFFFFDCF48E
:101E6000FFFFF00000005CFAFFFF000000004C03E1
:101E700000008B43E6FFFF93F8FFFFF00000008DAA
:101E8000FAFFFF00000000CB0000008B43E6FFFFDD
:101E900093F8FFFFF000000070FAFFFF0000000061
:101EA000850100008B3BDBFFFF93F8FFFFF0000094
:101EB000000BF9FFFF000000004C0300008B43E61D
:101EC000FFFF4AFCFFFFF00000003CF9FFFF0000AD
:101ED0000000CB0000008B43E6FFFF4AFCFFFFF051
:101EE0000000001FF9FFFF00000000850100008BCB
:101EF0003BDBFFFF4AFCFFFFF0000000BAF7FFFFEB
:101F0000000000004C0300008B43E6FFFF000000D0
:101F100000F0000000EBF7FFFF00000000CB000026
:101F2000008B43E6FFFF00000000F0000000CEF74A
:101F3000FFFF00000000850100008B3BDBFFFF007E
:101F4000000000F000000069F6FFFF000000004CF8
:101F50000300008B43E6FFFFB6030000F000000023
:101F60009AF6FFFF00000000CB0000008B43E6FF65
:101F7000FFB6030000F00000007DF6FFFF00000048
:101F800000850100008B3BDBFFFFB6030000F00083
:101F9000000019F5FFFF000000004C0300008B4318
:101FA000E6FFFF6D070000F000000049F5FFFF00AD
:101FB000000000CB0000008B43E6FFFF6D07000030
:101FC000F00000002CF5FFFF00000000850100007C
:101FD0008B3BDBFFFF6D070000F0000000C8F3FF44
:101FE000FF000000004C0300008B43E6FFFF240BC2
:101FF0000000F0000000F8F3FFFF00000000CB003D
:1020000000008B43E6FFFF240B0000F0000000DB24
:10201000F3FFFF00000000850100008B3BDBFFFFAA
:10202000240B0000F000000077F2FFFF000000002A
:102030004C0300008B43E6FFFFDB0E0000F00000C6
:1020400000A7F2FFFF00000000CB0000008B43E67A
:10205000FFFFDB0E0000F00000008AF2FFFF00002F
:102060000000850100008B3BDBFFFFDB0E0000F072
:1020700000000026F1FFFF000000004C0300008B71
:1020800043E6FFFF92120000F000000056F1FFFF50
:1020900000000000CB0000008B43E6FFFF9212001F
:1020A00000F000000039F1FFFF0000000085010092
:1020B000008B3BDBFFFF92120000F0000000D5EF29
:1020C000FFFF000000004C0300008B43E6FFFF48C9
:1020D000160000F000000005F0FFFF00000000CB3C
:1020E0000000008B43E6FFFF48160000F0000000F0
:1020F000E8EFFFFF00000000850100008B3BDBFFE5
:10210000FF48160000F000000084EEFFFF00000012
:10211000004C0300008BC0F4FFFFA6F8FFFF68012E
:102120000000B4EEFFFF00000000FE0000008BC0C6
:10213000F4FFFFA6F8FFFFF000000084EEFFFF00B1
:102140000000009C0000008BC0F4FFFFA6F8FFFF1A
:10215000F000000067EEFFFF0000000085010000B6
:102160008BC0F4FFFF5A070000F000000003EDFFF2
:10217000FF000000004A0300008B77F8FFFFA6F87D
:10218000FFFFF000000033EDFFFF00000000C7007C
:1021900000008B77F8FFFFA6F8FFFFF000000016A5
:1021A000EDFFFF00000000850100008B77F8FFFFC6
:1021B000AD030000F0000000B2EBFFFF00000000E4
:1021C0004C0300008B2DFCFFFFA6F8FFFFF0000082
:1021D00000E2EBFFFF00000000CB0000008B2DFCB5
:1021E000FFFFA6F8FFFFF0000000C5EBFFFF0000B7
:1021F0000000850100008B2DFCFFFFAD030000F007
:1022000000000061EAFFFF000000004C0300008BAB
:10221000E4FFFFFFA6F8FFFFF000000091EAFFFFD8
:1022200000000000CB0000008BE4FFFFFFA6F8FFDA
:10223000FFF000000074EAFFFF00000000850100CD
:10224000008BE4FFFFFFAD030000F000000010E989
:10225000FFFF000000004C0300008B9A030000A663
:10226000F8FFFFF000000040E9FFFF00000000CB96
:102270000000008B9A030000A6F8FFFFF0000000AA
:1022800023E9FFFF00000000850100008B9A030096
:1022900000AD030000F0000000BFE7FFFF000000FA
:1022A000004C0300008B51070000A6F8FFFFF00070
:1022B0000000EFE7FFFF00000000CB0000008B51A3
:1022C000070000A6F8FFFFF0000000D2E7FFFF00C4
:1022D000000000850100008B51070000AD030000E5
:1022E000F00000006EE6FFFF000000004C0300005D
:1022F0008B080B0000A6F8FFFFF00000009EE6FF31
:10230000FF00000000CB0000008B080B0000A6F8C7
:10231000FFFFF000000081E6FFFF000000008501E4
:1023200000008B080B0000AD030000F00000001D52
:10233000E5FFFF000000004C0300008BBF0E000013
:10234000A6F8FFFFF00000004DE5FFFF00000000D1
:10235000CB0000008BBF0E0000A6F8FFFFF00000CE
:102360000030E5FFFF00000000850100008BBF0E7C
:102370000000AD030000F0000000CCE3FFFF000010
:1023800000004C0300008B75120000A6F8FFFFF060
:10239000000000FCE3FFFF00000000CB0000008B0A
:1023A00075120000A6F8FFFFF0000000DFE3FFFF5A
:1023B00000000000850100008B75120000AD0300D5
:1023C00000F00000007BE2FFFF000000004C030073
:1023D000008B2C160000A6F8FFFFF0000000ABE217
:1023E000FFFF00000000CB0000008B2C160000A6B1
:1023F000F8FFFFF00000008EE2FFFF000000008504
:102400000100008B2C160000AD030000F00000005E
:102410002AE1FFFF000000004C0300008BE31900DD
:1024200000A6F8FFFFF00000005AE1FFFF000000E7
:1024300000CB0000008BE3190000A6F8FFFFF000BE
:1024400000003DE1FFFF00000000850100008BE37C
:10245000190000AD030000F0000000D9DFFFFF000D
:102460000000004C0300008B9A1D0000A6F8FFFF3F
:10247000F000000009E0FFFF00000000CB000000BA
:102480008B9A1D0000A6F8FFFFF0000000ECDFFFB4
:10249000FF00000000850100008B9A1D0000AD03C5
:1024A0000000F000000088DEFFFF000000004C0389
:1024B00000008B51210000A6F8FFFFF0000000B8DB
:1024C000DEFFFF00000000CB0000008B5121000068
:1024D000A6F8FFFFF00000009BDEFFFF00000000F9
:1024E000850100008B51210000AD030000F00000C9
:1024F0000037DDFFFF000000004C0300008B51217E
:102500000000AD030000F000000067DDFFFF0000E9
:1025100000000C0300008C51210000AD030000F00E
:102520000000000000000000000000860189188BF8
:1025300043E6FFFFF0E9FFFF680100000000000034
:1025400000000000D20000008B43E6FFFFF0E9FF2F
:10255000FF6801000000000000E4FFFFFF0C030023
:10256000008B43E6FFFFF0E9FFFFF00000000000F2
:102570000000D0FFFFFF3E0000008B43E6FFFFF0AE
:10258000E9FFFFF000000000000000B3FFFFFF853F
:102590000100008B4BF1FFFFF0E9FFFFF0000000AE
:1025A000000000004FFEFFFF4C0300008B43E6FFDE
:1025B000FF9EEDFFFFF0000000000000007FFEFF27
:1025C000FFCB0000008B43E6FFFF9EEDFFFFF00016
:1025D00000000000000063FEFFFF850100008B4B40
:1025E000F1FFFF9EEDFFFFF000000000000000FE85
:1025F000FCFFFF4C0300008B43E6FFFF4BF1FFFFA6
:10260000F0000000000000002EFDFFFFCB000000E6
:102610008B43E6FFFF4BF1FFFFF0000000000000DE
:102620000012FDFFFF850100008B4BF1FFFF4BF116
:10263000FFFFF000000000000000ADFBFFFF4C03B7
:1026400000008B43E6FFFFF8F4FFFFF000000000FE
:10265000000000DDFBFFFFCB0000008B43E6FFFF27
:10266000F8F4FFFFF000000000000000C1FBFFFFD6
:10267000850100008B4BF1FFFFF8F4FFFFF0000035
:1026800000000000005CFAFFFF4C0300008B43E6F3
:10269000FFFFA6F8FFFFF0000000000000008DFA29
:1026A000FFFFCB0000008B43E6FFFFA6F8FFFFF023
:1026B0000000000000000070FAFFFF850100008BA1
:1026C0004BF1FFFFA6F8FFFFF00000000000000044
:1026D0000BF9FFFF4C0300008B43E6FFFF53FCFFA9
:1026E000FFF0000000000000003CF9FFFFCB0000FD
:1026F000008B43E6FFFF53FCFFFFF00000000000EB
:1027000000001FF9FFFF850100008B4BF1FFFF5315
:10271000FCFFFFF000000000000000BAF7FFFF4CD4
:102720000300008B43E6FFFF00000000F000000004
:1027300000000000EBF7FFFFCB0000008B43E6FF3B
:10274000FF00000000F000000000000000CEF7FFD6
:10275000FF850100008B4BF1FFFF00000000F0003F
:1027600000000000000069F6FFFF4C0300008B43EF
:10277000E6FFFFAD030000F0000000000000009A3B
:10278000F6FFFFCB0000008B43E6FFFFAD03000028
:10279000F0000000000000007DF6FFFF8501000052
:1027A0008B4BF1FFFFAD030000F0000000000000C4
:1027B0000019F5FFFF4C0300008B43E6FFFF5A07AB
:1027C0000000F00000000000000049F5FFFFCB0012
:1027D00000008B43E6FFFF5A070000F000000000F6
:1027E0000000002CF5FFFF850100008B4BF1FFFF7F
:1027F0005A070000F000000000000000C8F3FFFFCF
:102800004C0300008B43E6FFFF080B0000F00000C4
:102810000000000000F8F3FFFFCB0000008B43E650
:10282000FFFF080B0000F000000000000000DBF3D9
:10283000FFFF850100008B4BF1FFFF080B0000F04C
:102840000000000000000077F2FFFF4C0300008B47
:1028500043E6FFFFB50E0000F0000000000000009E
:10286000A7F2FFFFCB0000008B43E6FFFFB50E0091
:1028700000F0000000000000008AF2FFFF85010068
:10288000008B4BF1FFFFB50E0000F00000000000D0
:10289000000026F1FFFF4C0300008B43E6FFFF62C0
:1028A000120000F00000000000000056F1FFFFCB16
:1028B0000000008B43E6FFFF62120000F000000002
:1028C0000000000039F1FFFF850100008B4BF1FF94
:1028D000FF62120000F000000000000000D5EFFFD2
:1028E000FF4C0300008B43E6FFFF10160000F000D2
:1028F00000000000000005F0FFFFCB0000008B434C
:10290000E6FFFF10160000F000000000000000E8E5
:10291000EFFFFF850100008B4BF1FFFF1016000059
:10292000F00000000000000084EEFFFF4C030000F8
:102930008BF8F4FFFF9EEDFFFF6801000000000030
:1029400000B4EEFFFFC10000008BF8F4FFFF9EED26
:10295000FFFFF00000000000000084EEFFFF9C007D
:1029600000008BF8F4FFFF9EEDFFFFF00000000079
:1029700000000067EEFFFF850100008BF8F4FFFF09
:10298000A6F8FFFFF00000000000000003EDFFFFCD
:102990004C0300008BA6F8FFFF9EEDFFFFF0000048
:1029A000000000000033EDFFFFCB0000008BA6F815
:1029B000FFFF9EEDFFFFF00000000000000016ED9D
:1029C000FFFF850100008BA6F8FFFFA6F8FFFFF0D0
:1029D00000000000000000B2EBFFFF4C0300008B82
:1029E00053FCFFFF9EEDFFFFF00000000000000021
:1029F000E2EBFFFFCB0000008B53FCFFFF9EEDFFDF
:102A0000FFF000000000000000C5EBFFFF850100A3
:102A1000008B53FCFFFFA6F8FFFFF0000000000052
:102A2000000061EAFFFF4C0300008B000000009EE5
:102A3000EDFFFFF00000000000000091EAFFFFCB77
:102A40000000008B000000009EEDFFFFF000000082
:102A50000000000074EAFFFF850100008B00000009
:102A600000A6F8FFFFF00000000000000010E9FFE2
:102A7000FF4C0300008BAD0300009EEDFFFFF00054
:102A800000000000000040E9FFFFCB0000008BAD1C
:102A90000300009EEDFFFFF0000000000000002397
:102AA000E9FFFF850100008BAD030000A6F8FFFFE2
:102AB000F000000000000000BFE7FFFF4C03000033
:102AC0008B5A0700009EEDFFFFF0000000000000A1
:102AD00000EFE7FFFFCB0000008B5A0700009EEDE0
:102AE000FFFFF000000000000000D2E7FFFF8501BB
:102AF00000008B5A070000A6F8FFFFF0000000005E
:102B00000000006EE6FFFF4C0300008B080B000086
:102B10009EEDFFFFF0000000000000009EE6FFFFBA
:102B2000CB0000008B080B00009EEDFFFFF00000C3
:102B3000000000000081E6FFFF850100008B080B0C
:102B40000000A6F8FFFFF0000000000000001DE5F7
:102B5000FFFF4C0300008BB50E00009EEDFFFFF061
:102B6000000000000000004DE5FFFFCB0000008BDF
:102B7000B50E00009EEDFFFFF00000000000000019
:102B800030E5FFFF850100008BB50E0000A6F8FFC1
:102B9000FFF000000000000000CCE3FFFF4C03004A
:102BA000008B621200009EEDFFFFF00000000000AD
:102BB0000000FCE3FFFFCB0000008B621200009ED0
:102BC000EDFFFFF000000000000000DFE3FFFF85E5
:102BD0000100008B62120000A6F8FFFFF000000069
:102BE000000000007BE2FFFF4C0300008B1016008A
:102BF000009EEDFFFFF000000000000000ABE2FFD0
:102C0000FFCB0000008B101600009EEDFFFFF000D0
:102C10000000000000008EE2FFFF850100008B1025
:102C2000160000A6F8FFFFF0000000000000002AD8
:102C3000E1FFFF4C0300008BBD1900009EEDFFFF7C
:102C4000F0000000000000005AE1FFFFCB00000090
:102C50008BBD1900009EEDFFFFF00000000000009A
:102C6000003DE1FFFF850100008BBD190000A6F8C3
:102C7000FFFFF000000000000000D9DFFFFF4C0361
:102C800000008B6B1D00009EEDFFFFF000000000B8
:102C900000000009E0FFFFCB0000008B6B1D00006F
:102CA0009EEDFFFFF000000000000000ECDFFFFFE2
:102CB000850100008B6B1D0000A6F8FFFFF00000EF
:102CC000000000000088DEFFFF4C0300008B18218D
:102CD00000009EEDFFFFF000000000000000B8DEE5
:102CE000FFFFCB0000008B182100009EEDFFFFF0DE
:102CF000000000000000009BDEFFFF850100008B4C
:102D000018210000A6F8FFFFF000000000000000FE
:102D100037DDFFFF4C0300008B18210000A6F8FFF1
:102D2000FF30F200000000000037DDFFFFC50000AB
:102D30000089008800030200008801030200008867
:102D4000001F0200005F002A06FF10000020205430
:102D50006865205265706C696361746F7220202011
:102D600020002020546865205265706C696361748E
:102D70006F722020202000202020202D2D2D2D2D91
:102D80002D2D2D2D2D202020202020002020202022
:102D90002020202020202020202020202020202033
:102DA000004669726D776172652056657273696F4E
:102DB0006E20352E2000436F6F6C210053746172BA
:102DC0007420507265686561742100526967687487
:102DD00020546F6F6C004E4120004F4E20004F4634
:102DE00046004578747275646572004C656674209F
:102DF000546F6F6C00506C6174666F726D00576534
:102E00006C636F6D65212020202020202020202051
:102E1000202049276D20546865205265706C6963D5
:102E200061746F722E205072657373207468652010
:102E3000726564204D20746F202067657420737460
:102E400061727465642120202020202020200057FA
:102E5000656C636F6D6521202020202020202020BC
:102E600020202049276D20546865205265706C69C8
:102E70006361746F722E205072657373207468657D
:102E800020726564204D20746F2020676574207364
:102E9000746172746564212020202020202020008D
:102EA0004120626C696E6B696E6720274D27206D2B
:102EB00065616E7349276D2077616974696E67205B
:102EC000616E642077696C6C636F6E74696E756592
:102ED000207768656E20796F752020207072657389
:102EE000732074686520627574746F6E2E2E2E20A8
:102EF000004120736F6C696420274D27206D656148
:102F00006E7320202049276D20776F726B696E6782
:102F100020616E642077696C6C75706461746520E3
:102F20006D79207374617475732020202077686533
:102F30006E2049276D2066696E69736865642E2E60
:102F40002E004F7572206E657874207374657073EF
:102F50002077696C6C20676574206D6520736574DB
:102F60002075702120202020202046697273742C47
:102F7000207765276C6C20726573746F72656D794C
:102F8000206275696C6420706C6174666F726D2E5E
:102F90002E2E00736F2069742773206E696365207D
:102FA000616E64202020206C6576656C2E2049744B
:102FB00027732070726F6261626C7961206269743C
:102FC000206F66662066726F6D202020202020739F
:102FD00068697070696E672E2E2E202020202020B8
:102FE00020202000416161682C2074686174206693
:102FF00065656C73202020206D75636820626574A0
:103000007465722E20202020202020204C657427FB
:103010007320676F206F6E20616E64206C6F616437
:10302000736F6D652066696C616D656E742120201B
:1030300020202020005765276C6C20747279206155
:103040006761696E21202020202020202020202060
:103050002020202020202020202020202020202070
:103060002020202020202020202020202020202060
:103070002020202020202020202020202020202050
:103080002020202020005765276C6C206B65657020
:1030900020676F696E6720202020616E64206C6F4E
:1030A000616420736F6D65202020202020206669D8
:1030B0006C616D656E742C466F722068656C702053
:1030C000676F746F206D616B6572626F742E636FD2
:1030D0006D2F68656C70005765276C6C20676F20DA
:1030E000746F20746865206D61696E6D656E752EF4
:1030F00020496620796F75206E6565642020206800
:10310000656C7020676F20746F3A2020202020208B
:103110002020206D616B6572626F742E636F6D2F5E
:1031200068656C7020202000417765736F6D6521A4
:103130002020202020202020202020205765276CC0
:103140006C20676F20746F207468652053442020C2
:1031500063617264206D656E7520616E6420796FA5
:103160007520202063616E2073656C656374206137
:10317000206D6F64656C21200049276D20676F69A1
:103180006E6720746F206D616B6520202061207355
:103190006572696573206F66206C696E6573207354
:1031A0006F77652063616E2066696E64206D79209B
:1031B00020202020206E6F7A7A6C6520616C696710
:1031C0006E6D656E742E202020004C6F6F6B206634
:1031D0006F722074686520626573742020206D61B1
:1031E0007463686564206C696E6520696E20656132
:1031F000636861786973207365742E204C696E650D
:103200007320617265206E756D6265726564203130
:103210002D313320616E642E2E2E006C696E652078
:103220006F6E652069732065787472612020206C50
:103230006F6E672E2054686520592061786973206D
:103240007365746973206C656674206F6E20746892
:103250006520706C617465616E64205820617869C6
:10326000732069732072696768742E004772656104
:1032700074212020492776652073617665642020BB
:1032800074686573652073657474696E6773206113
:103290006E64202049276C6C207573652074686506
:1032A0006D20746F202020206D616B65206E696336
:1032B00065206D6F64656C73212020200053656C60
:1032C0006563742062657374206C696E65732E008B
:1032D000582041786973204C696E65002D2D3E00A1
:1032E00020202000592041786973204C696E6500C8
:1032F000446F6E6521004D792074656D7065726153
:10330000747572652077617320206368616E6765EC
:10331000642065787465726E616C6C792E205265DC
:1033200073656C6563742066696C616D656E74208D
:1033300020206D656E7520746F207472792061672E
:1033400061696E2E004D79206578747275646572BE
:103350007320617265202020206E6F742068656183
:1033600074696E672075702E2020202020436865C8
:10337000636B206D79202020202020202020202019
:1033800020636F6E6E656374696F6E7321202020F9
:10339000202020202000507265737320646F776EA8
:1033A000206F6E2074686520202067726579207216
:1033B000696E677320617420746F70206F66746823
:1033C000652065787472756465727320616E64201F
:1033D000202070756C6C2074686520626C61636B72
:1033E0002E2E2E20202000507265737320646F777C
:1033F0006E206F6E207468652020206772657920CA
:1034000072696E6720617420746F70206F6620741B
:10341000686520657874727564657220616E6420D9
:1034200020202070756C6C2074686520626C61636C
:103430006B2E2E2E20202000506C65617365207746
:10344000616974207768696C6520492068656174DA
:10345000206D792065787472756465722120202052
:10346000202020202020202020202020202020205C
:10347000202020202020202020202020202020204C
:10348000202020202020202000677569646520749A
:1034900075626573206F75742E204E6F7766656553
:1034A000642066696C616D656E742066726F6D2054
:1034B00020746865206261636B207468726F756741
:1034C0006820746865747562657320756E74696CC4
:1034D0002069742E2E2E20202000677569646520D7
:1034E00074756265206F75742E20204E6F77666547
:1034F00065642066696C616D656E742066726F6DBF
:103500002020746865206261636B207468726F7537
:103510006768207468657475626520756E74696C7F
:103520002069742E2E2E2020202000706F707320B2
:103530006F757420696E2066726F6E742E2020493C
:10354000276D2068656174696E67207570206D79DC
:10355000202020657874727564657220736F2077FF
:10356000652063616E20206C6F6164207468652043
:1035700066696C616D656E742E2E2E0054686973D9
:10358000206D696768742074616B6520612020205C
:10359000666577206D696E757465732E2020202016
:1035A00020202020416E64207761746368206F754D
:1035B000742C2074686520206E6F7A7A6C65207791
:1035C000696C6C2067657420484F54210048656120
:1035D00074696E672050726F67726573733A20204A
:1035E00020202020202020202020202020202020DB
:1035F00020202020202020202020202020202020CB
:1036000020202020202020202020202020202020BA
:1036100020202020202020202020202020004F4B70
:103620002049276D207265616479212020202020A7
:1036300020204669727374207765276C6C206C6F4C
:103640006164207468657269676874206578747253
:10365000756465722E2020202020507573682066C6
:10366000696C616D656E7420696E2E2E2E20004788
:103670007265617421204E6F77207765276C6C200E
:103680002020206C6F616420746865206C6566740E
:103690002020202020202065787472756465722EA9
:1036A000205075736820202020202066696C616D91
:1036B000656E74207468726F7567682E2E2E2000F8
:1036C0004F4B2049276D20726561647921202020AD
:1036D0002020202050757368207468652066696C0E
:1036E000616D656E742020207468726F7567682E36
:1036F0002E2E2020202020202020202020202020AE
:1037000020202020202020202020202020202020B9
:103710000049276D207265616479212050756C6CB9
:10372000207468652067756964652074756265201A
:103730006F666620616E64202070757368207468FF
:10374000652066696C616D656E74202020746872F6
:103750006F7567682E2E2E2020202020202020200C
:10376000200049276D207265616479212050756CB5
:103770006C2074686520677569646520747562657E
:10378000206F666620616E64202070756C6C2074FA
:1037900068652066696C616D656E742020206765C0
:1037A0006E746C792E2E2E202020202020202020A8
:1037B00020200049276D20726561647921204465CD
:1037C000746163682020207468652067756964658A
:1037D00020747562652C206F70656E746865206C4E
:1037E000657665722061726D20616E6420202070A4
:1037F000756C6C2066696C616D656E7420667265AF
:10380000652E200049276D2072656164792120446E
:103810006574616368202020746865206775696439
:103820006520747562652C206F70656E7468652004
:103830006C657665722061726D20616E6420202057
:1038400070756C6C2066696C616D656E7420667253
:1038500065652E2000756E74696C20796F75206621
:1038600065656C2074686520206D6F746F722074BC
:10387000756720697420696E2E2020202050757392
:103880006820666F72206120666577206D6F7265B3
:10389000207365636F6E64732C207468656E207787
:1038A0006169742E20005768656E2066696C616DD1
:1038B000656E74206973202020206265696E672020
:1038C00065787472756465642066726F6D207468C3
:1038D00065206E6F7A7A6C652C2050726573732048
:1038E0004D20746F2073746F7020657874727564E6
:1038F000696E672E2020005768656E2066696C61CE
:103900006D656E74206973202020206265696E6782
:103910002065787472756465642066726F6D2074BA
:103920006865206E6F7A7A6C652C2020202020201C
:10393000202020507265737320274D2720746F203C
:10394000657869742E2020005768656E206D792097
:1039500066696C616D656E742069732072656C6553
:10396000617365642C20202020202020202020202E
:10397000507265737320274D2720746F2065786916
:10398000742E2020202020202020202020202020D5
:103990002020202020202020005768656E206D798F
:1039A0002066696C616D656E742069732072656C48
:1039B00065617365642C2020202020202020202099
:1039C00020507265737320274D2720746F2065780F
:1039D00069742E202020202020202020202020203C
:1039E00020202020202020202000477265617421A3
:1039F000202049276C6C2073746F70202020727512
:103A00006E6E696E67206D79206578747275646575
:103A1000722E5072657373204D20746F20636F6E29
:103A200074696E75652E2020202020202020202003
:103A300020202020202020202020004F4B21204922
:103A4000276C6C206B656570206D79202020206DBF
:103A50006F746F722072756E6E696E672E20596F6B
:103A60007520206D6179206E65656420746F20700B
:103A7000757368202020206861726465722E2E2E76
:103A80002020202020202020202020005765276C87
:103A90006C206B65657020676F696E672E20202033
:103AA0004C6574732074727920746865206C656647
:103AB0007420202065787472756465722E205075AC
:103AC000736820202020202066696C616D656E740B
:103AD00020646F776E2E2E2E202020200057652721
:103AE0006C6C206B65657020676F696E672E202097
:103AF00020496620796F7527726520686176696E46
:103B0000672020202074726F75626C652C206368BA
:103B100065636B206F757420206D616B6572626FD9
:103B2000742E636F6D2F68656C70202020004D79B6
:103B3000206D6F746F722074696D6564206F757489
:103B4000202061667465722035206D696E7574651C
:103B5000732E202020205072657373204D20746FC7
:103B600020657869742E202020202020202020200D
:103B7000202020202020202020202020202000483D
:103B80006F77276420697420676F3F2052656164F6
:103B900079202000746F206D616B6520736F6D65F7
:103BA0007468696E673F20200059657320202000EB
:103BB0004E6F2020202000446F6573206D79206EA9
:103BC0006F7A7A6C650068656967687420636865F8
:103BD000636B206F75743F004D7920686569676875
:103BE0007420697320676F6F6421004C65742773BC
:103BF0002074727920616761696E2E0044696420C7
:103C0000706C6173746963206578747275646500A3
:103C100066726F6D20746865206E6F7A7A6C653F8E
:103C200000556E6C6F616420726967687400556E30
:103C30006C6F6164004C6F6164206C656674005544
:103C40006E6C6F6164206C656674004C6F616420FB
:103C50007269676874004C6F616400202020202026
:103C60004A6F67206D6F646520202020202020008F
:103C70002020202020202020582B20202020202001
:103C80002020202000202020202020284261636B5B
:103C900029202020592D3E202000202020202020D7
:103CA0002020582D202020202020202020200020EF
:103CB00020202020202020592B20202020202020C0
:103CC0002020200020203C2D5820284261636B29B1
:103CD00020205A2D3E20202000202020202020209F
:103CE00020592D20202020202020202020002020AE
:103CF0002020202020205A2D20202020202020207D
:103D000020200020203C2D5920284261636B29206F
:103D100020202020202020002020202020202020C3
:103D20005A2B202020202020202020200047414DF9
:103D300045204F564552210048656174696E673AC7
:103D400020202020202020202020202000486561E5
:103D500074696E673A00202D2D25006572726F72AE
:103D60002100202020202020202020202020202072
:103D70002020202020200045787472756465723AF6
:103D80002020202D2D2D2F2D2D2D43005220457824
:103D90007472756465723A202D2D2D2F2D2D2D43B3
:103DA000004C2045787472756465723A202D2D2D73
:103DB0002F2D2D2D4300506C6174666F726D3A206B
:103DC00020202D2D2D2F2D2D2D430020204E412044
:103DD0002020200077616974696E6720002F202001
:103DE0002043004320202020002050726568656138
:103DF000742053657474696E6773202020005269C3
:103E000067687420546F6F6C2020202020202020B1
:103E10002020004C65667420546F6F6C2020202099
:103E20002020202020202000506C6174666F726D6D
:103E3000202020202020202000205265736574203F
:103E400053657474696E677320746F20200020447A
:103E5000656661756C742076616C7565733F00559D
:103E60006E506175736520202020202020202020A6
:103E70002020005061757365202020202020202004
:103E80002020202020200043616E63656C20427555
:103E9000696C64202020202020200057616974690B
:103EA0006E6720666F7220486F6D696E67200043F1
:103EB00068616E67652046696C616D656E7420206F
:103EC000202000536C6565702028436F6C6420507F
:103ED00061757365292000526573756D65204275A3
:103EE000696C6420202020202020004C4544204381
:103EF0006F6C6F7220202020202020202020005274
:103F00004544202020004F52414E47452000504953
:103F10004E4B202000475245454E2000424C55450F
:103F2000202000505552504C4500574849544520D8
:103F300000435553544F4D004F4646202020004625
:103F4000696C616D656E742046616E2020202020B2
:103F5000202020004275696C642053746174697379
:103F600074696373202020004261636B20746F20AA
:103F70004D6F6E69746F7220202020004275696C4D
:103F8000642046696E6973686564212020202020C2
:103F90002020202020202020202020202020202021
:103FA000202020204275696C642054696D652020B2
:103FB000202020206820206D004275696C64205408
:103FC000696D653A20202020206820206D004C6912
:103FD0006E653A2020202020202020202020202034
:103FE000202000457374696D6174656420427569B1
:103FF0006C642054696D654C69666574696D6520F3
:10400000546F74616C3A2020202068004C617374F6
:10401000204275696C643A20202020206820206DA1
:104020000043616E63656C20746869732062756912
:104030006C643F00517569742074686973207072F4
:104040006F636573733F004275696C642066726FBD
:104050006D20534420202020202000507265686588
:1040600061742020202020202020202020200055A6
:1040700074696C69746965732020202020202020D9
:10408000202000496E666F20616E64205365747451
:10409000696E67732020004D6F6E69746F72204DDA
:1040A0006F646520202020202020004368616E6717
:1040B000652046696C616D656E7420202020004C7F
:1040C0006576656C204275696C6420506C6174651E
:1040D0002020004A6F67204D6F646520202020203B
:1040E00020202020202000486F6D652041786573D6
:1040F000202020202020202020200052756E2053D8
:104100007461727475702053637269707420004515
:104110006E61626C652053746570706572732020E7
:1041200020200044697361626C652053746570706F
:104130006572732020200053746F7020426C696E8A
:104140006B696E6721202020202000426C696E6B15
:10415000204C454473202020202020202020004394
:10416000616C696272617465204E6F7A7A6C6573F6
:1041700020200065786974206D656E7520202020F0
:1041800020202020202000426F7420537461746925
:10419000737469637320202020200047656E657268
:1041A000616C2053657474696E6773202020005021
:1041B0007265686561742053657474696E677320F5
:1041C00020200056657273696F6E204E756D6265B2
:1041D00072202020202000526573746F7265204485
:1041E000656661756C747320202000536F756E6472
:1041F00020202020202020202020202020200048B7
:10420000656174656420506C61746500546F6F6CF7
:1042100020436F756E742020202020202020200055
:1042200053494E474C45004455414C2020004865B9
:104230006174204C45447320202020202020202021
:1042400020004865617420486F6C64202020202085
:10425000206D2020200048656C7020546578742003
:1042600020202020202020202000416363656C65F1
:1042700072617465202020202020202020004E6FB5
:10428000205344206361726420666F756E6400532E
:104290004420636172642072656164206572726F8C
:1042A0007200492063616E27742072656164207416
:1042B0006869732020205344206361726420666F14
:1042C000726D617421202020202054727920726543
:1042D000666F726D617474696E6720202020746847
:1042E00065206361726420746F2046415431362E1C
:1042F0002000492063616E27742072656164205339
:1043000044200920202063617264732077697468F7
:104310002073746F7261676520206C6172676572CB
:10432000207468616E203247422E202020202020F9
:10433000202020202020202020202020202020207D
:1043400000205344206361726420726561642065BB
:1043500072726F72002049276D20616C7265616412
:1043600079206275696C64696E67005761726E6965
:104370006E673A4275696C64207370656564736634
:104380006173746572207468616E2035306D6D2FB5
:1043900073202072657175697265207833672066B5
:1043A0006F726D61742020666F7220626573742075
:1043B000726573756C74732E202020000100490310
:1043C0003600FF006B00D100A000B800D500A600A9
:1043D0000A0199003F018E0074018400A9017C004C
:1043E000DE01740013026C00480265007D025D006E
:1043F000B2025600E7024E001C03460051033D0086
:1044000086033200BB032200F0030300D0FEC0FF8E
:1044100018FFD0FF63FFE0FFB1FFF0FF00000000D6
:1044200051001000A4002000F800300040014000BE
:10443000A2015000F70160004B0270009F02800053
:10444000F20290004503A0009703B000E803C0000B
:104450003A04D0008C04E000DF04F00032050001D3
:1044600086051001DB0520012F063001DA06500118
:104470003007600186077001DC0780016808900141
:104480002039C9FFE03CE7FFF83F000000000000D2
:1044900008000000200319004006320060094B00AC
:1044A000000A5000800C640000108000FD3B253C99
:1044B000E33FAD49124A6B540E568659F45AC36E07
:1044C00012813B849D8FD5906A916592A693F39556
:1044D00057A238A3F0A687A779A838A974AABBAFBA
:1044E0000CB0BCB385B725D7F5D89ADA88DC43DDA4
:1044F00023DE11241FBECFEFD1E2DEBFCDBF16E019
:10450000A0E0B2E0ECEFF6EC01E00BBF02C00790D8
:104510000D92A438B107D9F71DE1A4E8B6E001C0B7
:104520001D92AA39B107E1F714E4C2EFD4E400E028
:1045300006C022970109FE010BBF0E94EAE2CC3AB5
:10454000D10780E00807A9F70E94FE490C947CE39C
:104550000C940000A0E3B0E0E0EBF2E20C94B5E2D2
:10456000298F3A8F4B8F5C8F6D8F7E8F8F8F98A3A3
:10457000A98ABA8ACB8ADC8AED8AFE8A0F8B188FC9
:10458000098D1A8D2B8D3C8D09A31AA32BA33CA357
:10459000680179018FEF9FEFA0E0B0E0C822D92237
:1045A000EA22FB2289012227332709A71AA72BA772
:1045B0003CA709891A892B893C890DA31EA32FA327
:1045C00038A74801590188229922AA22BB22290131
:1045D00066247724C501B401A70196010E9424E254
:1045E0006DA77EA78FA798ABC301B2010E9424E2FA
:1045F0006B017C01C501B40129A53AA54BA55CA5B9
:104600000E9424E24B015C01C301B2010E9424E23A
:10461000AB01BC01C80CD91CEA1CFB1C0DA51EA5D6
:104620002FA538A9C901AA27BB27C80ED91EEA1E83
:10463000FB1EC814D904EA04FB0420F44050504087
:104640006F4F7F4FC701AA27BB27840F951FA61F57
:10465000B71F8D839E83AF83B8877601DD24CC247A
:104660004DA55EA56FA578A960707070C40ED51EAB
:10467000E61EF71EC982DA82EB82FC821C2D0A81BB
:104680008B804C808D878E818E878F818F878885E8
:10469000888B2D893E894F89588D69A17AA18BA17C
:1046A0009CA10E9424E26B017C012D8D3E8D4F8DDB
:1046B00058A16DA17EA18FA198A50E9424E2DC01E2
:1046C000CB01C80ED91EEA1EFB1E8D859E85AF85C7
:1046D000B8898C0D9D1DAE1DBF1D8D879E87AF8730
:1046E000B88B682F7E85212F302F482D542D8F8534
:1046F0009889E096E0E10C94D1E20F93CF93DF9399
:10470000CDB7DEB760970FB6F894DEBF0FBECDBF52
:10471000002309F456C029873A874B875C876D8749
:104720007E878F87988B20E2201B8D859E85AF85A5
:10473000B889AC01BD011216B4F0770F440B542FA9
:10474000BA014D835E836F837887332727FD3095C9
:10475000309521953F4F04C0B595A79597958795BE
:104760002A95D2F722C0002E04C0759567955795FB
:1047700047950A94D2F74D835E836F83788704C090
:10478000880F991FAA1FBB1F2A95D2F749855A8502
:104790006B857C8504C076956795579547950A95F6
:1047A000D2F7842B952BA62BB72B89839A83AB83C7
:1047B000BC8329813A814B815C816D817E818F81AF
:1047C000988560960FB6F894DEBF0FBECDBFDF911F
:1047D000CF910F910895A8E4B0E0E1EFF3E20C94DB
:1047E000B4E2F50129A33AA34BA35CA36DA37EA376
:1047F0008FA398A7A98EFA8FCB8EDC8EED8EFE8EBE
:104800000F8F18A38DA09EA0AFA0B8A4B7FE67C05D
:104810002195B1E0121608F0B0E03195A1E0131631
:1048200008F0A0E0B32EBB1ABB2D882483943B155F
:1048300008F08824A829419531E0141608F030E0EA
:10484000B42EBA1AAB2D882483944B1508F0882413
:104850003829519541E0151608F040E0452E431ADD
:1048600031E0541508F030E0432B619531E0161625
:1048700008F030E0862E841A41E0681508F040E028
:10488000342B719541E0171608F040E0572F531B69
:1048900031E0751708F030E0432B819531E01816B0
:1048A00008F030E0682F641B462F61E0841708F0A1
:1048B00060E0362B9195931B29A3BAA3ABA34CA21E
:1048C0008DA25EA34FA398A78FEF9FEFAFEFBFEF2F
:1048D00025968CAF9DAFAEAFBFAF259706C025968E
:1048E0001CAE1DAE1EAE1FAE25978D8D9E8DAF8D5D
:1048F000B8A1B7FF68C025962CAD3DAD4EAD5FADFC
:104900002597209530954095509525962CAF3DAF35
:104910004EAF5FAF2597E19581E01E1608F080E06D
:10492000F19591E01F1608F090E04F2F481B81E0B1
:10493000F41708F080E0982BC19481E01C1408F073
:1049400080E06C2D691B91E0C61608F090E0892B81
:10495000D19491E01D1408F090E05D2D581B81E08A
:10496000D51608F080E0982BE19481E01E1408F041
:1049700080E03E2D391B91E0E31608F090E0892B92
:10498000F19491E01F1408F090E02F2D281B81E096
:10499000F21608F080E0982B019581E0101608F0DF
:1049A00080E0702F791B972F71E0091708F070E0F5
:1049B000872B1195181BE98F4A8F6B8F5C8F3D8F6A
:1049C0002E8F9F8F18A3798D6A8D5B8D4C8D3D8DB9
:1049D0002E8D9F8D88A1E9A1E98BEAA1EA8BEBA13D
:1049E000EB8BECA1EC8BEDA1ED8BEEA1EE8BEFA1AF
:1049F000EF8BE8A5E88F79876A875B874C873D87CF
:104A00002E879F87888B89849A84AB84BC848D850C
:104A10009E85AF85B889E988FA880B891C89EDAA3B
:104A2000FEAA0FAB18AFCD88DE88EF88F88C009710
:104A3000A105B10509F0BFC3C814D904EA04FB04F9
:104A400008F04EC100E0801600E0900601E0A006EC
:104A500000E0B00660F41FEF81169104A104B104D8
:104A600009F098F480E090E0A0E0B0E017C020E00A
:104A7000821620E0920620E0A20621E0B20650F461
:104A800080E190E0A0E0B0E009C088E090E0A0E024
:104A9000B0E004C088E190E0A0E0B0E0B501A4017E
:104AA000082E04C076956795579547950A94D2F7D6
:104AB000FA01E25AFD4F208140E250E060E070E0F0
:104AC000481B590B6A0B7B0B421B51096109710989
:104AD0004115510561057105A1F1042E04C0880C32
:104AE000991CAA1CBB1C0A94D2F797018601042EBC
:104AF00004C0000F111F221F331F0A94D2F780E257
:104B000090E0841B950BCDA8DEA8EFA8F8AC04C0FC
:104B1000F694E794D794C7948A95D2F7C02AD12AFD
:104B2000E22AF32A0DA91EA92FA938AD04C0000F4F
:104B3000111F221F331F4A95D2F70DAB1EAB2FABAF
:104B400038AF2501662477249501840120703070E8
:104B500009AB1AAB2BAB3CABC701B601A301920169
:104B60000E9476E22DA73EA74FA758AB69A77AA768
:104B70008BA79CA7C701B601A30192010E9476E210
:104B8000CA01B90129A93AA94BA95CA90E9424E24A
:104B9000AB01BC0109A51AA52BA53CA57801DD2414
:104BA000CC240DA91EA92FA938ADC901AA27BB275E
:104BB000C82AD92AEA2AFB2A0DA51EA52FA538A99D
:104BC000C416D506E606F70638F501501040204019
:104BD000304009A71AA72BA73CA7C80CD91CEA1C70
:104BE000FB1CC814D904EA04FB04D0F0C416D50693
:104BF000E606F706A8F40DA51EA52FA538A90250B4
:104C000010402040304009A71AA72BA73CA7C80C8A
:104C1000D91CEA1CFB1C04C009A71AA72BA73CA798
:104C2000C41AD50AE60AF70AC701B601A301920120
:104C30000E9476E22DA73EA74FA758AB69AF7AAF87
:104C40008BAF9CAFC701B601A30192010E9476E22F
:104C5000CA01B90129A93AA94BA95CA90E9424E279
:104C60006B017C0149AD5AAD6BAD7CAD9A0111274A
:104C700000274DA95EA96FA978AD60707070042BF4
:104C8000152B262B372B8DA59EA5AFA5B8A90C15E6
:104C90001D052E053F05C0F40197A109B109080DB6
:104CA000191D2A1D3B1D081519052A053B0560F035
:104CB0000C151D052E053F0538F48DA59EA5AFA545
:104CC000B8A90297A109B10909A51AA52BA53CA568
:104CD0007801DD24CC24C82AD92AEA2AFB2AB9C4BF
:104CE00081149104A104B10451F461E070E080E00A
:104CF00090E0A50194010E9476E249015A0110E07A
:104D0000811610E0910611E0A10610E0B10660F4F2
:104D10002FEF82169104A104B10409F098F480E009
:104D200090E0A0E0B0E017C030E0831630E09306DA
:104D300030E0A30631E0B30650F480E190E0A0E05B
:104D4000B0E009C088E090E0A0E0B0E004C088E1F5
:104D500090E0A0E0B0E0B501A401082E04C0769573
:104D60006795579547950A94D2F7FA01E25AFD4F95
:104D70002081AC01BD01420F511D611D711D80E2FA
:104D800090E0A0E0B0E0841B950BA60BB70B51F4AC
:104D9000C818D908EA08FB08F1E04F2E512C612C05
:104DA000712C28C1082E04C0880C991CAA1CBB1C9D
:104DB0000A94D2F797018601042E04C036952795F0
:104DC000179507950A94D2F709AB1AAB2BAB3CABFE
:104DD00097018601082E04C0000F111F221F331FE8
:104DE0000A94D2F70DA71EA72FA738ABEDA8FEA8EF
:104DF0000FA918AD04C016950795F794E7944A9546
:104E0000D2F7B801A7010DA51EA52FA538A9042B1F
:104E1000152B262B372B0DA71EA72FA738ABEDA8D8
:104E2000FEA80FA918AD04C0EE0CFF1C001F111F37
:104E30008A95D2F7EDAAFEAA0FAB18AF250166241A
:104E40007724950184012070307009AF1AAF2BAF21
:104E50003CAF69A97AA98BA99CA9A30192010E94E0
:104E600076E229A73AA74BA75CA76B017C0169A949
:104E70007AA98BA99CA9A30192010E9476E2CA019A
:104E8000B90129AD3AAD4BAD5CAD0E9424E2AB0156
:104E9000BC017601DD24CC240DA51EA52FA538A9C3
:104EA000C901AA27BB27C82AD92AEA2AFB2A09A5A9
:104EB0001AA52BA53CA5C416D506E606F70638F5B7
:104EC000015010402040304009AB1AAB2BAB3CAB3B
:104ED000C80CD91CEA1CFB1CC814D904EA04FB0446
:104EE000D0F0C416D506E606F706A8F409A51AA55B
:104EF0002BA53CA5025010402040304009AB1AAB16
:104F00002BAB3CABC80CD91CEA1CFB1C04C009AB86
:104F10001AAB2BAB3CABC41AD50AE60AF70AC70199
:104F2000B601A30192010E9476E229A73AA74BA7F6
:104F30005CA721966CAF7DAF8EAF9FAF2197C70165
:104F4000B601A30192010E9476E2CA01B90129AD1E
:104F50003AAD4BAD5CAD0E9424E28B019C012196E1
:104F60004CAD5DAD6EAD7FAD2197DA0199278827F5
:104F70004DA55EA56FA578A960707070842B952BE8
:104F8000A62BB72B49A55AA56BA57CA58017910721
:104F9000A207B307F0F44150504060407040880DC4
:104FA000991DAA1DBB1D88159905AA05BB0588F08A
:104FB00080179107A207B30760F449A55AA56BA50E
:104FC0007CA54250504060407040880D991DAA1D3C
:104FD000BB1D6C017D01C01AD10AE20AF30A09A9BE
:104FE0001AA92BA93CA9380155244424442A552A3E
:104FF000662A772A8501222733270DA71EA72FA708
:1050000038AB950184012070307009AF1AAF2BAF17
:105010003CAFC701B6012DA53EA54FA558A90E94DA
:1050200076E229A73AA74BA75CA769AB7AAB8BAB13
:105030009CABC701B6012DA53EA54FA558A90E945E
:1050400076E2CA01B90129AD3AAD4BAD5CAD0E9423
:1050500024E2AB01BC0109A91AA92BA93CA978013A
:10506000DD24CC240DA91EA92FA938ADC901AA277A
:10507000BB27C82AD92AEA2AFB2A09A51AA52BA5E3
:105080003CA5C416D506E606F70638F501501040D3
:105090002040304009AB1AAB2BAB3CABC80CD91C41
:1050A000EA1CFB1CC814D904EA04FB04D0F0C416A3
:1050B000D506E606F706A8F409A51AA52BA53CA572
:1050C000025010402040304009AB1AAB2BAB3CAB38
:1050D000C80CD91CEA1CFB1C04C009AB1AAB2BABD7
:1050E0003CABC41AD50AE60AF70AC701B6012DA5DA
:1050F0003EA54FA558A90E9476E229A73AA74BA73B
:105100005CA721966CAF7DAF8EAF9FAF2197C70193
:10511000B6012DA53EA54FA558A90E9476E2CA0169
:10512000B90129AD3AAD4BAD5CAD0E9424E28B01D3
:105130009C0121964CAD5DAD6EAD7FAD2197DA013E
:10514000992788274DA95EA96FA978AD6070707006
:10515000842B952BA62BB72B49A55AA56BA57CA50F
:1051600080179107A207B307D0F441505040604028
:105170007040880D991DAA1DBB1D88159905AA05AB
:10518000BB0568F080179107A207B30740F449A553
:105190005AA56BA57CA5425050406040704009A9BB
:1051A0001AA92BA93CA97801DD24CC24C42AD52A2C
:1051B000E62AF72A51C2C816D906EA06FB0608F401
:1051C00038C2803010E0910711E0A10710E0B1076C
:1051D00058F48F3F9105A105B10509F090F400E066
:1051E00010E020E030E016C0803020E0920720E0A0
:1051F000A20721E0B20750F400E110E020E030E027
:1052000009C008E010E020E030E004C008E110E050
:1052100020E030E0AC01BD01002E04C0769567951A
:10522000579547950A94D2F7FA01E25AFD4F40810B
:10523000040F111D211D311D40E250E060E070E0BF
:10524000401B510B620B730BA1F48C159D05AE0531
:10525000BF0508F4F5C1EDA8FEA80FA918AD4424B8
:1052600055243201E814F9040A051B0508F0EBC1C6
:10527000E3C1342E2C013D0104C0440C551C661CB6
:10528000771C4A95D2F7D501C401002E04C0B6950B
:10529000A795979587950A94D2F7482A592A6A2A9A
:1052A0007B2AA5019401032C04C0220F331F441F45
:1052B000551F0A94D2F729AF3AAF4BAF5CAFB70195
:1052C000A601002E04C076956795579547950A94D8
:1052D000D2F749AB5AAB6BAB7CABC701B601032C21
:1052E00004C0660F771F881F991F0A94D2F76DA715
:1052F0007EA78FA798AB8DA99EA9AFA9B8AD04C012
:10530000B695A795979587950A95D2F74DA55EA571
:105310006FA578A9482B592B6A2B7B2B4DA75EA72D
:105320006FA778AB4301AA24BB24930182012070AC
:10533000307021960CAF1DAF2EAF3FAF219769A9FA
:105340007AA98BA99CA9A50194010E9476E229A7BC
:105350003AA74BA75CA76B017C0169A97AA98BA925
:105360009CA9A50194010E9476E2CA01B901219687
:105370002CAD3DAD4EAD5FAD21970E9424E2DC0126
:10538000CB017601DD24CC240DA51EA52FA538A9BF
:10539000A90166277727C42AD52AE62AF72A09A56C
:1053A0001AA52BA53CA5C816D906EA06FB0638F5B2
:1053B000015010402040304009AB1AAB2BAB3CAB46
:1053C000C40CD51CE61CF71CC414D504E604F70471
:1053D000D0F0C816D906EA06FB06A8F409A51AA556
:1053E0002BA53CA5025010402040304009AB1AAB21
:1053F0002BAB3CABC40CD51CE61CF71C04C009ABA2
:105400001AAB2BAB3CABC81AD90AEA0AFB0AC70194
:10541000B601A50194010E9476E229A73AA74BA7FD
:105420005CA729966CAF7DAF8EAF9FAF2997C70160
:10543000B601A50194010E9476E2CA01B901219644
:105440002CAD3DAD4EAD5FAD21970E9424E24B01E6
:105450005C0129964CAD5DAD6EAD7FAD29979A018B
:10546000112700278DA59EA5AFA5B8A9A070B07083
:10547000082B192B2A2B3B2B89A59AA5ABA5BCA5DC
:10548000081519052A053B05E0F40197A109B109A2
:10549000040D151D261D371D041515052605370598
:1054A00080F0081519052A053B0558F489A59AA529
:1054B000ABA5BCA50297A109B109040D151D261DB8
:1054C000371DB901A801481959096A097B094DA777
:1054D0005EA76FA778AB09A91AA92BA93CA97801E7
:1054E000DD24CC24C82AD92AEA2AFB2AFFEF8F2EF2
:1054F000FFEF9F2EA12CB12C8C209D20AE20BF2031
:1055000087012227332709A71AA72BA73CA749AC55
:105510005AAC6BAC7CAC2FEF3FEF40E050E0422246
:1055200053226422752229AD3AAD4BAD5CAD8A01A0
:105530002227332709AB1AAB2BAB3CABC501B40117
:10554000A30192010E9424E269AF7AAF8BAF9CAFB6
:10555000C501B40129A93AA94BA95CA90E9424E27A
:105560004B015C0169A57AA58BA59CA5A3019201BD
:105570000E9424E22B013C0169A57AA58BA59CA57C
:1055800029A93AA94BA95CA90E9424E2AB01BC015C
:10559000840C951CA61CB71C09AD1AAD2BAD3CADF7
:1055A000C901AA27BB27880E991EAA1EBB1E8414F8
:1055B0009504A604B70420F4405050406F4F7F4F2D
:1055C000C501AA27BB27840F951FA61FB71F0DA5CE
:1055D0001EA52FA538A9081719072A073B0718F198
:1055E00080179107A207B307A1F5540199248824D5
:1055F00089AD9AADABADBCADA070B070880E991EF0
:10560000AA1EBB1E4DA95EA96FA978AD032C04C0CC
:10561000440F551F661F771F0A94D2F74815590586
:105620006A057B05B0F40894C108D108E108F108C7
:1056300010C0442455243201CC24DD2476010CC052
:1056400044245524320181E0C82ED12CE12CF12CC8
:1056500003C0442455243201FE01319688E0DF0165
:105660001D928A95E9F7C982DA82EB82FC824D822B
:105670005E826F8278862C2D3A814B815C81642D0D
:105680007E818F8198852596ECACFDAC0EAD1FAD6B
:105690002597E114F1040105110509F456C021957F
:1056A000E1E0121608F0E0E03195F1E0131608F0A1
:1056B000F0E0032F0E1BE1E0301708F0E0E0FE2BD6
:1056C0004195E1E0141608F0E0E0142F1F1B31E0D3
:1056D000411708F030E0E32B5195F1E0151608F082
:1056E000F0E0B52FBE1B31E05B1708F030E0F32B84
:1056F0006195E1E0161608F0E0E0462E4F1A31E021
:10570000641508F030E0E32B7195F1E0171608F00E
:10571000F0E0A72FAE1B31E07A1708F030E0F32B52
:105720008195E1E0181608F0E0E0F82EFF1AFF2D51
:1057300031E08F1508F030E0E32B9195302F412FA9
:105740005B2F642D7A2F8F2F9E1BC85BDF4FE1E10B
:105750000C94D0E2FA01DC0102C005900D922150B8
:105760003040D8F70895F8942091C8063091C906C2
:105770008091C6069091C706821B930B789408957A
:105780008093BF06089581E08093BD0608958091BF
:10579000BF0608958091BE0608952091C8063091F5
:1057A000C90681E02115310509F080E00895482FF0
:1057B0008091C8069091C9066091C6067091C7068F
:1057C00086179707E8F42091C8063091C9068091A2
:1057D000CA069091CB06820F931F0E944FE2E09180
:1057E000CC06F091CD06E80FF91F40838091C806E2
:1057F0009091C90601969093C9068093C8060895B2
:1058000081E0E6ECF6E0808708951092C9061092D8
:10581000C8061092CB061092CA061092CE061092BD
:10582000CF061092C1061092C2061092C3061092C3
:10583000C4061092C0061092BF061092BE061092C7
:10584000B8061092B9061092BA061092BB061092D2
:10585000A3061092B7061092B6061092B5060895E8
:1058600081E02091B5063091B6062630310509F069
:1058700080E008956091C1067091C2068091C306D0
:105880009091C40608951092C1061092C20610921B
:10589000C3061092C40608954F925F926F927F9252
:1058A0008F929F92AF92BF92CF92DF92EF92FF9230
:1058B0000F931F93CF93DF93CDB7DEB7C656D0407B
:1058C0000FB6F894DEBF0FBECDBFCE018D5B9F4FEC
:1058D0000E948C86A7E8B6E0FE01ED5BFF4F84E1F5
:1058E00001900D928150E1F7CE0101966FE97AE1C6
:1058F00045E00E942EDACE0101960E9477DA80936D
:10590000860687E896E060E070E00E946F56FC0132
:1059100020813181428153816B962CAF3DAF4EAFD8
:105920005FAF6B9787E896E061E070E00E946F568A
:10593000FC0120813181428153816F962CAF3DAFB4
:105940004EAF5FAF6F9787E896E062E070E00E942D
:105950006F56FC012081318142815381A3962CAF87
:105960003DAF4EAF5FAFA39787E896E063E070E08E
:105970000E946F56FC0180809180A280B38083E0FA
:105980000E9490836B017C0187E896E064E070E000
:105990000E946F56FC0160817181828193810E9417
:1059A000BDE02B013C0184E00E9490839B01AC018F
:1059B00000D000D00DB71EB70F5F1F4FC701B60153
:1059C000A4962FAFA497A5963FAFA597A6964FAFE5
:1059D000A697A7965FAFA7970E948FE0DC01CB0147
:1059E000880E991EAA1EBB1EC301B201A4962FAD3C
:1059F000A497A5963FADA597A6964FADA697A79657
:105A00005FADA7970E946DDF0E948AE0DC01CB01A9
:105A1000F80180839183A283B383CE018F966B9626
:105A20004CAD5DAD6EAD7FAD6B976F960CAD1DADA2
:105A30002EAD3FAD6F97A396CCACDDACEEACFFAC1A
:105A4000A3970E9433560F900F900F900F90CE01A6
:105A50008F9648E052E060E070E00E9427878EED6C
:105A600099E00E949FAD90939E0680939D068EE8DC
:105A70009AE00E949FAD9093A00680939F068FE3CB
:105A80009CE00E949FAD90939C0680939B06809122
:105A9000BC06882391F08EED99E060E070E00E94F2
:105AA000CEAC8EE89AE060E070E00E94CEAC8FE36E
:105AB0009CE060E070E00E94CEACDE015B96FE01EF
:105AC000BF9684E101900D928150E1F7CE014B9693
:105AD00062E070E00E946F564C0182E00E94908369
:105AE0000E948AE026E930E040E050E00E9424E293
:105AF000DC01CB01F40180839183A283B383DE01B7
:105B00001796FE017B9684E101900D928150E1F79A
:105B1000CE01079660E070E00E946F564C0180E075
:105B20000E94908320E030E04DED52EC0E94C1E1F4
:105B30000E948AE0DC01CB01F40180839183A2837F
:105B4000B383CE01079661E070E00E946F564C016E
:105B500081E00E94908320E030E044E952EC0E9412
:105B6000C1E10E948AE0DC01CB01F40180839183D2
:105B7000A283B383CE014B964CE850E060E070E026
:105B80000E942787CE01079642E850E060E070E06F
:105B90000E9427878EE999E060E00E943454CA5938
:105BA000DF4F0FB6F894DEBF0FBECDBFDF91CF91B0
:105BB0001F910F91FF90EF90DF90CF90BF90AF902B
:105BC0009F908F907F906F905F904F900895EF928D
:105BD000FF920F931F93CF93DF93CDB7DEB76497F8
:105BE0000FB6F894DEBF0FBECDBFCE0101960E9466
:105BF0008C86CE01019663E070E00E946F567C01B6
:105C000007E816E0C80163E070E00E946F56FC01EF
:105C100080819181A281B381F70180839183A283E6
:105C2000B383CE01019664E070E00E946F567C0160
:105C3000C80164E070E00E946F56FC018081918190
:105C4000A281B381F70180839183A283B383CE01C4
:105C500001960E94FE84CE01019662E070E00E94EF
:105C60006F567C01C80162E070E00E946F56FC0133
:105C700080819181A281B381F70180839183A28386
:105C8000B383CE0101964CE850E060E070E00E94E2
:105C90002787C80142E850E060E070E00E94278753
:105CA0008EE999E0609186060E94345464960FB69E
:105CB000F894DEBF0FBECDBFDF91CF911F910F9142
:105CC000FF90EF90089560919D0670919E068EED75
:105CD00099E00E94CEAC60919F067091A0068EE87C
:105CE0009AE00E94CEAC60919B0670919C068FE377
:105CF0009CE00E94CEAC8FE39CE00E94B5AD88236F
:105D000011F18FE39CE00E94CFAD8823E1F48EED8A
:105D100099E00E94CFAD882341F48EED99E061E0D7
:105D20000E9401AE81E08093C0068EE89AE00E9456
:105D3000CFAD882341F48EE89AE061E00E9401AE85
:105D400081E08093C0060895CF93DF93EB017093B9
:105D50005F0360935E039091BE06981709F44CC0F0
:105D6000882329F1209781F481E08093BC0684E7A1
:105D70009BE06CE171E00E9414B181E090E09093AF
:105D8000A2068093A1060FC06130710561F41092E4
:105D9000BC0684E79BE062E571E00E9414B1D093F9
:105DA000A206C093A10681E08093BE0625C0809123
:105DB000A1069091A2068130910529F41092A206C5
:105DC0001092A10617C08230910529F40E94632E1B
:105DD00084E090E007C08330910549F40E94632E6F
:105DE00085E090E09093A2068093A10605C0623002
:105DF000710511F41092BE06DF91CF910895CF93F3
:105E0000DF93FC0182819381009721F481E08187F7
:105E100080E019C08481958120813181B9010E947F
:105E20004FE2C681D781C80FD91F84819581019621
:105E3000B9010E944FE29583848382819381019707
:105E4000938382838881DF91CF910895EF92FF92AF
:105E50001F93CF93DF9300D0CDB7DEB786ECE82E4B
:105E600086E0F82EC7010E94FF2E682FC7016A83C3
:105E70000E94FF2E782FC70179830E94FF2E182FD2
:105E8000C7010E94FF2E982F6A817981812F0F9080
:105E90000F90DF91CF911F91FF90EF9008951F9386
:105EA000CF93DF93C6ECD6E0CE010E94FF2E182FD1
:105EB000CE010E94FF2E982F812FDF91CF911F914D
:105EC000089586EC96E00E94FF2E08951F93CF93CD
:105ED000DF930E94612F182F0E94612FC82F0E940C
:105EE000612FCA3009F40DC1CB30B0F4C63009F4CB
:105EF00005C1C73050F4C43009F403C1C53008F0FF
:105F000000C1C33009F000C11DC0C83009F4F9C098
:105F1000C93008F0F6C0F2C0CE3009F4F2C0CF307C
:105F200038F4CC3009F486C0CD3008F094C0E9C014
:105F3000C73109F478C0CF3109F498C0CF3009F0E7
:105F4000E3C0DFC0809185068823A1F08EED99E043
:105F50000E94C5AB8EE89AE00E94C5AB8091840692
:105F6000882321F48FE39CE00E94C5AB1092840645
:105F700010928506113019F4C5E7DAE002C0C5ECCD
:105F8000D9E00E944F2FBC01CE0149960E94CEACB1
:105F90008FE39CE00E94B5AD882309F4BCC08FE379
:105FA0009CE00E94CFAD882309F0B5C0113019F4F0
:105FB00085E79AE002C085EC99E049960E94CFAD52
:105FC000882309F0A8C081E08093C006113019F43D
:105FD00085E79AE002C085EC99E0499661E004C04B
:105FE00085E79AE0499660E00E9401AE8EE999E06B
:105FF00061E070E040E00E94964C113009F086C0EC
:106000000E94943D882309F481C08EE999E068E8F4
:1060100071E040E00E94E64F8EE89AE060E070E0B8
:106020000E94CEAC73C09091BF0681E089270E9488
:10603000F5436CC0113019F4C5E7DAE002C0C5ECD5
:10604000D9E00E94612F682F70E061707070CE01FE
:106050000E9426935BC00E94612F682F70E06170E0
:1060600070708EE999E00E94345450C08EE999E036
:1060700061E00E942F5480918506882319F081E009
:10608000809384060E944F2FBC018FE39CE00E9406
:10609000CEAC8FE39CE00E94CFADC1E0C827C09397
:1060A000C0068EED99E06C2F0E9401AE8EE89AE05A
:1060B0006C2F0E9401AE8EE999E061E070E040E053
:1060C0000E94964C0E947C3E882301F50E948443E6
:1060D0008530910539F08EE999E068ED71E040E096
:1060E0000E94E64F8FE39CE060E070E00E94CEAC3F
:1060F0008EE999E060E00E942F5408C00E94262F8C
:1061000005C00E94612F02C080E001C081E0DF91E4
:10611000CF911F910895113009F462CF85EC99E079
:1061200061CF2F923F924F925F926F927F928F92A8
:106130009F92AF92BF92CF92DF92EF92FF920F9316
:106140001F93CF93DF93CDB7DEB7C95AD0400FB6B8
:10615000F894DEBF0FBECDBF0E94EE57882309F52D
:10616000E3C02091C8063091C9068091CA0690917B
:10617000CB06820F931F0E944FE2E091CC06F09174
:10618000CD06E80FF91F40838091C8069091C9069B
:1061900001969093C9068093C80604C00093CE066A
:1061A00001C001E08091C8069091C9062091C60601
:1061B0003091C7062817390711F40C94893B0E94C7
:1061C0005B58882311F40C94893B8091B806909118
:1061D000B906A091BA06B091BB060196A11DB11DEA
:1061E0008093B8069093B906A093BA06B093BB0605
:1061F0000E945E58482F8091C8069091C906609110
:10620000C6067091C7068617970708F4AACFC6CFAF
:10621000C090B806D090B906E090BA06F090BB06E0
:106220000E949D57DC01CB01C816D906EA06FB0681
:1062300010F00C948F3B8091A306882311F00C94EE
:106240008F3B8091B7068F5F8093B706863008F446
:106250006BC084E79BE00E9452B08EE999E069E24E
:1062600072E040E00E94E64F81E08093A3060E9426
:10627000628C1092C9061092C8061092CB0610923A
:10628000CA061092CE061092CF068EED99E060E01D
:1062900070E00E94CEAC8EE89AE060E070E00E9470
:1062A000CEAC8FE39CE060E070E00E94CEACCE010B
:1062B00089579F4F0E94EE85CE0189579F4F62E01C
:1062C00070E00E946F568C0182E00E94908320E073
:1062D00030E046E153E40E94C1E10E948AE0DC0123
:1062E000CB01F80180839183A283B3831092BF0610
:1062F000CE0189579F4F46E950E060E070E00E9470
:1063000027870E946D581092B7060EC08091C8066C
:106310009091C906009741F48091B5069091B60618
:10632000009711F40E946D580E946090882309F52F
:1063300052C02091C8063091C9068091CA0690913A
:10634000CB06820F931F0E944FE2E091CC06F091A2
:10635000CD06E80FF91F40838091C8069091C906C9
:1063600001969093C9068093C80604C00093CE0698
:1063700001C001E08091C8069091C9062091C6062F
:106380003091C7062817390711F40C94973B0E94E7
:106390006990882311F40C94973B0E947790482FC2
:1063A0008091C8069091C9066091C6067091C70693
:1063B0008617970708F4BDCFD9CF8091C806909172
:1063C000C906009741F48091B5069091B6060097F2
:1063D00011F40E94CF908091C006882391F08FE342
:1063E0009CE00E947BAD882361F08EED99E060E037
:1063F0000E9401AE8EE89AE060E00E9401AE109229
:10640000C0068091BF06882311F00C94E33B809175
:10641000BD06882311F00C94E33B8091B506909162
:10642000B6068330910581F40E946084882341F090
:1064300086EA96E00E94BADC882331F00E94628CE2
:106440001092B6061092B5068091B5069091B606E8
:106450008130910541F40E946084882321F41092D8
:10646000B6061092B5068091B5069091B6068230B8
:10647000910551F486EA96E00E94BADC882321F067
:106480001092B6061092B5068091B5069091B606A8
:106490008430910509F04DC086EA96E00E94BADC8E
:1064A000882341F08EE999E06AE772E040E00E94BB
:1064B000E64F3BC08091C506813019F485E79AE02C
:1064C00002C085EC99E049960E947BAD882311F4C7
:1064D0000C949F3B8091C506813019F485E79AE0C2
:1064E00002C085EC99E081579F4FFC018081882391
:1064F00011F00C949F3B87E00E94D45516C085ECA8
:1065000099E049960E94B5AD882399F48091C5061B
:10651000813019F485E79AE002C085EC99E0815753
:106520009F4FFC018081882321F41092B6061092BF
:10653000B5068091B5069091B60685309105F1F4C7
:1065400086EA96E00E94BADC882341F08EE999E061
:106550006FEA72E040E00E94E64F0CC08FE39CE0DF
:106560000E94B5AD882331F08FE39CE00E947BADA3
:10657000882321F01092B6061092B5068091B506D8
:106580009091B6068630910509F03FC086EA96E004
:106590000E94BADC8823B1F08091A40681FF06C076
:1065A0008EE999E060E00E94CE512FC01092B606AD
:1065B0001092B5068EE999E060E170E040E00E943B
:1065C000964C23C084E79BE00E94B4B38823E9F093
:1065D0008091A40682FF04C084E79BE00E9495B1ED
:1065E0008EE999E060E070E040E050E00E94754F75
:1065F0008EE999E060E170E040E00E94964C0E94D4
:1066000057951092B6061092B5068091B5069091F6
:10661000B606009711F00C946B3B8091BE06882360
:1066200009F4E8C08091A1069091A20681309105FD
:1066300011F00C94A93B0E948B6D882311F40C94EB
:10664000A93B80915E0390915F03009729F484E752
:106650009BE064EE72E007C08130910531F484E77D
:106660009BE062E373E00E9414B10E944C2C82E034
:1066700090E082C00E948B6D882311F40C94B23B91
:106680000E94FDAF83E090E09093A2068093A10664
:1066900080E064E10E94818B81E064E10E94818B53
:1066A00080915E0390915F03009711F00C94E33B9F
:1066B00083E064E10E94818B84E064E10E94818B2D
:1066C0000C94E33B0E948B6D882349F48091A106D2
:1066D0009091A2068530910511F00C94BD3B80E0AD
:1066E0006FE70E94818B81E06FE70E94818B809130
:1066F0005E0390915F03009741F483E06FE70E948F
:10670000818B84E06FE70E94818B84E79BE064E6E5
:1067100073E00E9414B11092C50685E090E090935A
:10672000B6068093B50686EA96E040E052ED69E44D
:106730007BE60E9494DC86E090E09093A206809332
:10674000A1068EE999E063E040E024E10E94BE4C9E
:106750000C94E33B1092C50684E090E09093B6065B
:106760008093B50686EA96E040E052ED69E47BE668
:106770000E9494DC87E090E09093A2068093A106AB
:106780000C94E33B87309105A1F481E08093C5062A
:1067900084E090E09093B6068093B50686EA96E092
:1067A00040E052ED69E47BE60E9494DC88E090E0F2
:1067B000E3CF8830910549F48EE999E00E94D44CEA
:1067C0000E94E72D89E090E0D7CF8930910511F044
:1067D0000C94E33B0E948B6D882309F4F4C784E793
:1067E0009BE00E9477B31092A2061092A10610922D
:1067F000BE06E9C78091C8069091C906009709F4C2
:106800006AC78EE999E00E940C4F8091CA06909168
:10681000CB066091C6067091C7060E944FE2E091D8
:10682000CC06F091CD06E80FF91F00810B3839F145
:106830000E3809F4ADC70B3909F4B3C7093809F4A8
:10684000A3C7063909F4A0C7063809F4B3C70C3842
:1068500009F49AC70C3909F497C7003909F494C7A9
:10686000033809F491C7043809F48EC7083809F4CD
:106870008BC70E948B6D882309F086C7A4C78091BF
:10688000C8069091C9068931910508F424C78EE99C
:1068900099E00E940C4F0E94612F81E090E090935C
:1068A000B6068093B5060E94262F4B015C010E941C
:1068B000262F8B019C01C855DF4F2883C85AD04032
:1068C000C755DF4F3883C95AD0400E94262F2B016D
:1068D0003C010E94262FC556DF4F688379838A8347
:1068E0009B83CB59D0400E94262F6B017C010E94D4
:1068F000262FC156DF4F688379838A839B83CF59C4
:10690000D0408091C1069091C206A091C306B0917B
:10691000C4060196A11DB11D8093C1069093C206C5
:10692000A093C306B093C40600D000D0EDB7FEB765
:10693000C182D282E382F482CE01855B9F4FB50192
:10694000A401C855DF4F2881C85AD040C755DF4F32
:106950003881C95AD04073016201C556DF4F888023
:106960009980AA80BB80CB59D0400E9433560F90AB
:106970000F900F900F90CE01855B9F4FC156DF4F58
:10698000488159816A817B81CF59D0400E942787F5
:10699000A2C68EE999E00E940C4F0E94612F81E00F
:1069A00090E09093B6068093B5060E94262F4B0187
:1069B0005C010E94262F8B019C01C855DF4F288364
:1069C000C85AD040C755DF4F3883C95AD0400E94BB
:1069D000262F2B013C010E94262FC556DF4F6883CE
:1069E00079838A839B83CB59D0400E94262F6B01E9
:1069F0007C010E94262FC156DF4F688379838A83EA
:106A00009B83CF59D0400E94612F382E8091C106C0
:106A10009091C206A091C306B091C4060196A11D33
:106A2000B11D8093C1069093C206A093C306B09394
:106A3000C40600D000D0EDB7FEB7C182D282E38297
:106A4000F482CE01C796B501A401C855DF4F288155
:106A5000C85AD040C755DF4F3881C95AD04073015A
:106A60006201C556DF4F88809980AA80BB80CB59D0
:106A7000D0400E9433560F900F900F900F90CE0190
:106A8000C796C156DF4F488159816A817B81CF59B2
:106A9000D040232D0E9412881EC68EE999E00E94E4
:106AA0000C4F0E94612F81E090E09093B606809396
:106AB000B5060E94262F4B015C010E94262F8B01F8
:106AC0009C01C855DF4F2883C85AD040C755DF4FB7
:106AD0003883C95AD0400E94262F2B013C010E94C6
:106AE000262FC556DF4F688379838A839B83CB59D2
:106AF000D0400E94262F6B017C010E94262FC15698
:106B0000DF4F688379838A839B83CF59D0400E946B
:106B1000612FCD55DF4F8883C35AD0400E94262F66
:106B2000CC55DF4F688379838A839B83C45AD040D6
:106B30000E944F2F1C018091C1069091C206A09126
:106B4000C306B091C4060196A11DB11D8093C10674
:106B50009093C206A093C306B093C40600D000D0A1
:106B6000EDB7FEB7C182D282E382F482CE01839672
:106B7000B501A401C855DF4F2881C85AD040C75578
:106B8000DF4F3881C95AD04073016201C556DF4FCB
:106B900088809980AA80BB80CB59D0400E94335610
:106BA0000F900F900F900F90CE018396C156DF4F3C
:106BB000488159816A817B81CF59D040CD55DF4FC3
:106BC0002881C35AD040CC55DF4FE880F9800A8134
:106BD0001B81C45AD04061010E942A897CC50E9451
:106BE000612F0E94612F8093C5064091C10650918C
:106BF000C2066091C3067091C4064F5F5F4F6F4F2E
:106C00007F4F4093C1065093C2066093C3067093B2
:106C1000C4060E94968B5FC58091C8069091C906F4
:106C20008230910508F457C50E94612F0E94612FA0
:106C3000C82E4091C1065091C2066091C306709162
:106C4000C4064F5F5F4F6F4F7F4F4093C106509315
:106C5000C2066093C3067093C4060E948B6D88239E
:106C600009F439C5FC2CFF1CFF24FF1C00E010E0D8
:106C7000DD24C601002E02C0959587950A94E2F79F
:106C800080FF04C0802F6F2D0E94688B0F5F1F4F05
:106C90000530110571F71FC50D3909F04CC0809101
:106CA000C8069091C9068B30910508F414C50E945E
:106CB000612F0E94612F082F0E94612F24E6029FFE
:106CC00090011124280F311D2436310539F08EE949
:106CD00099E069E773E040E00E94E64F0E94612F6F
:106CE0000E94262F0E944F2FF3ED84319F0739F029
:106CF0008EE999E06AEC73E040E00E94E64F0E9462
:106D00004F2F0E94262F0E94262F0E94612F8091D4
:106D1000C1069091C206A091C306B091C406019627
:106D2000A11DB11D8093C1069093C206A093C30616
:106D3000B093C406D0C40C3809F05CC08091C8067A
:106D40009091C9068531910508F4C5C40E94612F50
:106D50000E94262F6B017C010E94262F2B013C01F3
:106D60000E94262F4B015C010E94262FC556DF4F43
:106D7000688379838A839B83CB59D0400E94262FD6
:106D8000AB01BC018091C1069091C206A091C306DF
:106D9000B091C4060196A11DB11D8093C1069093C8
:106DA000C206A093C306B093C40600D000D0EDB7CE
:106DB000FEB74183528363837483CE018D589F4F06
:106DC000B701A6019301820175016401C556DF4F29
:106DD00088809980AA80BB80CB59D0400E943356CE
:106DE0000F900F900F900F90CE018D589F4F0E94E3
:106DF000FE8471C4053871F58091C8069091C9066A
:106E00008530910508F467C482E090E09093B6065F
:106E10008093B5060E94612F0E94262FAB01BC0112
:106E20008091C1069091C206A091C306B091C4069C
:106E30000196A11DB11D8093C1069093C206A09337
:106E4000C306B093C406CB01BA0128EE33E040E09C
:106E500050E078C1043909F049C08091C80690918A
:106E6000C9068530910508F436C40E94612F0E943E
:106E7000612F8093A5060E944F2F8C010E94612FE5
:106E80008093A4068091C1069091C206A091C3068A
:106E9000B091C4060196A11DB11D8093C1069093C7
:106EA000C206A093C306B093C4060115110581F074
:106EB000B80180E090E020E432E44FE050E00E942E
:106EC00024E2AB01BC0186EA96E00E9494DC9EC0FD
:106ED000CE0144960E9490DCA6EAB6E0FE017496CC
:106EE0008FE001900D928150E1F790C0053909F0D3
:106EF000A9C084E79BE00E9478B06C018091C8062D
:106F00009091C9068630910508F4E5C30E94612F6F
:106F10000E94612F082F0E94612F482E0E94612F2E
:106F2000882E0E94612FF82E4091C1065091C20612
:106F30006091C3067091C4064F5F5F4F6F4F7F4FE4
:106F40004093C1065093C2066093C3067093C40673
:106F500010E000FD03C0C6010E9461D3F601428229
:106F60008382C60166EC76E00E94C2D201FFB3C301
:106F7000E091240CFF27E7FDF095EE0FFF1FEA5E7E
:106F8000F34F808191818C159D0531F084E79BE062
:106F9000B6010E9488B003C0C6010E94B0D304703D
:106FA0001070FF2039F00115110521F4C6016F2D75
:106FB0000E949AD30115110509F48DC3FF2089F0B1
:106FC0006F2D70E080E090E020E432E44FE050E08C
:106FD0000E9424E2AB01BC0186EA96E00E9494DCA8
:106FE0000DC0CE0105960E9490DCA6EAB6E0FE0137
:106FF00035968FE001900D928150E1F781E080930A
:10700000A5068091A40684708093A4068EE999E079
:1070100069E170E04FE050E00E94754F84E79BE02B
:107020006091A5060E94AFB38EE999E060E170E03F
:1070300041E00E94964C86E090E09093B6068093E3
:10704000B50649C3802F8358823008F046C080912E
:10705000C8069091C9068830910508F43CC30E9487
:10706000612F0E94612F882E0E94262F6B017C01C8
:107070000E944F2F4091C1065091C2066091C306F5
:107080007091C4064F5F5F4F6F4F7F4F4093C106B3
:107090005093C2066093C3067093C40623E030E0A9
:1070A0003093B6062093B506BC0180E090E020E462
:1070B00032E44FE050E00E9424E2AB01BC0186EADA
:1070C00096E00E9494DC81E0043809F080E0682DAD
:1070D000A70196010E94DA8AFEC20738E1F5809185
:1070E000C8069091C9068630910508F4F4C284E080
:1070F00090E09093B6068093B5060E94612F0E949F
:10710000612F8093C5060E944F2F0E944F2F409100
:10711000C1065091C2066091C3067091C4064F5FCC
:107120005F4F6F4F7F4F4093C1065093C2066093ED
:10713000C3067093C406BC0180E090E020E432E412
:107140004FE050E00E9424E2AB01BC0186EA96E0E9
:107150000E9494DCC0C20D3859F48091C806909109
:10716000C9068630910508F4B6C285E090E0C1CF2B
:107170000F3809F072C08091C8069091C90682301C
:10718000910508F4A8C20E94612F0E94612F4091CE
:10719000C1065091C2066091C3067091C4064F5F4C
:1071A0005F4F6F4F7F4F4093C1065093C20660936D
:1071B000C3067093C40634E2C32E32E0D32E00E03F
:1071C00010E0482E5524E8EE8E2EE3E09E2EA12CF2
:1071D000B12CC201002E02C0959587950A94E2F762
:1071E00080FF30C0CE01815A9F4F0E948C86CE0115
:1071F000815A9F4FB8010E946756FC0160817181DE
:107200008281938169837A838B839C83402F0E9440
:10721000AE8320E030E04AE754E40E94C1E10E94DE
:107220008AE0A50194010E9498E229833A834B8366
:107230005C83F894CE010196B60144E050E00E94D0
:1072400057E378940F5F1F4F84E090E0C80ED91E7B
:107250000530110509F0BDCF3EC2003909F071C0FB
:107260008091C8069091C9068230910508F433C216
:107270000E94612F0E94612F282E8091C10690915B
:10728000C206A091C306B091C4060196A11DB11D0E
:107290008093C1069093C206A093C306B093C40620
:1072A0008E0109571F4FC8010E948C8624E2822E4E
:1072B00022E0922ECC24DD243324F02E012FC101B4
:1072C0000C2C02C0959587950A94E2F780FF28C0A0
:1072D000F8948F2D902FB6010E946F56B40144E0B0
:1072E00050E00E9441E378948F2D902FB6010E94C8
:1072F0006F562C018F2D902FB6010E946F56FC0106
:1073000060817181828193810E94BDE04C2D0E9439
:10731000DB83DC01CB01F20180839183A283B38301
:107320000894C11CD11C84E090E0880E991E95E061
:10733000C916D10421F6CE0189579F4F0E948B8533
:10734000CAC1013949F58091C8069091C9068330B8
:10735000910508F4C0C10E94612F0E94612F082F7F
:107360000E94612F982F4091C1065091C2066091F2
:10737000C3067091C4064F5F5F4F6F4F7F4F4093BE
:10738000C1065093C2066093C3067093C406802F53
:10739000692F0E94818B9FC1023909F045C08091FD
:1073A000C8069091C9068630910508F494C10E94E0
:1073B000612F0E94612FF82E0E94612FC755DF4F69
:1073C0008883C95AD0400E94612FC855DF4F8883F7
:1073D000C85AD0400E94612FC82E0E94612F009190
:1073E000C1061091C2062091C3063091C4060F5FFA
:1073F0001F4F2F4F3F4F0093C1061093C20620939B
:10740000C3063093C4068C2D0E94E9958F2DC75575
:10741000DF4F6881C95AD040C855DF4F4881C85AEC
:10742000D0400E94459557C1033951F58091C80657
:107430009091C9068630910508F44DC10E94612FD4
:107440000E944F2F8C010E944F2F6C010E94612FD0
:107450008091C1069091C206A091C306B091C40666
:107460000196A11DB11D8093C1069093C206A09301
:10747000C306B093C406C801B6010E946F552BC164
:107480000838E1F58091C8069091C90684309105CD
:1074900008F421C18091CA069091CB062091C806BC
:1074A0003091C90603966091C6067091C7060E9486
:1074B0004FE2E091CC06F091CD06E80FF91F8081F4
:1074C00090E004962817390708F405C10E94612F3F
:1074D0008091C1069091C206A091C306B091C406E6
:1074E0000196A11DB11D8093C1069093C206A09381
:1074F000C306B093C4060E94662FEDC0063939F565
:107500008091C8069091C9068330910508F4E3C0C4
:107510000E94612F0E94612F082F0E94612F4091CD
:10752000C1065091C2066091C3067091C4064F5FB8
:107530005F4F6F4F7F4F4093C1065093C2066093D9
:10754000C3067093C406802F0E94E8AFC4C00739F9
:1075500019F58091C8069091C9068230910508F40A
:10756000BAC00E94612F0E94612F4091C1065091C4
:10757000C2066091C3067091C4064F5F5F4F6F4FA4
:107580007F4F4093C1065093C2066093C306709329
:10759000C4060E94D4559FC0083939F58091C806A9
:1075A0009091C9068230910508F495C00E94612F20
:1075B0000E94612F8091C1069091C206A091C306DE
:1075C000B091C4060196A11DB11D8093C106909390
:1075D000C206A093C306B093C4060E94E93D8EE99B
:1075E00099E060E00E94CE5176C0093939F580916A
:1075F000C8069091C9068530910508F46CC00E94B8
:10760000612F0E94262F8091C1069091C206A09101
:10761000C306B091C4060196A11DB11D8093C10699
:107620009093C206A093C306B093C40686EC96E07E
:107630000E945A4481E0809385064DC00A3919F5AD
:107640008091C8069091C9068230910508F443C024
:107650000E94612F0E94612F4091C1065091C20685
:107660006091C3067091C4064F5F5F4F6F4F7F4FAD
:107670004093C1065093C2066093C3067093C4063C
:107680000E94724528C00C3931F58091C80690914E
:10769000C90682309105F8F00E94612F0E94612F87
:1076A0004091C1065091C2066091C3067091C40614
:1076B0004F5F5F4F6F4F7F4F4093C1065093C2069D
:1076C0006093C3067093C40691E0813009F090E0A6
:1076D000892F0E94938B8091C1069091C206A09140
:1076E000C306B091C4068130EAEC9E07EAE9AE0712
:1076F000EBE3BE0708F467C081E09AECAAE9BBE3BC
:107700008093C1069093C206A093C306B093C406AB
:107710005AC00E945B58882311F40C9408310E94CF
:107720005B58882311F40C9486310C9494310E9498
:107730006990882311F40C94DD310C94EB31809125
:10774000C506813011F00C947F3285E79AE00C94E5
:1077500081328091A1069091A2068230910511F4A8
:107760000C943A338091A1069091A2068430910541
:1077700011F00C9466330C9462338630910511F04D
:107780000C94C2330C94AA33093809F085CA44CA50
:107790008091C8069091C9068A31910508F49BCF63
:1077A000F8C88091C8069091C9068032910508F406
:1077B00092CF73C98091C8069091C9068230910515
:1077C00008F00DCA88CFC755DF4F0FB6F894DEBF5B
:1077D0000FBECDBFDF91CF911F910F91FF90EF9022
:1077E000DF90CF90BF90AF909F908F907F906F90E1
:1077F0005F904F903F902F90089580ED98E06DE955
:107800007AE140E00E942EDA80E092E09093C70691
:107810008093C6061092C9061092C8061092CB0635
:107820001092CA0680ED96E09093CD068093CC0628
:107830001092CE061092CF0686EA96E00E9490DC67
:1078400087E896E00E94325608958CEF98E06DE943
:107850007AE140E00E942EDA86ED98E00E9491D90C
:107860000895CF93DF9300D0CDB7DEB7BC0181E0A0
:10787000898382E38A83CE01019642E050E00E9430
:1078800057E30F900F90DF91CF910895CF93DF933F
:10789000EC0140E050E060EE70E40E9438AACE01B6
:1078A000029646E656E666EA7EE30E9438AACE01D4
:1078B000049640E050E060E172E40E9438AADF9153
:1078C000CF9108950F931F93CF93DF938B01EB011B
:1078D0006896009739F4CB0167E00E9461E3CE011E
:1078E0006CE006C0CB0168E30E9461E3CE0160E278
:1078F0000E9461E3C8010A960E94463CC801409676
:107900000E94463CC8014A960E94313CC801069636
:1079100064EF71E00E9477E3C801029665E070E0D1
:107920000E9477E3C801049664EF71E00E9477E358
:10793000C80108966CE271E00E9477E3DF91CF9175
:107940001F910F9108950F931F93CF93DF9300D052
:107950000F92CDB7DEB78C0160E00E9461E3C801F1
:10796000029661E00E9461E38FEF89831B821A8295
:10797000B8016C5F7F4FCE01019643E050E00E945A
:1079800057E30F900F900F90DF91CF911F910F91C0
:107990000895FF920F931F93CF93DF9300D000D0F1
:1079A000CDB7DEB7F82E062F1FB7F89480E491E02C
:1079B00068E04C830E9461E3F9820A834C814B8327
:1079C000CE01019664E471E043E050E00E9457E389
:1079D0001FBF0F900F900F900F90DF91CF911F91CD
:1079E0000F91FF90089561E00E9461E30895CF93A5
:1079F000DF93EC0166EE70E00E9477E3CE01029621
:107A000066EE70E00E9477E3CE0104966EE670E0C9
:107A10000E9477E3CE01069665E00E9461E3DF9164
:107A2000CF9108958EE691E061E00E9461E382E7E4
:107A300091E068EE73E00E9477E384E791E068EEFE
:107A400073E00E9477E386E791E066E970E00E94C8
:107A500077E388E791E060EA7FE00E9477E38AE7D6
:107A600091E060EA7FE00E9477E380E791E060EDDB
:107A700077E00E9477E386E891E060EA7FE00E9489
:107A800077E38CE791E06AE070E00E9477E38EE7AD
:107A900091E06AE070E00E9477E380E891E06AE0BC
:107AA00070E00E9477E382E891E06EE170E00E946E
:107AB00077E384E891E06EE170E00E9477E388ED7F
:107AC00091E042E553E060E070E00E946FE38CEDEE
:107AD00091E044E853E060E070E00E946FE380EEE4
:107AE00091E060E070E00E9477E382EE91E060E078
:107AF00070E00E9477E384EE91E061E00E9461E330
:107B000088E891E060E80E9461E30895CF93CFB7E1
:107B1000F89480E092E062E270E040E150E00E9480
:107B200057E3CFBFCF91089582E490E061E00E94D7
:107B300077A991E0813009F090E0892F08951F9393
:107B4000CF93DF93CDB7DEB764970FB6F894DEBF5F
:107B50000FBECDBFDE011196EFE0F2E084E10190AF
:107B60000D928150E1F70E94943D882381F088E9CD
:107B700090E0A0E0B0E089839A83AB83BC8388E483
:107B800090E0A0E0B0E08D839E83AF83B8871FB7FD
:107B9000F894CE01019664E272E044E150E00E9464
:107BA00057E31FBF64960FB6F894DEBF0FBECDBF7C
:107BB000DF91CF911F910895CF93682FCFB7F8949D
:107BC00082E490E00E9461E30E949F3DCFBFCF918D
:107BD00008951F93CF93DF93CDB7DEB729970FB6E4
:107BE000F894DEBF0FBECDBFDE011596E3E2F2E0F2
:107BF00085E001900D928150E1F70E94863D1FB70C
:107C0000F89481EC93E29A83898384E193ED9C83D9
:107C10008B83CE01059666E070E045E050E00E945F
:107C200057E384E090E06FE90E9461E38CE090E02C
:107C30006BE10E9461E384E492E060E00E9461E312
:107C40000E949F3D85E194E060E172E044E150E0F4
:107C50000E9457E389E294E064EA71E044E150E075
:107C60000E9457E38DE394E066E472E04AE050E05E
:107C70000E9457E30E94123D80EA91E060E070E0CC
:107C80000E9477E382EA91E060E00E9461E380E68F
:107C900091E061E00E9461E388E591E00E94F73C99
:107CA000CE01019664E470E044E050E00E9457E3A6
:107CB00080E090E060E071E00E94623C81E090E052
:107CC0006CE171E00E94623C80E491E00E94A33C80
:107CD0008AE491E00E94F33C86E591E060E00E9436
:107CE00061E31FBF29960FB6F894DEBF0FBECDBF6C
:107CF000DF91CF911F9108958CE490E061E00E94A4
:107D000077A991E0813009F090E0892F0895CF9311
:107D1000CFB7F89480E491E00E94A33C8AE491E01C
:107D20000E94F33C88E591E00E94F73C80E691E0F8
:107D300061E00E9461E38EE691E061E00E9461E310
:107D400081E00E94DC3D84E492E060E00E9461E317
:107D50008CE490E061E00E9461E3CFBFCF91089591
:107D60001F93CF93DF93CDB7DEB72C970FB6F89460
:107D7000DEBF0FBECDBF1FB7F89488EE90E8A0E03D
:107D8000B0E089839A83AB83BC831D821E821F82ED
:107D9000188619861A861B861C86CE01019668E312
:107DA00072E04CE050E00E9457E31FBF2C960FB6E4
:107DB000F894DEBF0FBECDBFDF91CF911F91089524
:107DC000FF920F931F93CF93DF93F82E162F80EA25
:107DD00091E060E070E00E9495A9EC0182EA91E0F8
:107DE00060E00E9477A9180F812F6CE30E9443E2A4
:107DF000092F1D3308F021961FB7F894CF0DD11D20
:107E000080EA91E0BE010E9477E382EA91E0602F70
:107E10000E9461E31FBFDF91CF911F910F91FF90EF
:107E200008951F93CF93DF9300D00F92CDB7DEB7A5
:107E30000E94E93D19821A821B821FB7F89482E0E2
:107E400090E067E10E9461E382E490E061E00E94DB
:107E500061E30E94B03E8CE490E061E00E9461E347
:107E600088E092E061E00E9461E3CE0101966AE061
:107E700072E043E050E00E9457E38EE092E061E759
:107E80000E9461E31FBF0F900F900F90DF91CF9181
:107E90001F9108950F931F93CF93DF93CDB7DEB754
:107EA00027970FB6F894DEBF0FBECDBF19821A8296
:107EB0001B820FB7F89485E194E060E172E044E141
:107EC00050E00E9457E389E294E064EA71E044E103
:107ED00050E00E9457E38DE394E066E472E04AE0EC
:107EE00050E00E9457E30E94123D0E949F3D88E0AF
:107EF00092E061E00E9461E3CE0101966AE072E0E7
:107F000043E050E00E9457E38EE092E061E70E9478
:107F100061E30FBF82E691E040E050E060E070E096
:107F20000E94BBA98B019C0100398CEB180785E5E9
:107F3000280788EA3807C8F4B801C90124E630E008
:107F400040E050E00E9424E228E335E74CE955E0A8
:107F50000E9476E289019A0108511F472F4F3F4F37
:107F60000C831D832E833F8316C0C901B80128E30B
:107F700035E74CE955E00E9476E2CA01B90124E6F2
:107F800030E040E050E00E9424E2DC01CB018C8331
:107F90009D83AE83BF830E94B03E0FB7F894CE019D
:107FA000049668E372E044E050E00E9457E30FBF9C
:107FB00027960FB6F894DEBF0FBECDBFDF91CF91ED
:107FC0001F910F91089582E099E06DE97AE140E018
:107FD0000E942EDA0895CF92DF92EF92FF920F93D4
:107FE0001F93CF93DF93EC018B0188818823E9F104
:107FF0006E01CE0160E00E9479D987FF36C00E94F1
:10800000F157882331F0CE010E94F457C80161E88E
:1080100011C00E94EE57882359F40E946090882373
:1080200039F480912309909124098430910539F520
:10803000C8016AE80E94D9D916C0C6016C2F0E94F7
:1080400079D90E94D72B219603C0C0E0D0E07901F6
:10805000CE15DF0594F3C80161E802C0C80162E8EB
:108060000E94D9D9789481E001C080E0DF91CF915E
:108070001F910F91FF90EF90DF90CF900895F894AB
:10808000C8810E94B32B2C2F30E082179307E8F6AB
:10809000E5CF86E090E0909324098093230981E066
:1080A000809308090895CF93DF93EB0161E00E946C
:1080B0007ED98A31910540F4CE0161E80E94D9D978
:1080C000CE0160E070E007C0CE0161E80E94D9D91E
:1080D000CE016EEB72E00E94DCD9DF91CF91089562
:1080E000CF93DF93EB0161E00E947ED9CE0161E87E
:1080F0000E94D9D9CE016EEB72E00E94DCD9CE018C
:1081000060E070E00E94DCD9CE0161E00E94D9D924
:10811000CE0160E00E94D9D9CE0160E070E00E94FB
:10812000DCD9DF91CF910895DF92EF92FF920F9308
:108130001F93CF93DF937B01CB0161E80E94D9D9D4
:1081400005E219E02FE1D22EE801C701F8016191A3
:108150008F010E94D9D98881882311F0DA94A1F780
:10816000DF91CF911F910F91FF90EF90DF900895D5
:10817000CF93DF93EB01CB0161E80E94D9D90E9434
:10818000B32BAC0160E070E0CE010E94F2D9DF9128
:10819000CF9108950F931F93CF93DF93CDB7DEB7A1
:1081A00064970FB6F894DEBF0FBECDBF8B01F89475
:1081B000CE0101960E948C86C80161E80E94D9D93F
:1081C000CE01019660E070E00E946756FC0140819C
:1081D000518162817381C8010E94F2D9CE0101965A
:1081E00061E070E00E946756FC014081518162812C
:1081F0007381C8010E94F2D9CE01019662E070E05D
:108200000E946756FC014081518162817381C801DF
:108210000E94F2D90E94A58B682FC8010E94D9D96B
:10822000789464960FB6F894DEBF0FBECDBFDF9191
:10823000CF911F910F9108950F931F93CF93DF93C9
:10824000CDB7DEB764970FB6F894DEBF0FBECDBFD3
:108250008B01F894CE0101960E948C86C80161E8DA
:108260000E94D9D9CE01019660E070E00E94675665
:10827000FC014081518162817381C8010E94F2D961
:10828000CE01019661E070E00E946756FC014081DA
:10829000518162817381C8010E94F2D9CE01019699
:1082A00062E070E00E946756FC014081518162816A
:1082B0007381C8010E94F2D9CE01019663E070E09B
:1082C0000E946756FC014081518162817381C8011F
:1082D0000E94F2D9CE01019664E070E00E946756D8
:1082E000FC014081518162817381C8010E94F2D9F1
:1082F0000E94A58B682FC80170E00E94DCD9789499
:1083000064960FB6F894DEBF0FBECDBFDF91CF915C
:108310001F910F9108950F931F93CF93DF93EC015B
:108320008B01CB0161E80E94D9D9CE0103960E944E
:108330003559682FC8010E94D9D9DF91CF911F917B
:108340000F910895CF93DF93EB01CB0161E80E9479
:10835000D9D90E941C58AB01BC01CE010E94F2D9B0
:108360000E947E58DF91CF9108958F929F92AF9295
:10837000BF92CF92DF92EF92FF920F931F93CF9312
:10838000DF93CDB7DEB78C017B018DB69EB6CEB63E
:10839000BDB6AEB6CB0161E80E94D9D9C80161E093
:1083A0000E9479D9882379F00E947459BC01009702
:1083B00051F0C7010E94D9D9C70160E00E94D9D904
:1083C0008DBECEBE34C08DB79EB74F970FB6F89412
:1083D0009EBF0FBE8DBFCDB6DEB60894C11CD11CAA
:1083E000C6016FE140E050E00E94F856BC01F60182
:1083F0008081882329F06115710511F48E3281F393
:10840000C7010E94D9D910E0E12FF0E0C7011F3168
:1084100049F0EC0DFD1D6081662321F00E94D9D941
:108420001F5FF2CF60E00E94D9D9BDBEAEBE0FB6CD
:10843000F8949EBE0FBE8DBEDF91CF911F910F911C
:10844000FF90EF90DF90CF90BF90AF909F908F9074
:108450000895CF93DF93EB01CB0161E80E94D9D956
:10846000F8940E948B6D882361F00E94CD2B8823A5
:1084700041F061E0CE010E94D9D97894DF91CF918B
:10848000089560E0F7CF6F927F928F929F92AF92A4
:10849000BF92CF92DF92EF92FF920F931F93CF93F1
:1084A000DF93CDB7DEB7A82EE92E6B016DB67EB691
:1084B00061E00E947ED98C018A2D9E2D63E00E948E
:1084C00079D9482F882E99248DB79EB78819990994
:1084D0000FB6F8949EBF0FBE8DBFADB6BEB6089462
:1084E000A11CB11CEFB6F894C501B80150E00E9480
:1084F00041E3EFBEC60161E80E94D9D9750100E0F1
:1085000010E008C0F70161917F01C6010E94D9D92E
:108510000F5F1F4F08151905ACF30FB6F8947EBE18
:108520000FBE6DBEDF91CF911F910F91FF90EF9025
:10853000DF90CF90BF90AF909F908F907F906F9083
:1085400008952F923F925F926F927F928F929F92A7
:10855000AF92BF92CF92DF92EF92FF920F931F9351
:10856000CF93DF9300D0CDB7DEB7E82ED92E3B01F5
:108570008DB79EB79A8389838E2D9D2D61E00E94D1
:108580007ED9C82EB92E8E2D9D2D63E00E9479D9FB
:10859000F82E282E3324EDB7FEB7E219F3090FB6F3
:1085A000F894FEBF0FBEEDBF0DB71EB70F5F1F4F94
:1085B0008FB6F894A02E512EC8016C2D7B2D4F2D17
:1085C00050E00E9441E38FBE480100E010E00BC084
:1085D000602F6C5F8E2D9D2D0E9479D9F4018193BF
:1085E0004F010F5F1F4F0215130594F30FB7F89457
:1085F0008A2D952D6C2D7B2D4F2D50E00E9457E339
:108600000FBFC30161E80E94D9D9C3016F2D0E9439
:10861000D9D989819A810FB6F8949EBF0FBE8DBFBC
:108620000F900F90DF91CF911F910F91FF90EF90DE
:10863000DF90CF90BF90AF909F908F907F906F9082
:108640005F903F902F9008950F931F93CF93DF93E8
:10865000EB0161E00E9479D9082F80FF02C00E94DF
:10866000628C01FF02C00E94052CCE0161E80E94CD
:10867000D9D9CE0160E00E94D9D9DF91CF911F9165
:108680000F910895CF93DF93EC0161E80E94D9D94F
:10869000CE016091BF0C0E94D9D9DF91CF9108958E
:1086A0000F931F93CF93DF9380914409882379F42C
:1086B00004E419E0C2E2D0E0CE0160E00E9477A9B4
:1086C000F80181938F012196C233D105A9F78091DA
:1086D0004409882379F4A4E4B9E080E090E0FC0147
:1086E000E85EFB4FE491ED9301968E309105B9F76A
:1086F0001092520984E499E0DF91CF911F910F917C
:10870000089585E299E008958091230990912409C4
:108710000895CF93DF9385E299E00E94F758EC012A
:10872000009789F40E94052C0E94628C0E94738C31
:108730008EE999E060E00E94CE5182E090E0909353
:10874000240980932309CE01DF91CF910895CF9220
:10875000DF92EF92FF920F931F93CF93DF936C0101
:108760007B01CB0161E80E94D9D905E219E0C1E0A3
:10877000D0E008C0C6016C2F0E9479D9F80181931E
:108780008F012196F601808190E0C817D90794F3F4
:10879000109243090E948943682FC7010E94D9D9CA
:1087A000DF91CF911F910F91FF90EF90DF90CF90CD
:1087B00008950E9494908823B9F085E090E090930A
:1087C00024098093230984E79BE00E947AB08EE914
:1087D00099E064E070E041E00E94964C0E94052C14
:1087E0000E94628C0E94738C0895CF93C82F0E94C0
:1087F000C72BC817D1F08C2F0E94C02BCC2351F06F
:1088000083E090E090932209809321098BE099E026
:1088100061E009C081E090E09093220980932109F2
:108820008BE099E060E00E94EADCCF910895CF935D
:10883000DF93EB010E94C72B91E089270E94F5434B
:10884000CE0161E80E94D9D9DF91CF9108951F939D
:10885000CF93DF93182FEB010E94CA2B1817D9F082
:10886000112351F025E030E03093220920932109B3
:108870008BE099E061E009C021E030E0309322090B
:10888000209321098BE099E060E00E94EADC812FCF
:10889000BE010E94A42EDF91CF911F9108958BE01D
:1088A00099E040E054EA63E976ED0E9494DC10928E
:1088B0001A090895DF92EF92FF920F931F93CF93BF
:1088C000DF93CDB7DEB76F970FB6F894DEBF0FBE5C
:1088D000CDBFFC018091230990912409813091053D
:1088E00009F44EC08230910524F4009709F442C087
:1088F00076C08230910529F08530910509F06FC06E
:108900003FC07E010894E11CF11C4FE1DD24D394AB
:1089100082819381009719F4D18680E01AC0848106
:10892000958120813181B9010E944FE20681178132
:10893000080F191F848195810196B9010E944FE2A9
:108940009583848382819381019793838283D80165
:108950008C91D7018D937D01882309F458C0415033
:10896000B9F655C085E299E0BE016F5F7F4F0E9466
:1089700012E335C081E090E09093240980932309AD
:1089800035E2E32E39E0F32E4FE1DD24D3948281EA
:108990009381009719F4D18680E01AC08481958173
:1089A00020813181B9010E944FE206811781080FB1
:1089B000191F848195810196B9010E944FE2958328
:1089C000848382819381019793838283D8018C91E0
:1089D000D7018D937D01882311F04150C1F60E948B
:1089E0004F440E94432C81E090E0909322098093B1
:1089F00021096F960FB6F894DEBF0FBECDBFDF9191
:108A0000CF911F910F91FF90EF90DF900895CE01CD
:108A1000019668E272E00E9409E3009701F3A2CF99
:108A20008BE099E00E94BADC882369F08BE099E042
:108A300040E054EA63E976ED0E9494DC80911A09E3
:108A40008F5F80931A090895CF93DF93FC01EB01A8
:108A500080910B09882339F48091200980838091CB
:108A60001F0988830EC080911A0980838BE099E0EA
:108A70000E9419DD20E037E843E953E00E9476E2E6
:108A80002883DF91CF910895CF93DF93CDB7DEB7E1
:108A90002F970FB6F894DEBF0FBECDBF80E299E0EE
:108AA0006FE179E00E9424458091200960911F09BF
:108AB0000E94E03ECE0101960E9490DCABE0B9E05E
:108AC000FE0131968FE001900D928150E1F71092F6
:108AD0001A092F960FB6F894DEBF0FBECDBFDF91F7
:108AE000CF910895CF93DF9300D000D000D0CDB7C1
:108AF000DEB784E79BE061E070E00E94E8B00E948E
:108B000044450E943A2CDC01CB0180931B099093D1
:108B10001C09A0931D09B0931E0982E090E0909378
:108B2000220980932109109224091092230983E0DD
:108B300060E00E94688B84E060E00E94688BCE0158
:108B400001966FE97AE145E00E942EDACE010196A6
:108B500060E00E9486DA26960FB6F894DEBF0FBE5C
:108B6000CDBFDF91CF9108950F931F93CF93DF93E4
:108B7000CDB7DEB766970FB6F894DEBF0FBECDBF98
:108B8000809123099091240901978230910508F082
:108B900077C00E94628C83E060E00E94688B84E072
:108BA00060E00E94688B8EE999E060E270E041E04D
:108BB0000E94964C0E943A2CDC01CB0180931B0949
:108BC00090931C09A0931D09B0931E090E9444456F
:108BD00081E062E070E00E94A42ECE010296BE0108
:108BE0006F5F7F4F0E9424450E949A8F082F882331
:108BF00009F446C0CE0103960E94EE85CE0103968D
:108C000062E070E0013059F40E946F568C0182E0FE
:108C10000E94908320E030E041E153E40AC00E94CA
:108C20006F568C0182E00E94908320E030E046E1A4
:108C300053E40E94C1E10E948AE0DC01CB01F8010B
:108C400080839183A283B38380E00E94C02BCE01F6
:108C5000039646E950E060E070E00E94278784E7D1
:108C60009BE067E274E00E9414B181E08093290CDC
:108C700084E599E040E856E968E970E00E9494DCF8
:108C8000809123099091240981309105C1F480914C
:108C90002109909122098430910589F084E090E0C7
:108CA000909324098093230981E08093080983E647
:108CB00099E040E452E46FE070E00E9494DC8EE9B9
:108CC00099E064E070E040E00E94964C81E080937F
:108CD0000A0984E090E09093220980932109669626
:108CE0000FB6F894DEBF0FBECDBFDF91CF911F91BD
:108CF0000F9108950F931F93CF93DF9300D0CDB7BB
:108D0000DEB78C0161E80E94D9D9CE010296BE017E
:108D10006F5F7F4F0E942445C801609121090E9426
:108D2000D9D9C8016A810E94D9D9C80169810E9434
:108D3000D9D980912109909122098130910531F092
:108D40008330910519F08530910529F40E943A2C61
:108D5000AB01BC0108C040911B0950911C096091F6
:108D60001D0970911E09C8010E94F2D9C80140E096
:108D700050E060E070E00E94F2D90F900F90DF9118
:108D8000CF911F910F910895EF92FF920F931F9330
:108D9000CF93DF937C018B01FC018081882309F450
:108DA000F7C0C70161E00E9479D9C82FC70162E00E
:108DB0000E9479D9803209F44AC0813268F4823045
:108DC00019F1833018F48823B9F0E2C0863149F1F3
:108DD0008E3109F0DDC032C0833209F44EC08432D6
:108DE00020F4813209F0D4C03FC0843209F44FC06E
:108DF000853209F0CDC084C0C80161E80E94D9D98C
:108E0000C8016EEB72E0C0C0C80161E80E94D9D908
:108E1000C13019F485E79AE002C085EC99E04996E3
:108E200013C0C80161E80E94D9D9C13019F485E79F
:108E30009AE002C085EC99E0499625C0C80161E836
:108E40000E94D9D98FE39CE00E94A5AD9BC0C801C8
:108E500061E80E94D9D9C13019F485E79AE002C0CF
:108E600085EC99E0499606C0C80161E80E94D9D90D
:108E70008FE39CE00E949FAD85C0C80161E80E941D
:108E8000D9D98FE39CE00E947BAD682F35C0C80123
:108E900061E80E94D9D9C13019F485E79AE002C08F
:108EA00085EC99E049960E94B1AF882311F0D0E893
:108EB00001C0D0E08FE39CE00E94B1AF882311F0A5
:108EC00080E401C080E0D82BC13019F485E79AE036
:108ED00002C085EC99E049960E94B6AFD82BC1300C
:108EE00019F425E73AE002C025EC39E0C9014996BA
:108EF0000E947BAD6D2F682BC8010E94D9D946C056
:108F0000C80161E80E94D9D9C13019F485E79AE017
:108F100002C085EC99E049960E94A9ADBC01C80148
:108F20000E94DCD9C13019F485E79AE002C085ECD3
:108F300099E049960E94ADADBC01C8010E94DCD900
:108F4000C13019F485E79AE002C085EC99E04996B2
:108F50000E94B1ADBC01C8010E94DCD98FE39CE046
:108F60000E94A9ADBC01C8010E94DCD98FE39CE03E
:108F70000E94ADADBC01C8010E94DCD98FE39CE02A
:108F80000E94B1ADBC01C8010E94DCD981E001C0E2
:108F900080E0DF91CF911F910F91FF90EF900895A6
:108FA0000F931F93CF93DF93EC018B01888188236C
:108FB00009F491C0CE0160E00E9479D987FD8BC091
:108FC000E82FF0E0EC31F10508F085C0EE58FF4FD6
:108FD000EE0FFF1F0590F491E02D0994CE01B8012A
:108FE0000E94534076C0CE01B8010E94944071C0E7
:108FF00080912309909124099C0121503040223016
:10900000310518F08530910579F484E090E0909373
:109010002209809321090E94B4458EE999E064E019
:1090200070E00E943E4F03C081E080930A09C801AE
:1090300061E80E94D9D94DC0CE01B8010E94B84064
:1090400048C0CE01B8010E94CA4043C0CE01B80159
:109050000E941C413EC0CE01B8010E948B4139C024
:10906000CE01B8010E94A24134C0CE01B8010E94D5
:10907000A7432FC0CE01B8010E94B5412AC0CE013E
:10908000B8010E94174425C0CE01B8010E94C44611
:1090900023C0CE01B8010E9429421BC0CE01B801F5
:1090A0000E94434216C0CE01B8010E94A14211C0E5
:1090B000CE01B8010E9424430CC0C8010E94424363
:1090C00008C0C8010E947A4604C0CE01B8010E94BF
:1090D000704081E001C080E0DF91CF911F910F913E
:1090E0000895CF93DF93CDB7DEB7AD970FB6F89461
:1090F000DEBF0FBECDBF8091841D9091851D00976E
:1091000009F415C18091841D9091851D84309105CD
:1091100009F01AC10CC180910809882339F083E64F
:1091200099E00E94BADC882309F406C180915409B1
:10913000882359F084E599E00E94BADC882329F459
:109140000E948B6D882309F4F7C0809121099091CA
:1091500022098130910531F08330910519F0853075
:10916000910541F484E090E09093220980932109D5
:109170000E94B44510920A0910920809CE014F9638
:109180000E9490DCA3E6B9E0FE017F968FE001909B
:109190000D928150E1F7CE0140960E9490DCA4E54B
:1091A000B9E0FE0170968FE001900D928150E1F7D9
:1091B000809109090E94C54910920909CE010196C2
:1091C0000E9490DCA2E7B9E0FE0131968FE00190A9
:1091D0000D928150E1F710924409109225091092E6
:1091E000240910922309B0C080915E1D90915F1DEB
:1091F00084309105D1F080917209882349F482E787
:1092000099E040E45DE063E070E00E9494DC0DC012
:1092100082E799E00E94BADC882339F08BE39DE174
:109220000E9416D984E080935D1D80915D1D882386
:1092300021F08BE39DE10E9424D980915E1D9091E5
:109240005F1D8430910509F04AC082E799E00E94D1
:10925000E4DC81E69DE10E9499D9809123099091F7
:109260002409209108098630910561F481E69DE189
:10927000222331F069E80E94D9D91092080927C049
:109280006BE823C0222371F081E69DE169E80E942A
:10929000D9D9109208098EE999E066E070E00E9441
:1092A0003E4F15C08BE39DE161E67DE10E94EB3FFF
:1092B000882369F48BE39DE161E67DE10E94D0475C
:1092C000882329F481E69DE165E80E94D9D98BE3E2
:1092D0009DE10E9424D987E39DE10E9472DD809187
:1092E0002309909124098230910541F40E94EE57A0
:1092F000882321F4109224091092230980912309D4
:10930000909124098530910579F40E94609088231A
:1093100021F410922409109223098EE999E064E067
:1093200070E040E00E94964C0E9410450DC0809174
:109330000A09882309F0EFCE80915E1D90915F1D90
:10934000009709F051CF71CFAD960FB6F894DEBFFC
:109350000FBECDBFDF91CF91089581E899E06DE90F
:109360007AE140E00E942EDA82E799E00E9490DCE8
:1093700083E699E00E9490DC84E599E00E9490DC0D
:109380008BE099E00E9490DC0895CF93DF930F92D9
:10939000CDB7DEB7682FF89484B76623A1F088E1D3
:1093A0000FB6F89480936000109260000FBE14BE58
:1093B00089E228E130E00FB6F894A8952093600088
:1093C0000FBE8093600069830E947E580E9477548C
:1093D0000E9463900E94052C0E9440A90E94E08494
:1093E0000E94628C0E94738C8EE999E069810E94D0
:1093F000CE5178940F90DF91CF9108958EE999E046
:109400000E94644B81E00E94C54978940E94714893
:109410000E9491308EE999E00E9404500E94C35549
:10942000A895F4CF87E899E06DE97AE140E00E94E1
:109430002EDA08950F931F93CF93DF9300D000D0BF
:1094400000D0CDB7DEB7062F1FB7F894CE01019636
:109450006FE97AE144E00E942EDA61E0002309F42A
:1094600060E0CE0101960E9486DA1FBF26960FB6F5
:10947000F894DEBF0FBECDBFDF91CF911F910F914A
:1094800008958F929F92AF92CF92EF92FF920F9397
:109490001F93CF93DF93CDB7DEB7E6970FB6F8945F
:1094A000DEBF0FBECDBF4C0104960E9490DCC4010C
:1094B00043960E9490DCCE01C19665EA7AE143E0D2
:1094C0000E942EDACE018B9665EA7AE144E00E9492
:1094D0002EDACE0185966BEA7AE143E00E942EDA1D
:1094E000C401879660E0AE014F5C5F4F9E01255D31
:1094F0003F4F8E010B5D1F4FE12CE1E0FE2E0E94DD
:109500006D92CE014F9661EB7AE145E00E942EDA32
:10951000CE01499661EB7AE146E00E942EDACE0157
:1095200043966BEA7AE144E00E942EDAC401895244
:109530009F4F61E0AE01415E5F4F9E01275E3F4F4E
:109540008E010D5E1F4FFCE1EF2EF1E0FF2E0E9419
:109550006D92C40189579E4F0E9490DCC4018A56C7
:109560009E4F0E9490DC84010B551E4FC80102964D
:109570000E9490DCAAEBEA2EA1E0FA2EE80CF91C7E
:10958000CE010D966FEA7AE144E00E942EDACE0118
:1095900007966FEA7AE143E00E942EDACE01019647
:1095A0006FEA7AE142E00E942EDAC701BE01635FF2
:1095B0007F4FAE01495F5F4F9E012F5F3F4F0E947B
:1095C000F2B3C4018A529E4FB801A7010E9415B0A0
:1095D000840103571D4FC8016FE040E00E94BBDBD0
:1095E000A40141565D4F8BE494E0FA01918380839E
:1095F000C4018F559D4FB80100E513EC20E030E029
:10960000B0E1EB2EB1E0FB2ECC24A2E0AA2E0E940A
:109610007FAB8CE490E061E00E9477A9F401E55E05
:10962000FC4F91E0882309F490E09083E6960FB612
:10963000F894DEBF0FBECDBFDF91CF911F910F9188
:10964000FF90EF90CF90AF909F908F9008950E94E1
:10965000BF54109220018AE08093210110922201D0
:1096600080E090E2909329018093280182E080932A
:1096700073008093B00094E09093B10099E19093CF
:10968000B3001092B4008093700091E0909380003A
:109690008BE08093810010928900109288001092D4
:1096A0008B0010928A0010926F009093A00080931C
:1096B000A1001092A9001092A8001092AB00109285
:1096C000AA00109272000895CF92DF92EF92FF925B
:1096D0000F931F93CF93DF93CDB7DEB7E0970FB60D
:1096E000F894DEBF0FBECDBF8C0183E69DE00E94E3
:1096F000155A0E94C3AFF80186A31082118212820C
:109700001382C8010E94274BB1EBCB2EBAE1DB2EAE
:10971000CE018B96B60147E00E942EDACE018B96E1
:1097200061E00E9463DA2FEAE22E2AE1F22ECE01F6
:109730008596B70141E00E942EDACE01859661E060
:109740000E9463DACE014F96B70140E00E942EDA04
:10975000CE014F9661E00E9463DA37EAE32E3AE1E8
:10976000F32ECE014996B70141E00E942EDACE01D8
:10977000499661E00E9463DACE014396B60147E064
:109780000E942EDACE01439661E00E9463DACE0198
:109790000D96B70140E00E942EDACE010D9661E0F1
:1097A0000E9463DACE01079661EA7AE146E00E9400
:1097B0002EDACE01079661E00E9463DAC801829634
:1097C0000E940E92C80189579E4F40E251EA67E01D
:1097D00070E00E9494DCC80187960E94F792C8014D
:1097E00089529F4F0E94F792CE0101966FE97AE16C
:1097F00044E00E942EDACE01019661E00E9463DA15
:10980000C80183579D4F0E94B4DBC8018F559D4FFF
:109810000E947CAAC8018A569E4F40E553EC60E046
:1098200070E00E9494DCE0960FB6F894DEBF0FBEA5
:10983000CDBFDF91CF911F910F91FF90EF90DF90FF
:10984000CF9008950F931F934FB7F894FC010081B8
:109850001181228133814FBFB801C9011F910F913E
:1098600008950E94C72B882369F5809170008D7F31
:1098700080937000809173008D7F80937300789443
:109880000E94578FF89480917000826080937000DE
:109890008091730082608093730020912401309145
:1098A000250180912801909129012817390750F04E
:1098B00081E090E090932901809328011092250186
:1098C000109224010895CF93DF93EC01FC01E15E37
:1098D000FC4F7183608362307105E1F48F559D4FB9
:1098E0000E94B1AF8823D9F40E94943D8823B9F037
:1098F000CE01805C9F4F0E94B1AF8823A1F0CE01C2
:1099000080519F4F0E94B1AF882369F008C081E069
:1099100080939D09C45EDC4F81E0888304C0809100
:109920009D098823A1F3DF91CF910895FC01EF5D9C
:10993000FC4F442321F08081862B8083089560951D
:109940008081682360830895CF93DF93EC01805C6E
:109950009F4F0E94B5AD882369F4CE0180519F4F7F
:109960000E94B5AD882331F4CE018F559D4F0E94E2
:10997000B5AD01C081E0DF91CF910895FC01E65DB6
:10998000FC4F31E03083FC01E55DFC4F6083FC015E
:10999000E45DFC4F4083FC01E35DFC4F2083825D6E
:1099A0009C4FFC0110820895DF92EF92FF920F937B
:1099B0001F93CF93DF938C01FC01E65DFC4F108277
:1099C0004AEBE42E41E0F42EE80EF91EEC01C45DF2
:1099D000DC4FFC01E55DFC4FC701688140810E94BE
:1099E00076B6D880E801C35DDC4F06C0C70163E3EB
:1099F00072E00E9467B5D3948881D816B8F3DF91DE
:109A0000CF911F910F91FF90EF90DF9008958F926B
:109A10009F92AF92BF92CF92DF92FF920F931F93CC
:109A2000CF93DF934C01A62E142FC22E241708F4D7
:109A300079C0422F50E0411B5109802F90E0481718
:109A400059070CF46FC0F401E95DFC4F608171812E
:109A500016161706ECF4F401EB5DFC4FD401AD5D76
:109A6000BC4F208131818D919C911197281B390B1E
:109A700037FF03C0309521953F4F249FC001259F9C
:109A8000900D349F900D11240E9463E2F62E01C0C8
:109A9000FF24F01698F4E401C654DE4FCE01612F86
:109AA0004A2D0E9476B6012F06C0CE0163E372E014
:109AB0000E9467B50F5F0C15C1F700E05AEBC52E89
:109AC00051E0D52EC80CD91C602F610FC6014A2D5C
:109AD0000E9476B6AA24BB24C02FD0E00F2D10E040
:109AE00007C0C6016FEF0E94B7B60894A11CB11C55
:109AF000C5018C0F9D1F801791079CF3F401E75D52
:109B0000FC4F808191E089278083882331F0C60152
:109B100068E474E00E947EB506C0C6016FEF0E9443
:109B2000B7B601C0FF248F2DDF91CF911F910F9108
:109B3000FF90DF90CF90BF90AF909F908F9008954F
:109B40008F929F92AF92BF92CF92DF92EF92FF924D
:109B50000F931F93CF93DF937C0105E2A02E03E0C8
:109B6000B02EA80EB91EF50111821082FC01E95D2C
:109B7000FC4F11821082EC01CD5DDC4F19821882FE
:109B80000E94A44C882309F416C111EAC12E12E0E8
:109B9000D12ECE0CDF1CC6010E94B5AD8823E1F0AA
:109BA00008811981C6010E94EBAD880F991F800FB3
:109BB000911F99838883F501C081D181C6010E94DC
:109BC0009FAD880F991F8C0F9D1FF5019183808396
:109BD000B6EEAB2EB12C1AC0F701EA54FF4F8081CC
:109BE000882331F0C701805C9F4F60E00E9401AE86
:109BF000F701EA59FE4F8081882331F0C701805177
:109C00009F4F60E00E9401AEAA24BB2470E4C72EDF
:109C1000D12CCE0CDF1CC6010E94B5AD882331F1DA
:109C2000F701EA54FF4F8081882301F587010D5D1C
:109C30001C4FF801C081D181C6010E94EBADC80F55
:109C4000D91FF801D183C08387010B5D1C4FF80138
:109C5000C081D181C6010E949FADC80FD91FF801F4
:109C6000D183C08386EE90E0A80EB91E60EFC62EA9
:109C7000D12CCE0CDF1CC6010E94B5AD882331F17A
:109C8000F701EA59FE4F8081882301F587010D5DB8
:109C90001C4FF801C081D181C6010E94EBADC80FF5
:109CA000D91FF801D183C08387010B5D1C4FF801D8
:109CB000C081D181C6010E949FADC80FD91FF80194
:109CC000D183C0838EE690E0A80EB91EF701EB5D4C
:109CD000FC4F20813181F701ED5DFC4F8081918146
:109CE000F701E95DFC4F281739072CF4A21AB30AD3
:109CF000B182A08202C0318320838081918100974C
:109D000009F462C082E491E061E00E9477A98823AF
:109D100009F45AC080E491E067E00E9477A9873097
:109D200009F452C0E701CE5DDC4F8881882321F41D
:109D30000E94579481E08883F701ED5DFC4F00811C
:109D40001181F701E95DFC4F80809180AA2497FC86
:109D5000A094BA2CF701EB5DFC4F60817181601B10
:109D6000710B77FF03C0709561957F4F882777FD52
:109D70008095982F2FEF30E040E050E00E9424E2E1
:109D8000A50194010E9498E2C22FB801882777FDAF
:109D90008095982F2FEF30E040E050E00E9424E2C1
:109DA000A50194010E9498E28C2F60E0422F20E0F0
:109DB0000E946A9409C0E701CE5DDC4F8881882348
:109DC00019F00E9457951882F701E65DFC4F8081DB
:109DD0008823A9F0F701E55DFC4FD701A45DBC4FD6
:109DE0009701235D3C4FE701C25DDC4FC7016081F5
:109DF0004C91F901208108810E94074D8883DF91F1
:109E0000CF911F910F91FF90EF90DF90CF90BF9077
:109E1000AF909F908F900895439640E052ED69E493
:109E20007BE60E9494DC08951F920F920FB60F926A
:109E30000BB60F9211242F933F934F935F936F9321
:109E40007F938F939F93AF93BF93EF93FF938EE98D
:109E500099E00E94314CFF91EF91BF91AF919F919A
:109E60008F917F916F915F914F913F912F910F90C3
:109E70000BBE0F900FBE0F901F9018950F931F935E
:109E8000CF93DF9300D000D000D0CDB7DEB78B01E9
:109E90006115710589F41092970910929609CE0107
:109EA000019661EB7AE147E00E942EDACE0101963D
:109EB00060E00E9486DA0CC080919A0990E08617D3
:109EC000970731F082E090E090939709809396098C
:109ED00000939A0926960FB6F894DEBF0FBECDBF49
:109EE000DF91CF911F910F910895CF93DF93CDB75D
:109EF000DEB768970FB6F894DEBF0FBECDBF411531
:109F00005105D9F41092950910929409CE01439607
:109F10006FEA7AE145E00E942EDACE01439661E0D5
:109F20000E9486DACE010D966FEA7AE146E00E9441
:109F30002EDACE010D9661E01DC061157105E9F4C0
:109F40001092950910929409CE0107966FEA7AE172
:109F500045E00E942EDACE01079660E00E9486DA84
:109F6000CE0101966FEA7AE146E00E942EDACE0138
:109F7000019660E00E9486DA0AC0609399094093D6
:109F8000980981E090E090939509809394096896F0
:109F90000FB6F894DEBF0FBECDBFDF91CF9108950D
:109FA000CF93DF93EC0169E170E04FE050E00E9455
:109FB000754FCE018A529E4F6FEF0E94AFB3C35EC2
:109FC000DC4F81E08883DF91CF9108950F931F9339
:109FD000CF93DF930F92CDB7DEB78C018A529E4F9D
:109FE00049830E9414B1C8010E94D04F80E00E94B2
:109FF000D455F801E25EFC4F498140830F90DF9118
:10A00000CF911F910F910895DF92EF92FF920F93DE
:10A010001F93CF93DF938C01FC0186A18823F1F07D
:10A02000E801CA52DE4FCE010E945BB024E0E22E6E
:10A03000F12CE00EF11EC7010E94BADC882371F0FA
:10A04000CE010E9419B2CE010E9461B0AB01BC01E9
:10A05000C7010E9494DCDD24D39401C0DD24F80103
:10A06000E55EFC4F80818823A1F0E801CA56DE4FEF
:10A07000CE010E94BADC882361F0C8018F559D4F44
:10A080000E948BAECE0140E553EC60E070E00E9490
:10A0900094DC9DE1E92E93E0F92EE00EF11EF7012C
:10A0A0008081882301F1E801CA52DE4FCE010E946F
:10A0B000B4B38823C1F0C80160E070E040E050E034
:10A0C0000E94754F0E945795F7011082CE010E94A1
:10A0D000E1B1F801E25EFC4F8081882311F00E941B
:10A0E000B44510929B09E8016396CE010E94BADC48
:10A0F000882309F477C0F801E45EFC4F808188234F
:10A1000009F070C00E9484438230910509F46AC04E
:10A110000E9484438130910509F464C0F801EF5D29
:10A12000FC4F808180648E7F808380E4E82EF12C58
:10A13000E00EF11EC7010E949FAD1816190684F0AB
:10A14000C80180519F4F0E949FAD1816190644F018
:10A15000C8018F559D4F0E949FAD1816190664F5D2
:10A16000F801E15DFC4F80819181A281B38180344F
:10A17000F2E49F07FFE0AF07F0E0BF0769F4CE010C
:10A180000E9419DDDC01CB01803022ED920729E429
:10A19000A2072BE6B20780F0C8018A529E4F6AE4FC
:10A1A00074E00E9414B1C8010E94D04F80E060E0CA
:10A1B0004FEF21E00E946A94C70160E070E00E94C6
:10A1C000CEACC80180519F4F60E070E00E94CEACE1
:10A1D000C8018F559D4F60E070E00E94CEACCE016B
:10A1E0000E94E7DCE801C45EDC4F8881882309F423
:10A1F000A5C080919B09882309F0A0C00E94C0558A
:10A20000882309F09BC081E080939B09C8016AE024
:10A2100070E04AE050E00E94754FF801E15EFC4FAB
:10A220008081918188309105C9F08930910544F48D
:10A230008230910549F18430910509F057C008C07A
:10A240008031910599F08032910509F04FC014C01A
:10A25000C8018A529E4F63E774E005C0C8018A5264
:10A260009E4F63EC74E00E9414B140C0C8018A5252
:10A270009E4F64E175E0F7CFC80165E675E040E008
:10A280000E94E64F188282C0C80166EB75E040E08C
:10A290000E94E64FE801C05CDF4FCE010E94B1AFE3
:10A2A000882329F0CE0160E070E00E94CEACE80186
:10A2B000C051DF4FCE010E94B1AF882329F0CE01FB
:10A2C00060E070E00E94CEACE801CF55DD4FCE01DA
:10A2D0000E94B1AF882329F0CE0160E070E00E94B7
:10A2E000CEACF801E45EFC4F108250C0C801805C27
:10A2F0009F4F60E070E00E94CEACC80180519F4F3C
:10A3000060E070E00E94CEACC8018F559D4F60E0C8
:10A3100070E00E94CEAC80E00E94D4550E945D9413
:10A320000E9449400E94C32B0E94628CC0E08C2F87
:10A3300060E00E94688BCF5FC530C9F7E801C9575C
:10A34000DE4FCE010E94BADC8823E1F0DD20D1F49B
:10A35000C80187960E941893C8010E94A04DCE01A3
:10A3600040E251EA67E070E00E9494DC81E0809373
:10A370009C090CC0C80189529F4F0E9418931092EB
:10A380009C0904C080919C098823A1F7DF91CF919B
:10A390001F910F91FF90EF90DF900895DF92EF9261
:10A3A000FF920F931F93CF93DF93CDB7DEB76897DC
:10A3B0000FB6F894DEBF0FBECDBF8C01D62E60E085
:10A3C00070E00E943E4F82E090E060E00E9477A93A
:10A3D0008095881F8827881F0E94248787E39DE136
:10A3E00061E00E9494DD8BE39DE10E9424D9F80195
:10A3F000108211821282138284E492E060E00E9453
:10A4000077A94FE2E42E43E0F42EE00EF11E682F10
:10A4100070E080E090E020E037E843E953E00E94FC
:10A4200024E2DC01CB01805C9D4BA04FBF4FF701C4
:10A4300080839183A283B383F80186A1882309F4E2
:10A4400061C036EDE32E31E0F32EE00EF11EC701C0
:10A450000E9454B1CE0143966FEA7AE145E00E9432
:10A460002EDACE01439661E00E9463DACE010D96AA
:10A470006FEA7AE146E00E942EDACE010D9661E0A5
:10A480000E9463DACE0107966FEA7AE145E00E9406
:10A490002EDACE01079661E00E9486DACE0101969F
:10A4A0006FEA7AE146E00E942EDACE01019661E081
:10A4B0000E9486DA86E591E060E00E9477A9882311
:10A4C00021F4C70165E070E003C0C70164E070E0FB
:10A4D0000E94E8B0DD2051F020E335E740E951E08B
:10A4E000CA010197F1F721503040D1F7C7010E940E
:10A4F000F0AFC7010E9461B0AB01BC01C801049676
:10A500000E9494DCC80160E070E040E050E00E94EE
:10A51000754FDD2071F00E94EE9583E00E94D455C6
:10A52000F801E45EFC4F1082F801E15EFC4F1182FD
:10A530001082F801EF5DFC4FEE24E394E0820E946C
:10A54000943D682FC80180519F4F0E94C2AC0E9469
:10A550007C3E682F6E25C8018F559D4F0E94C2AC6E
:10A56000F801E15DFC4F4081518162817381C80136
:10A5700043960E9494DC0E945795F801E35EFC4FDD
:10A580001082F801ED5DFC4F11821082F801EB5D45
:10A59000FC4F11821082F801E95DFC4F118210829C
:10A5A000F801EE5DFC4F1082F801E65DFC4F108271
:10A5B000F801E55DFC4F1082F801E45DFC4F10826C
:10A5C000F801E35DFC4F1082F80186A1882349F071
:10A5D00086E591E060E00E9477A9882311F00E944F
:10A5E000FDAF68960FB6F894DEBF0FBECDBFDF910A
:10A5F000CF911F910F91FF90EF90DF9008951F92E0
:10A600000F920FB60F920BB60F9211242F933F9318
:10A610004F935F936F937F938F939F93AF93BF936A
:10A62000EF93FF93CF93DF93CDB7DEB7AA97DEBF4B
:10A63000CDBF80919E0990919F09A091A009B091F2
:10A64000A1098C599F4FAF4FBF4F80939E099093A4
:10A650009F09A093A009B093A1090E94978F8091B0
:10A660008D09982F9F5F90938D09853A08F4DFC07C
:10A6700010928D09809192099091930918161906EC
:10A6800014F401973CC0809196099091970981300C
:10A69000910501F58091900990919109019690930F
:10A6A00091098093900982E090E0909397098093BC
:10A6B000960982E190E09093930980939209CE01EC
:10A6C000859661EB7AE147E00E942EDACE0185960D
:10A6D00060E04DC08230910569F580919A0990E063
:10A6E0002091900930919109281739076CF083E087
:10A6F00090E0909397098093960980E590E090937D
:10A7000093098093920935C081E090E09093970976
:10A710008093960982E190E0909393098093920947
:10A72000CE014F9661EB7AE147E00E942EDACE012E
:10A730004F961CC083309105E1F41092910910925C
:10A74000900981E090E0909397098093960982E1C7
:10A7500090E09093930980939209CE01499661EB22
:10A760007AE147E00E942EDACE01499661E00E942C
:10A7700086DA80918E0990918F091816190634F4A3
:10A78000019790938F0980938E0951C0809194090D
:10A79000909195098130910519F582E090E09093B0
:10A7A0009509809394098091990980938E0910925C
:10A7B0008F09CE0143966FEA7AE145E00E942EDAD6
:10A7C000CE01439661E00E9486DACE010D966FEAD3
:10A7D0007AE146E00E942EDACE010D9661E025C0B6
:10A7E0008230910521F581E090E090939509809366
:10A7F00094098091980980938E0910928F09CE0157
:10A8000007966FEA7AE145E00E942EDACE010796BC
:10A8100060E00E9486DACE0101966FEA7AE146E0B6
:10A820000E942EDACE01019660E00E9486DAAA9696
:10A83000DEBFCDBFDF91CF91FF91EF91BF91AF917F
:10A840009F918F917F916F915F914F913F912F9148
:10A850000F900BBE0F900FBE0F901F901895FC012C
:10A86000E55EFC4F60830895EF92FF920F931F9374
:10A87000CF93DF93CDB7DEB72C970FB6F894DEBF3A
:10A880000FBECDBFE62EFFB6F8940FE91AE1CE0158
:10A890000796B80145E00E942EDACE01079661E0E6
:10A8A0000E9463DACE010196B80145E00E942EDADB
:10A8B000CE0101966E2D0E9486DAFFBE2C960FB651
:10A8C000F894DEBF0FBECDBFDF91CF911F910F91E6
:10A8D000FF90EF90089581ED9CE06DE97AE140E012
:10A8E0000E942EDA8EE999E00E94414A0895CF93A2
:10A8F000DF93CDB7DEB72C970FB6F894DEBF0FBE4F
:10A90000CDBF8AE491E061E00E9477A991E08823BD
:10A9100009F490E09093310D1092DA0C1092D90C5A
:10A920001092DC0C1092DB0C1092DF0C1092E00CF9
:10A9300082E39DE00E94E7DC1092410DCE01079674
:10A9400067EA7AE145E00E942EDACE01079661E0DF
:10A950000E9463DACE01019667EA7AE145E00E943F
:10A960002EDACE01019660E00E9486DA2C960FB6B0
:10A97000F894DEBF0FBECDBFDF91CF91089514BC18
:10A9800015BC17BC18BC16BC10926E000895CF926F
:10A99000DF92EF92FF92CF938091D90C9091DA0CD5
:10A9A000009739F482E39DE00E94E7DC1092410DAC
:10A9B0004FC021E02093410D8091D90C9091DA0C89
:10A9C000009731F42093E00CCC24DD2476012EC0D6
:10A9D0008091DB0C9091DC0C2091D70C3091D80C3D
:10A9E000B9010E944FE2880F991F880F991FE091CB
:10A9F000DD0CF091DE0CE80FF91F8091DB0C9091DB
:10AA0000DC0C0196B9010E944FE29093DC0C80931C
:10AA1000DB0C8091D90C9091DA0C01979093DA0CB1
:10AA20008093D90CC080D180E280F380B70180E0B0
:10AA300090E028EE33E040E050E00E9424E2AB01D9
:10AA4000BC0182E39DE00E9494DCC601009719F4EA
:10AA50000E94BF543EC0A0E0B0E082342FE09207D5
:10AA600020E0A20720E0B20780F4883E21E09207B0
:10AA700020E0A20720E0B20758F48A379105A1052B
:10AA8000B10548F0C4E068E008C0C2E063E005C07A
:10AA9000C3E066E002C0C5E06AE09C01AD01220FA0
:10AAA000331F441F551F04C0220F331F441F551F5F
:10AAB0006A95D2F760E074E284EF90E00E9476E25B
:10AAC000215082E184BDC5BD27BD18BC16BC1092C3
:10AAD0006E00CF91FF90EF90DF90CF900895CF93CD
:10AAE000482FE92FF62FC72F8091310D882309F4C5
:10AAF00045C06091D70C7091D80C8091D90C909181
:10AB0000DA0C68177907A1F18091D90C9091DA0CD1
:10AB10008617970750F52091D90C3091DA0C809167
:10AB2000DB0C9091DC0C820F931F0E944FE2880F88
:10AB3000991F880F991FA091DD0CB091DE0CA80F12
:10AB4000B91F4C931196EC9311971296FC931297A0
:10AB50001396CC9313978091D90C9091DA0C0196AF
:10AB60009093DA0C8093D90C03C081E08093DF0CC2
:10AB70008091410D882311F40E94C754CF9108950C
:10AB80008091410D08958091310D882361F080916D
:10AB9000410D882341F082E39DE00E94BADC8823C6
:10ABA00011F00E94C7540895EF92FF921F93CF9324
:10ABB000DF93883038F5E82FF0E0EE0FFF1FE35BFE
:10ABC000FB4FE080F180E114F104E1F010E0812F0F
:10ABD00090E0880F991F880F991FF701E80FF91F60
:10ABE0002591349102968E0D9F1DFC01C591D49143
:10ABF000209721F0C901BE010E946F551F5F209769
:10AC000031F706C08BE790E064EF71E00E946F556A
:10AC1000DF91CF911F91FF90EF90089582E49DE026
:10AC20006DE97AE140E00E942EDA84E190E09093B1
:10AC3000D80C8093D70C1092DA0C1092D90C109289
:10AC4000DC0C1092DB0C81EE9CE09093DE0C809388
:10AC5000DD0C1092DF0C1092E00C82E39DE00E946C
:10AC600090DC089508958F929F92AF92BF92CF92F9
:10AC7000DF92EF92FF920F931F93CF93DF93CDB7A5
:10AC8000DEB7FC01408351836283738304831583A1
:10AC900026833783C086D186E286F38684869586AE
:10ACA000A686B7868F859889A989BA89808B918B6A
:10ACB000A28BB38BDF91CF911F910F91FF90EF90FB
:10ACC000DF90CF90BF90AF909F908F900895660FC8
:10ACD000771F660F771F680F791FCB010895660FE6
:10ACE000771F660F771F680F791FCB0108950F93A9
:10ACF00082E394EA6FEC74EA4BED55EA26E936EA12
:10AD000000E00E945FA290935C0D80935B0D009722
:10AD100079F482E394EA6FEC74EA4BED55EA26E9A4
:10AD200036EA0FEF0E945FA290935C0D80935B0D5B
:10AD300081E020915B0D30915C0D2115310509F406
:10AD400080E00F91089580915B0D90915C0D0E94C1
:10AD5000619B9C0190935A0D8093590D81E02115C0
:10AD6000310509F480E00895CF93DF93CDB7DEB7C6
:10AD7000AB970FB6F894DEBF0FBECDBF8091590DD3
:10AD800090915A0D65E372E0AE014F5F5F4F0E94F4
:10AD9000BBA08091590D90915A0DBE016F5F7F4FFE
:10ADA0000E94A99F9C019093580D8093570D81E0BC
:10ADB0002115310509F480E0AB960FB6F894DEBF9B
:10ADC0000FBECDBFDF91CF9108958091590D909125
:10ADD0005A0D0E9434A2DC01CB0180959095A0957C
:10ADE000B0958827B7FD83959927AA27BB27089593
:10ADF000AF92BF92CF92DF92EF92FF921F93CF93C9
:10AE0000DF93CDB7DEB7AB970FB6F894DEBF0FBEBA
:10AE1000CDBF7C015A0115E0C62EDD240894C1087F
:10AE2000D1088091570D9091580DBE016F5F7F4FF3
:10AE30000E94EC9FF7018823E1F0DE01119680E08B
:10AE400090E08C159D0534F42D91222319F0219367
:10AE50000196F7CFF701E80FF91F1082009731F044
:10AE6000A114B10439F0F501808304C01150C9F672
:10AE700001C0108280E090E0AB960FB6F894DEBF80
:10AE80000FBECDBFDF91CF911F91FF90EF90DF906C
:10AE9000CF90BF90AF9008950F931F93CF93DF9300
:10AEA0008C01EB010EC0CE01B8010E9409E30097AE
:10AEB00041F48091570D9091580D0E9446A181E078
:10AEC00009C08091570D9091580DBE010E94EC9FD2
:10AED000882349F7DF91CF911F910F9108950F9328
:10AEE0001F93CF93DF93CDB7DEB7AB970FB6F89430
:10AEF000DEBF0FBECDBF8B01BE016F5F7F4F0E94D3
:10AF00004C57882371F08091590D90915A0DBE01D4
:10AF10006F5F7F4F0E940C9DF8019183808381E0D9
:10AF200001C080E0AB960FB6F894DEBF0FBECDBF78
:10AF3000DF91CF911F910F9108956091510D709104
:10AF4000520D8091530D9091540D0895CF93DF933E
:10AF5000CDB7DEB7AB970FB6F894DEBF0FBECDBF4F
:10AF6000BE016F5F7F4F0E944C57882359F080913C
:10AF7000590D90915A0DBE016F5F7F4F0E94B0A195
:10AF800081E001C080E0AB960FB6F894DEBF0FBE43
:10AF9000CDBFDF91CF910895CF93DF93CDB7DEB7CB
:10AFA000AB970FB6F894DEBF0FBECDBFBC0180914A
:10AFB000570D9091580DAE014F5F5F4F0E9453A106
:10AFC00091E0882309F490E0892FAB960FB6F894AE
:10AFD000DEBF0FBECDBFDF91CF91089580914F0DA1
:10AFE00008958091500D0895CF93DF93EC018091E7
:10AFF000550D9091560D0097E1F0BE016E5F7F4FA9
:10B00000488150E00E94689E288180914B0D90916C
:10B010004C0DA0914D0DB0914E0D820F911DA11DB3
:10B02000B11D80934B0D90934C0DA0934D0DB0939B
:10B030004E0DDF91CF9108958091500D882381F0BE
:10B040008091550D9091560D009721F00E94439DDF
:10B050000E94D8A31092560D1092550D1092500DCB
:10B0600060914B0D70914C0D80914D0D90914E0D56
:10B0700008950E94A0A3882391F08091550D90918E
:10B08000560D6AE47DE041E050E00E94569D21E0CB
:10B09000181619060CF020E02093490D08958EE94A
:10B0A00099E063E877E041E00E94E64F1092490D95
:10B0B0001092480D08958091490D0895CF93DF9324
:10B0C0000F92CDB7DEB780914A0D89830E9439581F
:10B0D00089810F90DF91CF91089510924F0D80914B
:10B0E000550D9091560D009721F00E94439D0E94AE
:10B0F000D8A31092560D1092550D089580914F0DC2
:10B10000882311F00E946D588091500D882311F012
:10B110000E941C588091570D9091580D009731F066
:10B120000E94E69F1092580D1092570D8091590D74
:10B1300090915A0D009731F00E94069D10925A0D81
:10B140001092590D80915B0D90915C0D009731F03C
:10B150000E9430A310925C0D10925B0D1092510D65
:10B160001092520D1092530D1092540D08950E949A
:10B1700023A5882371F40E94A0A3882329F40E94A8
:10B180007E5881E090E008950E947E5882E090E031
:10B1900008950E947756882329F40E947E5883E000
:10B1A00090E008950E94A356882329F40E947E58B7
:10B1B00084E090E008950E94B456882329F40E9408
:10B1C0007E5885E090E008950E94E556882329F492
:10B1D0000E947E588AE090E008950E94BDA38823D3
:10B1E00019F086E090E0089580E090E00895CF9314
:10B1F000DF93EC010E947E580E94B758009719F027
:10B2000086309105D9F410924B0D10924C0D10928E
:10B210004D0D10924E0D1092560D1092550DCE01FF
:10B2200065E57DE00E946F57882331F08091550DD0
:10B230009091560D009729F487E090E0DF91CF912F
:10B2400008950E942EA2DC01CB018093510D9093B2
:10B25000520DA093530DB093540D81E080934F0D88
:10B260000E94395880E090E0E9CF0F931F93CF936D
:10B27000DF938C010E947E580E94B758EC01009722
:10B2800069F510924B0D10924C0D10924D0D1092CD
:10B290004E0D1092560D1092550DC8010E94A657E2
:10B2A000C8010E94CC57882389F0C80165E57DE07C
:10B2B0000E946F57882369F08091550D9091560D2B
:10B2C000009751F081E08093500D08C0C7E0D0E0B6
:10B2D00005C0C3E0D0E002C0C8E0D0E0CE01DF91FD
:10B2E000CF911F910F9108950E947E580E94B758E8
:10B2F000009719F08630910541F48091570D909197
:10B30000580D0E9446A180E090E008958DE59DE0F3
:10B310006DE97AE140E00E942EDA0895CF92DF9243
:10B32000EF92FF920F931F93CF93DF93CDB7DEB7CA
:10B330006E970FB6F894DEBF0FBECDBF6C017C01D7
:10B340008C01025E1F4FC7010E9420DA86E090E068
:10B35000E80EF91EE016F106B1F7C6014E9663EA53
:10B360007AE145E00E942EDA85E0F60184A3CE0161
:10B37000499669EA7AE143E00E942EDAD601FE019D
:10B38000799686E001900D928150E1F7CE014396C7
:10B3900069EA7AE147E00E942EDAD6011696FE01AC
:10B3A000739686E001900D928150E1F7CE010D96E3
:10B3B00061EA7AE143E00E942EDAD6011C96FE0192
:10B3C0003D9686E001900D928150E1F7CE010796FF
:10B3D00063EB7AE145E00E942EDAD6015296FE0137
:10B3E000379686E001900D928150E1F7CE010196EB
:10B3F00063EA7AE146E00E942EDAD6015896FE0111
:10B40000319686E001900D928150E1F76E960FB66D
:10B41000F894DEBF0FBECDBFDF91CF911F910F918A
:10B42000FF90EF90DF90CF900895FF920F931F93BE
:10B43000CF93DF938C01FF2414C08F2D90E0EC019B
:10B44000CC0FDD1FC80FD91FCC0FDD1FC00FD11FC0
:10B45000CE0161E00E9463DACE0161E00E9486DAEB
:10B46000F394F80184A1F81640F3025E1F4FC8015F
:10B4700061E00E9463DAC80161E00E9486DADF9130
:10B48000CF911F910F91FF9008951F93CF93DF935A
:10B49000EC0115E1812F8A95F1F7CE014E9661E01E
:10B4A0000E9486DA1A95F1F710E00FC0212F30E0E4
:10B4B000C901880F991F820F931F880F991F8C0F46
:10B4C0009D1F61E00E9486DA1F5F8CA1181770F340
:10B4D00085E18A95F1F7DF91CF911F910895BF9291
:10B4E000CF92DF92EF92FF920F931F93CF93DF9350
:10B4F000D62EEA01A8E0EA2EF12CB0E8CB2E8C0182
:10B50000025E1F4F25E1B22E8C2D8D2161E009F4E2
:10B5100060E0CE010E9486DAC80161E00E9486DA0E
:10B520008B2D8A95F1F7C80160E00E9486DAC694F7
:10B530000894E108F108E114F10431F7CE0161E06B
:10B540000E9486DACE0160E00E9463DAC80161E001
:10B550000E9486DACE010E9477DAE82EC80160E008
:10B560000E9486DACE0161E00E9463DA81E0E11098
:10B5700080E0DF91CF911F910F91FF90EF90DF90CE
:10B58000CF90BF900895EF92FF920F931F93CF93A8
:10B59000DF93EC01162F7A0100E00FC0202F30E07E
:10B5A000C901880F991F820F931F880F991F8C0F55
:10B5B0009D1F60E00E9486DA0F5F8CA1081770F370
:10B5C00085E18A95F1F7CE014E9660E00E9486DA19
:10B5D000CE01612FA7010E946F5ADF91CF911F9179
:10B5E0000F91FF90EF90089588E89DE06DE97AE172
:10B5F00040E00E942EDA83E69DE00E948E59089575
:10B600004F925F926F927F928F929F92AF92BF9272
:10B61000CF92DF92EF92FF920F931F93CF93DF931E
:10B620008091A00D9091A10D009709F02DC49091EB
:10B63000CA0D8091C90D9817A1F02091C90D30E075
:10B6400087E790E0289FF001299FF00D389FF00DCB
:10B650001124E553F24FDF01AC58BF4F81E08C93CA
:10B6600002C0E0E0F0E0F093A10DE093A00D309770
:10B6700009F4ADC3808D918DA28DB38D80932C166E
:10B6800090932D16A0932E16B0932F16848D958D22
:10B69000A68DB78D8093301690933116A0933216F5
:10B6A000B093331680A191A1A2A1B3A180933416C7
:10B6B00090933516A0933616B093371684A195A1B2
:10B6C000A6A1B7A18093381690933916A0933A1685
:10B6D000B0933B1680A591A5A2A5B3A580933C1677
:10B6E00090933D16A0933E16B0933F1682AD809383
:10B6F000A20D8091A30D8823E1F18F01C4EADDE062
:10B700006CE97DE040E050E0F80184859585A685F0
:10B71000B7850097A105B10511F188818823F9F05B
:10B72000FA01E656F24F8081FA01EE0FFF1FED5D40
:10B73000F94E882349F080819181DB012D913C9164
:10B740001197821B930B08C080819181DB012D91A1
:10B750003C911197820F931F9183808318824F5FD2
:10B760005F4F0C5F1F4F21966E5F7F4F4230510538
:10B7700059F61092A60D1092A70D1092A80D1092D6
:10B78000A90DC091A00DD091A10DFE01E25AFF4F6D
:10B79000208131813F3460F03D3930F443E036950B
:10B7A00027954A95E1F702C028E833E188E014C004
:10B7B000383230F0369527953695279584E00CC0C1
:10B7C000343120F03695279582E006C020323105CD
:10B7D00010F420E230E081E08093AA0D2052304046
:10B7E000B8E020303B07C8F0E32FF0E0EE0FFF1F7A
:10B7F000EE0FFF1FED56F84F85919591A591B491ED
:10B80000AC01BD01AA27279FC001269F810D9A1F69
:10B8100006948A1F9A1F11241AC0F901F695E7951C
:10B82000EC7FED56F44F85919591A591B491AC01C3
:10B8300030E0277030702A9FC0012B9F900D3A9FF7
:10B84000900D112413E0969587951A95E1F7481B02
:10B85000590B5093AC0D4093AB0D8091AA0D809382
:10B86000AD0DFE01EE58FF4F8081882309F472C0B0
:10B87000CA59DF4F288139813093AF0D2093AE0D27
:10B880003F3460F03D3930F4A3E036952795AA9512
:10B89000E1F702C028E833E188E014C0383230F024
:10B8A000369527953695279584E00CC0343120F0E5
:10B8B0003695279582E006C02032310510F420E24B
:10B8C00030E081E08093AA0D20523040E8E0203043
:10B8D0003E07C8F0E32FF0E0EE0FFF1FEE0FFF1F53
:10B8E000ED56F84F85919591A591B491AC01BD01AC
:10B8F000AA27279FC001269F810D9A1F06948A1FA1
:10B900009A1F11241AC0F901F695E795EC7FED56C0
:10B91000F44F85919591A591B491AC0130E02770D9
:10B9200030702A9FC0012B9F900D3A9F900D1124DB
:10B9300063E0969587956A95E1F7481B590BCA0114
:10B94000A0E0B0E08093B00D9093B10DA093B20D44
:10B95000B093B30D5093290140932801E091A00DBD
:10B96000F091A10D80AD8093B40DEA58FF4F208176
:10B970008091231690912416009709F023608091FE
:10B98000251690912616009709F0246080912116C3
:10B99000281709F442C0EFE6F3E0EF01249640E0F7
:10B9A00050E061E070E0CB01042E02C0880F991FC7
:10B9B0000A94E2F7A82F309121163227382331F16B
:10B9C000A22390912116AA2389F0982B90932116F7
:10B9D000A081B1813C91CB01088002C0880F991FE2
:10B9E0000A94E2F7809583238C9310C08095892375
:10B9F00080932116A081B1813C91CB01088002C0C7
:10BA0000880F991F0A94E2F7382B3C934F5F5F4FE2
:10BA1000B396A3964530510531F6E091A00DF09113
:10BA2000A10DDF01AB58BF4FDC9174896589568940
:10BA30004789C091B40D008111812281338181E059
:10BA4000011511052105310509F480E080935C168C
:10BA5000882309F444C0872F962FA52FB42FEE24F6
:10BA6000E394EC22AC01BD01759567955795479518
:10BA700070956095509541955F4F6F4F7F4F409304
:10BA80005D1650935E1660935F167093601641E0EA
:10BA9000D11140E04093541680935516909356165A
:10BAA000A0935716B0935816009365161093661618
:10BAB0002093671630936816EE2011F08FEF01C0C7
:10BAC00081E080935A1681E08E2580935B16109258
:10BAD00061161092621610926316109264167489A1
:10BAE000658956894789048115812681378181E0DE
:10BAF000011511052105310509F480E080938516B3
:10BB0000882309F446C0872F962FA52FB42FEE2443
:10BB1000E394C1FFEE24AC01BD017595679557957F
:10BB2000479570956095509541955F4F6F4F7F4F4A
:10BB300040938616509387166093881670938916E3
:10BB400041E0D13009F040E040937D1680937E16AD
:10BB500090937F16A0938016B093811600938E1653
:10BB600010938F162093901630939116EE2011F0BB
:10BB70008FEF01C081E08093831681E08E25809352
:10BB8000841610928A1610928B1610928C161092B0
:10BB90008D167489658956894789008511852285A6
:10BBA000338581E0011511052105310509F480E097
:10BBB0008093AE16882309F446C0872F962FA52FB1
:10BBC000B42FEE24E394C2FFEE24AC01BD017595C1
:10BBD00067955795479570956095509541955F4F3E
:10BBE0006F4F7F4F4093AF165093B0166093B116CE
:10BBF0007093B21641E0D23009F040E04093A616AF
:10BC00008093A7169093A816A093A916B093AA168E
:10BC10000093B7161093B8162093B9163093BA163E
:10BC2000EE2011F08FEF01C081E08093AC1681E02F
:10BC30008E258093AD161092B3161092B416109202
:10BC4000B5161092B6167489658956894789048598
:10BC500015852685378581E00115110521053105FA
:10BC600009F480E08093D716882309F446C0872F13
:10BC7000962FA52FB42FEE24E394C3FFEE24AC013E
:10BC8000BD01759567955795479570956095509549
:10BC900041955F4F6F4F7F4F4093D8165093D91601
:10BCA0006093DA167093DB1641E0D33009F040E080
:10BCB0004093CF168093D0169093D116A093D216AE
:10BCC000B093D3160093E0161093E1162093E2167A
:10BCD0003093E316EE2011F08FEF01C081E08093E6
:10BCE000D51681E08E258093D6161092DC16109220
:10BCF000DD161092DE161092DF16DF01AB58BF4F33
:10BD0000DC91E488058936892789408951896289CF
:10BD1000738981E0411551056105710509F480E0E1
:10BD200080930017882309F445C08E2D902FA32FF0
:10BD3000B22FE1E0C4FFE0E08C019D01359527952D
:10BD40001795079530952095109501951F4F2F4F0A
:10BD50003F4F00930117109302172093031730935E
:10BD6000041721E0D43009F020E02093F8168093E6
:10BD7000F9169093FA16A093FB16B093FC16409315
:10BD8000091750930A1760930B1770930C17EE2343
:10BD900011F08FEF01C081E08093FE1681E08E27C5
:10BDA0008093FF161092051710920617109207172E
:10BDB000109208171092B60D1092B50D10928E0DBC
:10BDC00010928F0D1092900D1092910D5DC080ED2C
:10BDD00097E09093290180932801809123169091F8
:10BDE0002416009709F050C08091251690912616D0
:10BDF000009709F049C0209122168091211628173A
:10BE000009F442C0EFE6F3E0EF01249640E050E091
:10BE100061E070E0CB01042E02C0880F991F0A94E4
:10BE2000E2F7A82F309121163227382331F1A223CF
:10BE300090912116AA2389F0982B90932116A08126
:10BE4000B1813C91CB01088002C0880F991F0A94F0
:10BE5000E2F7809583238C9310C08095892380938B
:10BE60002116A081B1813C91CB01088002C0880FCE
:10BE7000991F0A94E2F7382B3C934F5F5F4FB396BC
:10BE8000A3964530510531F68091A30D882309F41E
:10BE900043C06091A00D7091A10DA4EABDE0CCE972
:10BEA000DDE040E050E001E086E7C82ED12CC60E70
:10BEB000D71E6115710561F0F601208130E0CA01DD
:10BEC000039602C0359527958A95E2F720FD1DC09F
:10BED0008C918823D1F4FA01E656F24F2081CA01F1
:10BEE000880F991FFC01ED5DF94E8081918122231D
:10BEF00029F028813981820F931F04C0288139815C
:10BF0000821B930B918380830C934F5F5F4F11963D
:10BF100022964230510569F68091A00D9091A10DB5
:10BF2000009711F40C94606BD090AA0DE090B50DC1
:10BF3000F090B60D4090B70D5090B80D6090B90DCF
:10BF40007090BA0D7094609450944094411C511CB0
:10BF5000611C711C452C562C672C772467FC7A9445
:10BF60008824C1E0D0E0CC24C394A4C5E091A00D06
:10BF7000F091A10DDF01AE58BF4F8C91882309F4D9
:10BF800076C0E114F104F1F002E0E016F104A1F54D
:10BF900086AD97AD909581959F4FAA2797FDA09567
:10BFA000BA2F4091D8165091D9166091DA16709137
:10BFB000DB16840F951FA61FB71F840D951DA61DA8
:10BFC000B71D12C044AD55AD662757FD6095762F5D
:10BFD0008091D8169091D916A091DA16B091DB16FF
:10BFE000840F951FA61FB71F8093D8169093D9165C
:10BFF000A093DA16B093DB16E114F10499F444AD82
:10C0000055AD662757FD6095762F80910117909169
:10C010000217A0910317B0910417840F951FA61F54
:10C02000B71F1DC012E0E116F10409F586AD97AD0A
:10C03000909581959F4FAA2797FDA095BA2F409183
:10C040000117509102176091031770910417840F24
:10C05000951FA61FB71F840D951DA61DB71D8093A4
:10C06000011790930217A0930317B09304178091C0
:10C070005C16882309F4FAC08091651690916616C3
:10C08000A0916716B091681600915D1610915E162A
:10C0900020915F1630916016080F191F2A1F3B1F51
:10C0A00000935D1610935E1620935F163093601612
:10C0B00010161106120613060CF0D8C04091611636
:10C0C0005091621660916316709164164817590773
:10C0D0006A077B070CF0CAC08091551690915616DE
:10C0E000A0915716B0915816081B190B2A0B3B0B41
:10C0F00000935D1610935E1620935F1630936016C2
:10C1000080915916882381F080911D1690911E16FA
:10C1100020915A16332727FD3095820F931F909355
:10C120001E1680931D1674C090915B168091411667
:10C1300081119C25E0916803F091690380916C0363
:10C140002081992349F0AE0102C0440F551F8A9502
:10C15000E2F7242B20830AC0BE0102C0660F771FBE
:10C160008A95E2F7CB0180958223808380915B16CC
:10C170008823A1F080917D0390917E03009749F17F
:10C18000E0917F03F0918003808190E00090810333
:10C1900002C0959587950A94E2F713C080917603C3
:10C1A000909177030097A9F0E0917803F0917903DB
:10C1B000808190E000907A0302C0959587950A945B
:10C1C000E2F78170907090914016981711F00C94DE
:10C1D000746BE0916103F09162032081CE010090C5
:10C1E000650302C0880F991F0A94E2F7282B208369
:10C1F000E0916103F09162032081CE01009065031C
:10C2000002C0880F991F0A94E2F7809582238083E9
:10C2100080912C1690912D16A0912E16B0912F166C
:10C2200040915A16552747FD5095652F752F840F5D
:10C23000951FA61FB71F80932C1690932D16A093C1
:10C240002E16B0932F168091611690916216A091D0
:10C250006316B09164160196A11DB11D80936116FD
:10C2600090936216A0936316B0936416809185161E
:10C27000882309F4FAC080918E1690918F16A091B0
:10C280009016B09191160091861610918716209104
:10C29000881630918916080F191F2A1F3B1F00931B
:10C2A00086161093871620938816309389161016D9
:10C2B0001106120613060CF0D8C040918A16509150
:10C2C0008B1660918C1670918D16481759076A0766
:10C2D0007B070CF0CAC080917E1690917F16A091CA
:10C2E0008016B0918116081B190B2A0B3B0B00938B
:10C2F000861610938716209388163093891680919E
:10C300008216882381F080911F169091201620912B
:10C310008316332727FD3095820F931F90932016A5
:10C3200080931F1674C09091841680916A168111B3
:10C330009C25E0918B03F0918C0380918F032081E9
:10C34000992349F0DE0102C0AA0FBB1F8A95E2F7CC
:10C350002A2B20830AC08E0102C0000F111F8A956C
:10C36000E2F7C80180958223808380918416882318
:10C37000A1F08091A0039091A103009749F1E09171
:10C38000A203F091A303808190E00090A40302C077
:10C39000959587950A94E2F713C08091990390913F
:10C3A0009A030097A9F0E0919B03F0919C03808190
:10C3B00090E000909D0302C0959587950A94E2F75E
:10C3C0008170907090916916981711F00C94786BA9
:10C3D000E0918403F09185032081CE0100908803D1
:10C3E00002C0880F991F0A94E2F7282B2083E0915E
:10C3F0008403F09185032081CE010090880302C060
:10C40000880F991F0A94E2F7809582238083809198
:10C41000301690913116A0913216B091331640919A
:10C420008316552747FD5095652F752F840F951F4F
:10C43000A61FB71F8093301690933116A093321623
:10C44000B093331680918A1690918B16A0918C161A
:10C45000B0918D160196A11DB11D80938A169093FF
:10C460008B16A0938C16B0938D168091AE168823F0
:10C4700009F4FAC08091B7169091B816A091B91638
:10C48000B091BA160091AF161091B0162091B11666
:10C490003091B216080F191F2A1F3B1F0093AF16C9
:10C4A0001093B0162093B1163093B21610161106E1
:10C4B000120613060CF0D8C04091B3165091B41672
:10C4C0006091B5167091B616481759076A077B0731
:10C4D0000CF0CAC08091A7169091A816A091A91639
:10C4E000B091AA16081B190B2A0B3B0B0093AF1631
:10C4F0001093B0162093B1163093B2168091AB16FC
:10C50000882381F080912116909122162091AC16FB
:10C51000332727FD3095820F931F90932216809327
:10C52000211674C09091AD168091931681119C25AF
:10C53000E091AE03F091AF038091B2032081992383
:10C5400049F0AE0102C0440F551F8A95E2F7242B33
:10C5500020830AC0BE0102C0660F771F8A95E2F7EA
:10C56000CB018095822380838091AD168823A1F032
:10C570008091C3039091C403009749F1E091C503F2
:10C58000F091C603808190E00090C70302C09595AA
:10C5900087950A94E2F713C08091BC039091BD0384
:10C5A0000097A9F0E091BE03F091BF03808190E075
:10C5B0000090C00302C0959587950A94E2F78170B8
:10C5C000907090919216981711F00C947C6BE091FA
:10C5D000A703F091A8032081CE010090AB0302C015
:10C5E000880F991F0A94E2F7282B2083E091A70374
:10C5F000F091A8032081CE010090AB0302C0880F08
:10C60000991F0A94E2F780958223808380913416E3
:10C6100090913516A0913616B09137164091AC1610
:10C62000552747FD5095652F752F840F951FA61F21
:10C63000B71F8093341690933516A0933616B09397
:10C6400037168091B3169091B416A091B516B0919B
:10C65000B6160196A11DB11D8093B3169093B41622
:10C66000A093B516B093B6168091D716882309F417
:10C67000FAC08091E0169091E116A091E216B09177
:10C68000E3160091D8161091D9162091DA16309140
:10C69000DB16080F191F2A1F3B1F0093D816109393
:10C6A000D9162093DA163093DB16101611061206EF
:10C6B00013060CF0D8C04091DC165091DD16609145
:10C6C000DE167091DF16481759076A077B070CF0D2
:10C6D000CAC08091D0169091D116A091D216B09177
:10C6E000D316081B190B2A0B3B0B0093D81610937B
:10C6F000D9162093DA163093DB168091D41688234E
:10C7000081F080912316909124162091D51633271D
:10C7100027FD3095820F931F909324168093231644
:10C7200074C09091D6168091BC1681119C25E09121
:10C73000D103F091D2038091D5032081992349F050
:10C74000DE0102C0AA0FBB1F8A95E2F72A2B2083C5
:10C750000AC08E0102C0000F111F8A95E2F7C801BE
:10C760008095822380838091D6168823A1F08091C2
:10C77000E6039091E703009749F1E091E803F09117
:10C78000E903808190E00090EA0302C095958795C7
:10C790000A94E2F713C08091DF039091E0030097C1
:10C7A000A9F0E091E103F091E203808190E0009034
:10C7B000E30302C0959587950A94E2F78170907023
:10C7C0009091BB16981711F00C94806BE091CA03FE
:10C7D000F091CB032081CE010090CE0302C0880FE0
:10C7E000991F0A94E2F7282B2083E091CA03F09165
:10C7F000CB032081CE010090CE0302C0880F991F89
:10C800000A94E2F780958223808380913816909174
:10C810003916A0913A16B0913B164091D51655277E
:10C8200047FD5095652F752F840F951FA61FB71FC5
:10C830008093381690933916A0933A16B0933B160E
:10C840008091DC169091DD16A091DE16B091DF1676
:10C850000196A11DB11D8093DC169093DD16A09367
:10C86000DE16B093DF1680910017882309F4F9C013
:10C870008091091790910A17A0910B17B0910C178E
:10C88000009101171091021720910317309104179E
:10C89000080F191F2A1F3B1F00930117109302173F
:10C8A000209303173093041710161106120613066F
:10C8B0000CF0D7C0409105175091061760910717EB
:10C8C00070910817481759076A077B070CF0C9C011
:10C8D0008091F9169091FA16A091FB16B091FC1672
:10C8E000081B190B2A0B3B0B00930117109302171F
:10C8F00020930317309304178091FD16882381F04D
:10C9000080912516909126162091FE16332727FD3B
:10C910003095820F931F909326168093251673C02F
:10C920009091FF168091E51681119C25E091F4030A
:10C93000F091F5038091F8032081992349F0AE012D
:10C9400002C0440F551F8A95E2F7242B20830AC0AA
:10C95000BE0102C0660F771F8A95E2F7CB01809572
:10C96000822380838091FF168823A1F0809109049F
:10C9700090910A04009741F1E0910B04F0910C04AE
:10C98000808190E000900D0402C0959587950A94EF
:10C99000E2F713C080910204909103040097A1F084
:10C9A000E0910404F0910504808190E00090060479
:10C9B00002C0959587950A94E2F7817090709091E6
:10C9C000E416981709F0A0C6E091ED03F091EE038C
:10C9D0002081CE010090F10302C0880F991F0A94B4
:10C9E000E2F7282B2083E091ED03F091EE03208104
:10C9F000CE010090F10302C0880F991F0A94E2F75C
:10CA000080958223808380913C1690913D16A09161
:10CA10003E16B0913F164091FE16552747FD5095A2
:10CA2000652F752F840F951FA61FB71F80933C1687
:10CA300090933D16A0933E16B0933F168091051734
:10CA400090910617A0910717B09108170196A11DA4
:10CA5000B11D8093051790930617A0930717B09305
:10CA6000081780918E0D90918F0DA091900DB0912F
:10CA7000910D0196A11DB11D80938E0D90938F0D88
:10CA8000A093900DB093910D80918E0D90918F0D8C
:10CA9000A091900DB091910DE091A00DF091A10D9C
:10CAA000448955896689778984179507A607B7074A
:10CAB00020F483948D140CF459CA40918E0D50913A
:10CAC0008F0D6091900D7091910DE091A00DF091FE
:10CAD000A10D84A595A5A6A5B7A584179507A607BA
:10CAE000B70708F4BDC08090B00D9090B10DA09034
:10CAF000B20DB090B30D44A955A966A977A99501C7
:10CB00008401AA27059FB12D169FE001269FD00D15
:10CB1000259FC00DD11D069FB00DC11DDA1F159FA9
:10CB2000B00DC11DDA1F249FB00DC11DDA1F149F67
:10CB3000B10DCA1FDA1FB695CA1FDA1F1124DF0113
:10CB4000AA59BF4F8D919C918C0F9D1F9093AF0D53
:10CB50008093AE0DE25AFF4F408151816281738113
:10CB6000A0E0B0E0481759076A077B0720F450930C
:10CB7000AF0D4093AE0D8091AE0D9091AF0D9F34EF
:10CB800060F09D3930F4E3E096958795EA95E1F7FA
:10CB900002C088E893E128E014C0983230F09695FE
:10CBA00087959695879524E00CC0943120F0969552
:10CBB000879522E006C08032910510F480E290E073
:10CBC00021E02093AA0D809718E080309107C8F0EB
:10CBD000E92FF0E0EE0FFF1FEE0FFF1FED56F84FAD
:10CBE00045915591659174916A01AB01AA27859F82
:10CBF0009001849F210D3A1F06942A1F3A1F112489
:10CC00001AC0FC01F695E795EC7FED56F44F45917F
:10CC10005591659174916A0190E087709070869F3C
:10CC20009001879F300D969F300D112443E036957B
:10CC300027954A95E1F7C21AD30AD0922901C092EA
:10CC40002801EE24FF24C80CD91CEA1CFB1CC0924E
:10CC5000B00DD092B10DE092B20DF092B30D3AC189
:10CC600040918E0D50918F0D6091900D7091910DAE
:10CC700080A991A9A2A9B3A92091B50D3091B60DB3
:10CC800084179507A607B70708F00FC121153105CE
:10CC900031F481E090E09093B60D8093B50D8091D2
:10CCA000B50D9091B60D8130910571F482E090E060
:10CCB0009093B60D8093B50D1092B70D1092B80DEC
:10CCC0001092B90D1092BA0DDF01A05CBF4F4091D8
:10CCD000B70D5091B80D6091B90D7091BA0D8D914D
:10CCE0009D910D90BC91A02D480F591F6A1F7B1F6D
:10CCF0004093B70D5093B80D6093B90D7093BA0D72
:10CD00008090A60D9090A70DA090A80DB090A90DB1
:10CD100044A955A966A977A995018401AA27059F69
:10CD2000B12D169FC001269F900D259F800D911D4E
:10CD3000069FB00D811D9A1F159FB00D811D9A1F72
:10CD4000249FB00D811D9A1F149FB10D8A1F9A1F39
:10CD5000B6958A1F9A1F11249093BC0D8093BB0D2A
:10CD60004091AE0D5091AF0D2091A00D3091A10DCD
:10CD70004817590758F426593F4FD9018D919C9176
:10CD800011979093BC0D8093BB0D1AC0FA01E81B5C
:10CD9000F90BCF01F093BC0DE093BB0D26593F4F2B
:10CDA000D9014D915D916D917C91A0E0B0E0841727
:10CDB0009507A607B70720F45093BC0D4093BB0D11
:10CDC0008091BB0D9091BC0D9F3460F09D3930F483
:10CDD00023E0969587952A95E1F702C088E893E1CC
:10CDE00028E014C0983230F09695879596958795EF
:10CDF00024E00CC0943120F09695879522E006C07F
:10CE00008032910510F480E290E021E02093AA0D99
:10CE10008097B8E080309B07C8F0E92FF0E0EE0F74
:10CE2000FF1FEE0FFF1FED56F84F4591559165918D
:10CE300074916A01FB01AA278F9F90018E9F210D9B
:10CE40003A1F06942A1F3A1F11241AC0FC01F695B6
:10CE5000E795EC7FED56F44F4591559165917491AE
:10CE60006A0190E087709070869F9001879F300DD7
:10CE7000969F300D1124C3E036952795CA95E1F7AA
:10CE8000C21AD30AD0922901C0922801EE24FF24AD
:10CE9000C80CD91CEA1CFB1CC092A60DD092A70D91
:10CEA000E092A80DF092A90D15C02115310531F4BD
:10CEB00081E090E09093B60D8093B50D8091AB0D1D
:10CEC0009091AC0D90932901809328018091AD0D34
:10CED0008093AA0D40918E0D50918F0D6091900D11
:10CEE0007091910DE091A00DF091A10D848995892B
:10CEF000A689B789481759076A077B0708F4E0C372
:10CF00001092A10D1092A00D9091CA0D8091C90DA3
:10CF1000981731F08091C90D8F5F8F708093C90D84
:10CF20009091CA0D8091C90D9817A1F02091C90D5B
:10CF300030E087E790E0289FF001299FF00D389FAF
:10CF4000F00D1124E553F24FDF01AC58BF4F81E0E3
:10CF50008C9302C0E0E0F0E0F093A10DE093A00D0F
:10CF6000309709F4AFC3808D918DA28DB38D8093DE
:10CF70002C1690932D16A0932E16B0932F16848DF9
:10CF8000958DA68DB78D8093301690933116A09312
:10CF90003216B093331680A191A1A2A1B3A18093C0
:10CFA000341690933516A0933616B093371684A195
:10CFB00095A1A6A1B7A18093381690933916A09396
:10CFC0003A16B0933B1680A591A5A2A5B3A5809370
:10CFD0003C1690933D16A0933E16B0933F1682AD3B
:10CFE0008093A20D8091A30D8823E1F18F01C4EA03
:10CFF000DDE06CE97DE040E050E0F8018485958556
:10D00000A685B7850097A105B10511F18881882310
:10D01000F9F0FA01E656F24F8081FA01EE0FFF1F98
:10D02000ED5DF94E882349F080819181DB012D91DE
:10D030003C911197821B930B08C080819181DB0189
:10D040002D913C911197820F931F918380831882B9
:10D050004F5F5F4F0C5F1F4F21966E5F7F4F4230D7
:10D06000510559F61092A60D1092A70D1092A80D19
:10D070001092A90DC091A00DD091A10DFE01E25A10
:10D08000FF4F208131813F3460F03D3930F443E07F
:10D09000369527954A95E1F702C028E833E188E004
:10D0A00014C0383230F0369527953695279584E0B0
:10D0B0000CC0343120F03695279582E006C020322E
:10D0C000310510F420E230E081E08093AA0D205277
:10D0D0003040B8E020303B07C8F0E32FF0E0EE0F1F
:10D0E000FF1FEE0FFF1FED56F84F85919591A5910B
:10D0F000B491AC01BD01AA27279FC001269F810DD5
:10D100009A1F06948A1F9A1F11241AC0F901F695D6
:10D11000E795EC7FED56F44F85919591A591B491EB
:10D12000AC0130E0277030702A9FC0012B9F900D1A
:10D130003A9F900D112413E0969587951A95E1F783
:10D14000481B590B5093AC0D4093AB0D8091AA0D29
:10D150008093AD0DFE01EE58FF4F8081882309F4C6
:10D1600072C0CA59DF4F288139813093AF0D2093A7
:10D17000AE0D3F3460F03D3930F4A3E0369527958D
:10D18000AA95E1F702C028E833E188E014C03832FC
:10D1900030F0369527953695279584E00CC03431CC
:10D1A00020F03695279582E006C02032310510F434
:10D1B00020E230E081E08093AA0D20523040E8E088
:10D1C00020303E07C8F0E32FF0E0EE0FFF1FEE0F18
:10D1D000FF1FED56F84F85919591A591B491AC0143
:10D1E000BD01AA27279FC001269F810D9A1F069483
:10D1F0008A1F9A1F11241AC0F901F695E795EC7F52
:10D20000ED56F44F85919591A591B491AC0130E024
:10D21000277030702A9FC0012B9F900D3A9F900D70
:10D22000112463E0969587956A95E1F7481B590BA1
:10D23000CA01A0E0B0E08093B00D9093B10DA0932F
:10D24000B20DB093B30D5093290140932801E091A2
:10D25000A00DF091A10D80AD8093B40DEA58FF4F61
:10D2600020818091231690912416009709F0236065
:10D270008091251690912616009709F024608091E0
:10D280002116281709F442C0EFE6F3E0EF012496D7
:10D2900040E050E061E070E0CB01042E02C0880F56
:10D2A000991F0A94E2F7A82F3091211632273823CC
:10D2B00031F1A22390912116AA2389F0982B909303
:10D2C0002116A081B1813C91CB01088002C0880F5A
:10D2D000991F0A94E2F7809583238C9310C0809560
:10D2E000892380932116A081B1813C91CB010880D4
:10D2F00002C0880F991F0A94E2F7382B3C934F5FC6
:10D300005F4FB396A3964530510531F6E091A00DDD
:10D31000F091A10DDF01AB58BF4FDC917489658995
:10D3200056894789C091B40D0081118122813381D2
:10D3300081E0011511052105310509F480E0809394
:10D340005C16882309F444C0872F962FA52FB42F8D
:10D35000EE24E394EC22AC01BD01759567955795D9
:10D36000479570956095509541955F4F6F4F7F4FF2
:10D3700040935D1650935E1660935F16709360162F
:10D3800041E0D11140E0409354168093551690939C
:10D390005616A0935716B09358160093651610931F
:10D3A00066162093671630936816EE2011F08FEF03
:10D3B00001C081E080935A1681E08E2580935B1630
:10D3C00010926116109262161092631610926416F3
:10D3D0007489658956894789048115812681378139
:10D3E00081E0011511052105310509F480E08093E4
:10D3F0008516882309F446C0872F962FA52FB42FB2
:10D40000EE24E394C1FFEE24AC01BD017595679550
:10D410005795479570956095509541955F4F6F4F23
:10D420007F4F4093861650938716609388167093AB
:10D43000891641E0D13009F040E040937D16809399
:10D440007E1690937F16A0938016B093811600935A
:10D450008E1610938F162093901630939116EE200F
:10D4600011F08FEF01C081E08093831681E08E255B
:10D470008093841610928A1610928B1610928C1636
:10D4800010928D16748965895689478900851185A2
:10D490002285338581E0011511052105310509F447
:10D4A00080E08093AE16882309F446C0872F962F1C
:10D4B000A52FB42FEE24E394C2FFEE24AC01BD01EE
:10D4C00075956795579547957095609550954195D9
:10D4D0005F4F6F4F7F4F4093AF165093B0166093DE
:10D4E000B1167093B21641E0D23009F040E040939B
:10D4F000A6168093A7169093A816A093A916B0938A
:10D50000AA160093B7161093B8162093B916309345
:10D51000BA16EE2011F08FEF01C081E08093AC16B7
:10D5200081E08E258093AD161092B3161092B4163A
:10D530001092B5161092B616748965895689478976
:10D54000048515852685378581E00115110521059E
:10D55000310509F480E08093D716882309F446C08A
:10D56000872F962FA52FB42FEE24E394C3FFEE242C
:10D57000AC01BD0175956795579547957095609578
:10D58000509541955F4F6F4F7F4F4093D816509302
:10D59000D9166093DA167093DB1641E0D33009F0A8
:10D5A00040E04093CF168093D0169093D116A0936D
:10D5B000D216B093D3160093E0161093E116209381
:10D5C000E2163093E316EE2011F08FEF01C081E0F8
:10D5D0008093D51681E08E258093D6161092DC16A6
:10D5E0001092DD161092DE161092DF16DF01AB5896
:10D5F000BF4FDC91E48805893689278940895189A4
:10D600006289738981E0411551056105710509F44D
:10D6100080E080930017882309F445C08E2D902F59
:10D62000A32FB22FE1E0C4FFE0E08C019D0135950E
:10D6300027951795079530952095109501951F4FC3
:10D640002F4F3F4F0093011710930217209303179A
:10D650003093041721E0D43009F020E02093F8162D
:10D660008093F9169093FA16A093FB16B093FC16CC
:10D670004093091750930A1760930B1770930C1778
:10D68000EE2311F08FEF01C081E08093FE1681E060
:10D690008E278093FF16109205171092061710928E
:10D6A0000717109208171092B60D1092B50D109230
:10D6B0008E0D10928F0D1092900D1092910D02C050
:10D6C00080E001C081E0DF91CF911F910F91FF9029
:10D6D000EF90DF90CF90BF90AF909F908F907F9012
:10D6E0006F905F904F900895109227160C94F860F9
:10D6F000109228160C94F761109229160C94F66279
:10D7000010922A160C94F56310922B166CC9709126
:10D71000BD0D7F5F7093BD0D8091BE0D8F5F8093B7
:10D72000BE0D5091BF0D6091C10D40E081E090E0D1
:10D7300052C02091BC16E091D103F091D2037081C8
:10D74000222309F0EDC09C010090D50302C0220FF6
:10D75000331F0A94E2F72095272320832091231674
:10D76000309124162F5F3F4F21C020912316309116
:10D770002416121613066CF52091BC16E091D10305
:10D78000F091D2037081222309F0D5C09C01009052
:10D79000D50302C0220F331F0A94E2F7722B708365
:10D7A00020912316309124162150304030932416B6
:10D7B00020932316E091CA03F091CB0370819C0162
:10D7C0000090CE0302C0220F331F0A94E2F7722B9F
:10D7D00070834F5F70E0209123163091241621153D
:10D7E000310511F0751760F47093BD0D5091C00DA7
:10D7F0006091C20D7091BE0D40E081E090E06BC081
:10D80000461791F3E091CA03F091CB0370819C011C
:10D810000090CE0302C0220F331F0A94E2F7209536
:10D8200027232083209123163091241637FF9DCF84
:10D8300080CF2091E516E091F403F091F50370811B
:10D84000222309F084C09C010090F80302C0220F3B
:10D85000331F0A94E2F72095272320832091251671
:10D86000309126162F5F3F4F21C020912516309111
:10D870002616121613066CF52091E516E091F403B6
:10D88000F091F5037081222309F06CC09C01009097
:10D89000F80302C0220F331F0A94E2F7722B708341
:10D8A00020912516309126162150304030932616AF
:10D8B00020932516E091ED03F091EE0370819C0119
:10D8C0000090F10302C0220F331F0A94E2F7722B7B
:10D8D00070834F5F70E02091251630912616211538
:10D8E000310509F44BC0751708F448C0461709F410
:10D8F00045C0E091ED03F091EE0370819C01009032
:10D90000F10302C0220F331F0A94E2F72095272368
:10D910002083209125163091261637FFA6CF89CF78
:10D920009C010090D50302C0220F331F0A94E2F736
:10D93000722B708313CF9C010090D50302C0220F7D
:10D94000331F0A94E2F720952723208329CF9C01D7
:10D950000090F80302C0220F331F0A94E2F7722BE3
:10D9600070837CCF9C010090F80302C0220F331F0C
:10D970000A94E2F720952723208392CF7093BE0D5F
:10D9800008952F923F924F925F927F928F929F9233
:10D99000AF92BF92CF92DF92EF92FF920F931F93BD
:10D9A000CF93DF9300D0CDB7DEB71092A20D12E96E
:10D9B000412E1DE0512E0DEB202E0DE0302E81EC7E
:10D9C000A82E8DE0B82E8FEB9DE09A838983882462
:10D9D000992477247394F201C190D190E190F19051
:10D9E0002F01882D8D5F0E9490839B01AC01C701A0
:10D9F000B6010E94C1E19B01AC0160E070E48CE1E2
:10DA000096E40E94E8DFC62EE72E182F092F980112
:10DA1000862F9E2DA32FB22FBC01CD0120E030E038
:10DA200040E85FE30E94BDE1980118166CF48C2D6C
:10DA30009E2DA32FB22FBC01CD010E94D1DFC62E97
:10DA4000E72E182F092F12C08C2D9E2DA32FB22F39
:10DA5000BC01CD0120E030E040E85FE30E94E4DF5C
:10DA600087FF04C0CC24EE2410E000E098018C2D48
:10DA70009E2DA32FB02FBC01CD010E948FE0F62E6A
:10DA8000E981FA816193FA83E983F50110826623C3
:10DA9000A1F460E070E080E89FE3412FF02F0C2DAF
:10DAA0001E2D242F3F2FA90198010E94E8DF0E941C
:10DAB000D1DF0E948FE0F5016083F501808188232A
:10DAC00009F47082F401EE0FFF1FED5DF94E118233
:10DAD0001082F101F1921F010894811C911C08949D
:10DAE000A11CB11CF2E08F16910409F074CF0F90C5
:10DAF0000F90DF91CF911F910F91FF90EF90DF90EA
:10DB0000CF90BF90AF909F908F907F905F904F90FD
:10DB10003F902F9008952091CA0D9091C90D81E0FA
:10DB2000291380E00895CF92DF92EF92FF920F9336
:10DB30001F93CF93DF93E9012FB7F894DC01CD90C9
:10DB4000DD90ED90FC90C0922C16D0922D16E092B4
:10DB50002E16F0922F16FB0180819181A281B38154
:10DB60008093301690933116A0933216B0933316EB
:10DB7000FA0180819181A281B381809334169093C0
:10DB80003516A0933616B093371688819981AA81ED
:10DB9000BB818093381690933916A0933A16B093B0
:10DBA0003B16F80180819181A281B38180933C165C
:10DBB00090933D16A0933E16B0933F162FBFDF9172
:10DBC000CF911F910F91FF90EF90DF90CF9008952C
:10DBD000CF92DF92EF92FF920F931F93CF93DF9339
:10DBE000FB01EA0169012FB7F89440912C1650917E
:10DBF0002D1660912E1670912F16DC014D935D93BA
:10DC00006D937C9313978091301690913116A0916B
:10DC10003216B091331680839183A283B3838091AF
:10DC2000341690913516A0913616B0913716888328
:10DC30009983AA83BB838091381690913916A0915D
:10DC40003A16B0913B16F60180839183A283B38389
:10DC500080913C1690913D16A0913E16B0913F16D2
:10DC6000F80180839183A283B3838091A20DD701B1
:10DC70008C932FBFDF91CF911F910F91FF90EF9069
:10DC8000DF90CF900895809173008D7F8093730013
:10DC900006C08091C90D8F5F8F708093C90D9091E0
:10DCA000CA0D8091C90D981709F05DC01092A10DA1
:10DCB0001092A00D2FB7F89480912C1690912D16EC
:10DCC000A0912E16B0912F16809350159093511558
:10DCD000A0935215B0935315809130169091311640
:10DCE000A0913216B0913316809354159093551528
:10DCF000A0935615B0935715809134169091351610
:10DD0000A0913616B09137168093581590935915F7
:10DD1000A0935A15B0935B158091381690913916DF
:10DD2000A0913A16B0913B1680935C1590935D15C7
:10DD3000A0935E15B0935F1580913C1690913D16AF
:10DD4000A0913E16B0913F16809360159093611597
:10DD5000A0936215B09363152FBF8091730082600A
:10DD60008093730008959091CA0D8091C90D981702
:10DD700009F495CF8ECF8093A30D81E08093A40DFD
:10DD80008093A50D089583EC9DE06DE97AE140E074
:10DD90000E942EDA08959C0190EC80E4889410F0A3
:10DDA000381710F0381B892B9695220F331F8927BF
:10DDB0009E7FA9F710F0220F8307891F08952F92E5
:10DDC0003F924F925F926F927F928F929F92AF920B
:10DDD000BF92CF92DF92EF92FF920F931F93CF9358
:10DDE000DF93CDB7DEB768970FB6F894DEBF0FBEEE
:10DDF000CDBF1C0168017901FC01EE58FF4F808105
:10DE00008823C1F08A019B01013040E0140741E002
:10DE1000240740E0340724F000E010E021E030E087
:10DE200051E0C51650E0D50651E0E50650E0F50694
:10DE30002CF409C000E010E021E030E0C12CD12C2E
:10DE400081E0E82EF12C8EE5882E912C820C931C1B
:10DE5000F40180819181A281B38177276627A9018E
:10DE600098010E9444DEDC01CB0180509048AF4F06
:10DE7000BF4F8D01332717FD3095232F09831A8358
:10DE80002B833C83F40180819181A281B381772728
:10DE90006627A70196010E9444DEDC01CB01805079
:10DEA0009048AF4FBF4F4D01BB2497FCB094AB2CB3
:10DEB0008D829E82AF82B88609811A812B813C8136
:10DEC000083711052105310548F4B8E78B2E912C50
:10DED000A12CB12C89829A82AB82BC820D811E81D9
:10DEE0002F813885083711052105310548F4A8E749
:10DEF0008A2E912CA12CB12C8D829E82AF82B88665
:10DF000069817A818B819C819B01AC010E9424E212
:10DF100069877A878B879C876D817E818F819885C1
:10DF20009B01AC010E9424E26D877E878F87988BCE
:10DF3000910122593F4FD901ED90FD900D911C9117
:10DF40001397ED8AFE8A0F8B188F67017801CC0C2E
:10DF5000DD1CEE1CFF1CF101EE58FF4F8081882371
:10DF6000B9F1F101EE59FF4F80809180A280B3801A
:10DF7000C114D104E104F10489F0C501B40109859B
:10DF80001A852B853C85601B710B820B930BA701B7
:10DF900096010E9498E229013A0103C044245524C5
:10DFA000320122273327A9012C193D094E095F09A7
:10DFB000B9F06D857E858F859889681979098A09F8
:10DFC0009B090E9498E2298B3A8B4B8B5C8B0CC08F
:10DFD000198A1A8A1B8A1C8A44245524320104C0D7
:10DFE000198A1A8A1B8A1C8AD10154968D909D9099
:10DFF000AD90BC905797D501C40184199509A60925
:10E00000B70909891A892B893C89801B910BA20BBE
:10E01000B30BB7FF40C0C114D104E104F10429F1EE
:10E02000C701B601A50194010E9424E2DC01CB01E5
:10E0300009851A852B853C85801B910BA20BB30BA0
:10E040000D851E852F853889800F911FA21FB31F54
:10E05000A7019601220F331F441F551FBC01CD019C
:10E060000E9498E289019A0104C000E010E020E0DB
:10E0700030E02801390137FF03C044245524320120
:10E08000481459046A047B0414F02401350180E02B
:10E0900090E0A0E0B0E053014201880E991EAA1E54
:10E0A000BB1E8D869E86AF86B88AF10123AD2223E2
:10E0B00009F42BC10097A105B10509F07FC0C30188
:10E0C000B2016F5F7F4F8F4F9F4F97FF24C0909596
:10E0D0008095709561957F4F8F4F9F4F2D893E8919
:10E0E0004F89588D0E9424E2AB01BC01440F551F9B
:10E0F000661F771F89849A84AB84BC8448155905B0
:10E100006A057B0508F051C0D501C401841B950B3D
:10E11000A60BB70B14C02D893E894F89588D0E94DC
:10E1200024E2DC01CB01880F991FAA1FBB1FE984E1
:10E13000FA840B851C858E0D9F1DA01FB11F80309A
:10E1400000E8900700E0A00700E0B00758F40E9444
:10E15000CB6E6C01EE24D7FCE094FE2C7601DD241E
:10E16000CC2426C000E072E0B695A79597958795D8
:10E170007A95D1F70F5F803010E8910710E0A10782
:10E1800010E0B10780F70E94CB6E6C01EE24D7FC43
:10E19000E094FE2C7601DD24CC2404C0CC0CDD1CE4
:10E1A000EE1CFF1C0A95D2F703C0CC24DD247601B7
:10E1B0006701FF24D7FCF094EF2C07C0F101E25A6D
:10E1C000FF4FC080D180E280F38014141504160440
:10E1D0001704E4F46091B5157091B6158091B715E8
:10E1E0009091B8159701860189809A80AB80BC8098
:10E1F000081919092A093B09A801332722270E9477
:10E2000044DEDC01CB014D01B7FF02C08824992414
:10E210004D855E856F8578894F5F5F4F6F4F7F4F6C
:10E22000F10184899589A689B789481759076A0732
:10E230007B070CF073C00091B5151091B6152091B5
:10E24000B7153091B81509871A872B873C87970136
:10E2500086014D815E816F817885041B150B260B2D
:10E26000370BA8013327222769857A858B859C8502
:10E270000E9444DEDC01CB016D016091B11570910B
:10E28000B2158091B3159091B41561157105810592
:10E290009105A1F120E030E044E650E00E9444DE28
:10E2A00069877A878B879C87F101E259FF4F8081CC
:10E2B0009181A281B38115E0B595A7959795879532
:10E2C0001A95D1F777276627E988FA880B891C8980
:10E2D000A701332722270E94C2DE9B01AC0169857A
:10E2E0007A858B859C850E9444DEDC01CB01CD01C3
:10E2F000BB2797FDB095AB2FB7FF04C080E090E03F
:10E30000A0E0B0E0D7FE10C00DC080E090E0A0E03B
:10E31000B0E0CC24DD248824992406C080E090E07D
:10E32000A0E0B0E0CC24DD242FB7F894F101EC5844
:10E33000FF4F3081332309F040C0F101EE58FF4F09
:10E340003081332369F0F10144A655A666A677A66D
:10E35000ED84FE840F851889E0AAF1AA02AB13AB05
:10E3600081010A591F4F49815A816B817C81F801D3
:10E370004083518362837383810106591F4F4D810E
:10E380005E816F817885F801408351836283738356
:10E39000F10195AE84AED7AEC6AEEC5BFF4F1182F5
:10E3A0001082F101EA5BFF4F11821082F101E05C03
:10E3B000FF4F80839183A283B3832FBF68960FB6EC
:10E3C000F894DEBF0FBECDBFDF91CF911F910F91AB
:10E3D000FF90EF90DF90CF90BF90AF909F908F9085
:10E3E0007F906F905F904F903F902F9008952F9265
:10E3F0003F924F925F926F927F928F929F92AF92D5
:10E40000BF92CF92DF92EF92FF920F931F93CF9321
:10E41000DF9300D000D000D0CDB7DEB79E838D83D0
:10E420001B01009709F4AAC16115710509F4A6C181
:10E430009C01205B3F4FD9018D919D910D90BC9126
:10E44000A02D89839A83AB83BC836D817E81645BBD
:10E450007F4FFB0180819181A281B38129813A8123
:10E460004B815C8182179307A407B50709F486C125
:10E47000AD81BE81A35ABF4F8C91882309F069C139
:10E48000D101AD58BF4F8C91882309F462C1D101ED
:10E49000A45BBF4F8D919D910D90BC91A02D8217D3
:10E4A0009307A407B5070CF054C19C01AD016CE0C3
:10E4B00055954795379527956A95D1F7ED81FE815A
:10E4C000E85AFF4F80809180A280B380B094A094DE
:10E4D00090948094811C911CA11CB11C76E0B59491
:10E4E000A794979487947A95D1F7ED81FE81EC5AA1
:10E4F000FF4FC080D180E280F38015E0F594E7946F
:10E50000D794C7941A95D1F7CA01B9010E9444DE85
:10E510002B013C01C701B601A50194010E9444DE14
:10E52000DC01CB01A3019201281B390B4A0B5B0BC9
:10E53000DA01C90100E00097A105B10509F44BC05B
:10E54000AC01BD01407050706070707E4115510586
:10E550006105710549F432E0880F991FAA1FBB1F9E
:10E560003A95D1F70F5FE7CF181619061A061B0662
:10E5700094F5CD01BB2797FDB095AB2F0730A8F0E0
:10E580000E94CB6EAC01662757FD6095762FBA01CD
:10E5900055274427802F90E0069704C0759567950E
:10E5A000579547958A95D2F71AC00E94CB6EAC0159
:10E5B000662757FD6095762FBA015527442786E0D8
:10E5C00090E0801B910904C0440F551F661F771F00
:10E5D0008A95D2F704C040E050E060E070E08981A5
:10E5E0009A81AB81BC8184179507A607B7074CF4C5
:10E5F000ED81FE81E05BFF4F80819181A281B3813B
:10E600009FC0F101E45BFF4F0081118122813381C2
:10E610006CE035952795179507956A95D1F7ED81AB
:10E62000FE81E85AFF4F80809180A280B380B09431
:10E63000A09490948094811C911CA11CB11C76E044
:10E64000B594A794979487947A95D1F7ED81FE813C
:10E65000EC5AFF4FC080D180E280F380A5E0F594B2
:10E66000E794D794C794AA95D1F7C901B801A90135
:10E6700098010E9444DE2B013C01C701B601A501AF
:10E6800094010E9444DEDC01CB01A3019201281B0E
:10E69000390B4A0B5B0BDA01C90100E00097A105B9
:10E6A000B10509F449C0AC01BD0140705070607003
:10E6B000707E411551056105710549F452E0880FDE
:10E6C000991FAA1FBB1F5A95D1F70F5FE7CF1816E6
:10E6D00019061A061B0684F5CD01BB2797FDB095D8
:10E6E000AB2F0730A0F00E94CB6EAA2797FDA09514
:10E6F000BA2FDC019927882710E00650104004C08B
:10E70000B595A795979587950A95D2F719C00E9458
:10E71000CB6EAA2797FDA095BA2FDC0199278827F1
:10E7200026E030E0201B310904C0880F991FAA1F82
:10E73000BB1F2A95D2F704C080E090E0A0E0B0E0D3
:10E74000ED81FE81E45BFF4F80839183A283B383DD
:10E750000FC089819A81AB81BC81FB018083918349
:10E76000A283B383ED81FE81ED58FF4F81E080836A
:10E77000ED81FE81E45AFF4F81E0808326960FB63B
:10E78000F894DEBF0FBECDBFDF91CF911F910F91E7
:10E79000FF90EF90DF90CF90BF90AF909F908F90C1
:10E7A0007F906F905F904F903F902F900895EF92E1
:10E7B000FF920F931F93CF93DF931091CA0D8FB7E2
:10E7C000F8940091C90D8FBF60E070E087E7E82EF4
:10E7D000F12C13C0112309F410E11150812F90E0A6
:10E7E0008E9DE0018F9DD00D9E9DD00D1124C553AF
:10E7F000D24FCE010E94F771BE01101759F7DF9179
:10E80000CF911F910F91FF90EF9008952F923F921B
:10E810004F925F926F927F928F929F92AF92BF9230
:10E82000CF92DF92EF92FF920F931F93CF93DF93DC
:10E8300000D000D000D0CDB7DEB79E838D831B0102
:10E84000009709F47EC1FB01EE58FF4F80818823B9
:10E8500009F477C1ED81FE81E35AFF4F808188235F
:10E8600009F06FC1ED81FE81ED58FF4F8081882353
:10E8700009F467C1ED81FE81E45BFF4F80819181E6
:10E88000A281B381645B7F4FFB0120813181428192
:10E89000538129833A834B835C8382179307A407B0
:10E8A000B5070CF04EC19C01AD016CE05595479544
:10E8B000379527956A95D1F7ED81FE81E85AFF4F8C
:10E8C00080809180A280B38076E0B594A7949794DD
:10E8D00087947A95D1F7ED81FE81EC5AFF4FC08085
:10E8E000D180E280F38015E0F594E794D794C79443
:10E8F0001A95D1F7CA01B9010E9444DE2B013C01EF
:10E90000C701B601A50194010E9444DEDC01CB01E0
:10E91000840D951DA61DB71D00E00097A105B1054A
:10E9200009F44BC0AC01BD01407050706070707E46
:10E93000411551056105710549F432E0880F991FB1
:10E94000AA1FBB1F3A95D1F70F5FE7CF181619061C
:10E950001A061B0694F5CD01BB2797FDB095AB2F8A
:10E960000730A8F00E94CB6EAC01662757FD60957A
:10E97000762FBA0155274427802F90E0069704C0D0
:10E9800075956795579547958A95D2F71AC00E9455
:10E99000CB6EAC01662757FD6095762FBA015527DF
:10E9A000442786E090E0801B910904C0440F551F66
:10E9B000661F771F8A95D2F704C040E050E060E000
:10E9C00070E089819A81AB81BC8184179507A60785
:10E9D000B70744F4F101E45BFF4F4081518162814C
:10E9E000738196C0ED81FE81E45BFF4F0081118150
:10E9F000228133816CE035952795179507956A95A7
:10EA0000D1F7ED81FE81E85AFF4F80809180A2808E
:10EA1000B38076E0B594A794979487947A95D1F7CC
:10EA2000ED81FE81EC5AFF4FC080D180E280F380FF
:10EA3000A5E0F594E794D794C794AA95D1F7C901B6
:10EA4000B801A90198010E9444DE2B013C01C701D5
:10EA5000B601A50194010E9444DEDC01CB01840DC6
:10EA6000951DA61DB71D00E00097A105B10509F48D
:10EA70004BC0AC01BD01407050706070707E41159C
:10EA800051056105710549F452E0880F991FAA1FCD
:10EA9000BB1F5A95D1F70F5FE7CF181619061A0654
:10EAA0001B0694F5CD01BB2797FDB095AB2F073022
:10EAB000A8F00E94CB6EAC01662757FD6095762FBB
:10EAC000BA015527442710E00650104004C0759540
:10EAD0006795579547950A95D2F71AC00E94CB6E55
:10EAE000AC01662757FD6095762FBA01552744275C
:10EAF00086E090E0801B910904C0440F551F661FFB
:10EB0000771F8A95D2F704C040E050E060E070E0E3
:10EB1000F101E45BFF4F80819181A281B381841771
:10EB20009507A607B70769F0408351836283738313
:10EB3000F101E45AFF4F81E08083F101ED58FF4F6E
:10EB4000808326960FB6F894DEBF0FBECDBFDF914F
:10EB5000CF911F910F91FF90EF90DF90CF90BF90DA
:10EB6000AF909F908F907F906F905F904F903F906D
:10EB70002F900895EF92FF920F931F93CF93C09120
:10EB8000C90D80E090E007E7E02EF12C13C02C2F98
:10EB900030E02E9D80012F9D100D3E9D100D112403
:10EBA0000553124FB8010E940674CF5FC03109F4BB
:10EBB000C0E0C8012091CA0DC21749F7CF911F913B
:10EBC0000F91FF90EF9008956F927F928F929F9296
:10EBD000AF92BF92CF92DF92FF920F931F93CF938A
:10EBE000DF93F090C90DC0E0D0E087E7682E712C6C
:10EBF00059C08F2D90E0869D6001879DD00C969D19
:10EC0000D00C11248BEC9DE0C80ED91E209709F47E
:10EC100043C0FE01EE58FF4F80818823E9F1F601E1
:10EC2000EE58FF4F80818823B9F1FE01E45AFF4F6F
:10EC30008081882331F4F601E45AFF4F80818823D4
:10EC400059F1FE01E45BFF4F608171818281938104
:10EC50008E01085B1F4FF801208131814281538171
:10EC60000E94C2DE4B015C01F601E45BFF4F608154
:10EC7000718182819381F8012081318142815381A8
:10EC80000E94C2DE8B019C01CE01B501A4010E944D
:10EC9000DF6EC45ADF4F1882F394F0E1FF1609F4D7
:10ECA000FF24E6018091CA0DF81609F0A2CF209743
:10ECB000D1F0FE01E45BFF4F60817181828193811D
:10ECC000FE01E85BFF4F20813181428153810E9428
:10ECD000C2DE8B019C01CE01B901A8010E94DF6E4A
:10ECE000C45ADF4F1882DF91CF911F910F91FF908F
:10ECF000DF90CF90BF90AF909F908F907F906F905C
:10ED000008950E94D7730E94BA750E94E475089511
:10ED10000F93DC01CB011092CA0D1092C90D109215
:10ED200050151092511510925215109253151092C1
:10ED300054151092551510925615109257151092A1
:10ED400058151092591510925A1510925B15109281
:10ED50005C1510925D1510925E1510925F15109261
:10ED600060151092611510926215109263158093D0
:10ED7000B5159093B615A093B715B093B815209319
:10ED8000B1153093B2154093B3155093B415009359
:10ED90003B1581E0809360030F9108952F923F927D
:10EDA0004F925F926F927F928F929F92AF92BF929B
:10EDB000CF92DF92EF92FF920F931F93CF93DF9347
:10EDC000CDB7DEB7C354D0400FB6F894DEBF0FBE48
:10EDD000CDBF6F8B788F898F9A8F5CA34BA319015E
:10EDE0008091CD159091CE15009749F09091CA0D64
:10EDF0008091C90D981719F481E0809360031091F8
:10EE0000CA0D1F5F1CA7103109F41CA68091CA0D02
:10EE100090E027E730E0829FA001839F500D929FF2
:10EE2000500D11244553524F5E8B4D8BFA01EC5817
:10EE3000FF4F1082FA01EE58FF4F0083DA01DA9695
:10EE4000EC928FB7F89400915015109151152091C4
:10EE5000521530915315ED89FE89008F118F228F45
:10EE6000338F4091541550915515609156157091FE
:10EE700057154F8F58A369A37AA3448F558F668F78
:10EE8000778F409158155091591560915A1570918E
:10EE90005B1548A759A76AA77BA740A351A362A304
:10EEA00073A340915C1550915D1560915E15709152
:10EEB0005F154DA75EA76FA778AB44A355A366A3C4
:10EEC00077A3409160155091611560916215709122
:10EED000631549AB5AAB6BAB7CAB40A751A762A79C
:10EEE00073A78FBF8090801590908115A090821598
:10EEF000B0908315ED89FE8980829182A282B382CF
:10EF000040908415509085156090861570908715F7
:10EF10004482558266827782409188155091891586
:10EF200060918A1570918B154B8F5C8F6D8F7E8FE2
:10EF30004087518762877387C0908C15D0908D155C
:10EF4000E0908E15F0908F15C486D586E686F786FC
:10EF50004091901550919115609192157091931573
:10EF6000408B518B628B738B809195159091961588
:10EF7000A0919715B0919815848B958BA68BB78B24
:10EF8000EB58FF4F80919415808381149104A10464
:10EF9000B104C9F44114510461047104A1F48B8DCE
:10EFA0009C8DAD8DBE8D0097A105B10561F4C11496
:10EFB000D104E104F10449F491E09FA34115510506
:10EFC0006105710521F41FA202C0A1E0AFA3ED8984
:10EFD000FE8910AE80913C1590913D15A0913E1593
:10EFE000B0913F1580179107A207B30714F481E091
:10EFF00080AF8091401590914115A0914215B0913C
:10F0000043150F8D18A129A13AA180179107A207D6
:10F01000B30744F4AD89BE89D8968C91D8978260A5
:10F02000D8968C938091441590914515A0914615E2
:10F03000B091471508A519A52AA53BA580179107EA
:10F04000A207B30744F4AD89BE89D8968C91D897AE
:10F050008460D8968C938091481590914915A09121
:10F060004A15B0914B150DA51EA52FA538A98017DF
:10F070009107A207B30744F4AD89BE89D8968C9155
:10F08000D8978860D8968C9380914C1590914D15A7
:10F09000A0914E15B0914F1509A91AA92BA93CA909
:10F0A00080179107A207B3074CF4AD89BE89D896A3
:10F0B0008C91D8978061D8968C93D897C114D1043D
:10F0C000E104F10449F0411551056105710559F458
:10F0D000ED89FE8911AE0EC041155105610571051E
:10F0E00011F081E002C0F1018081AD89BE89D9961D
:10F0F0008C93D99781149104A104B10429F08091D3
:10F100002216816080932216411451046104710417
:10F1100029F0809122168260809322160B8D1C8D1F
:10F120002D8D3E8D011511052105310529F08091A8
:10F130002216846080932216C114D104E104F104E4
:10F1400029F080912216886080932216411551057E
:10F150006105710529F08091221680618093221645
:10F1600080912216ED89FE89EA58FF4F80839091A5
:10F170003B15992311F0846080838091CA0D909192
:10F18000C90D891B8F70282F30E03C8F2B8F2115E4
:10F19000310541F5109207161092081610920916C3
:10F1A00010920A1610920B1610920C1610920D1651
:10F1B00010920E1610920F16109210161092111631
:10F1C0001092121610921316109214161092151611
:10F1D00010921616109217161092181610921916F1
:10F1E00010921A16EBA1FCA180819181A281B381BA
:10F1F000ED89FE89E25AFF4F80839183A283B38316
:10F200002091CD153091CE152115310509F453C04B
:10F2100080916003882349F00B8D1C8D0217130722
:10F220000CF449C01092600346C04B8D5C8D4217B0
:10F2300053070CF040C042305105ECF1CA01AA2737
:10F2400097FDA095BA2F7C01DD24CC24C901AA2703
:10F2500097FDA095BA2FAC0133272227C701B6012D
:10F260000E94C2DE6B017C016F89788D898D9A8D39
:10F27000A70196010E9444DE6F8B788F898F9A8F49
:10F280000D891E89025A1F4FF80180819181A28148
:10F29000B38177276627A70196010E9444DEDC012F
:10F2A000CB01CD01BB2797FDB095AB2FF801808333
:10F2B0009183A283B3830F89188D298D3A8D01150F
:10F2C00011052105310509F46AC02D893E892C5AA2
:10F2D0003F4F1FA11123C9F0AD89BE89D996EC918A
:10F2E000F0E0EE0FFF1FEE0FFF1FE755FA4E808193
:10F2F0009181A281B381B7FF10C0B095A095909580
:10F3000081959F4FAF4FBF4F08C080919915909145
:10F310009A15A0919B15B0919C15F901808391835A
:10F32000A283B383ED89FE89EC5AFF4F208131819E
:10F330004281538160E070E081E090E00E94C2DE93
:10F340006F8F78A389A39AA36F89788D898D9A8D01
:10F350002F8D38A149A15AA10E9444DE6B017C0186
:10F360001DE9812E15E1912E2E010894411C511C9E
:10F3700000E0D4016D917D918D919D914D01A7018A
:10F3800096010E9444DEDC01CB01F201819391934E
:10F39000A193B1932F010F5F053059F704C01F8E61
:10F3A00018A219A21AA2ED89FE89EE58FF4F80819A
:10F3B000882309F03DC1EBA1FCA180819181A2814C
:10F3C000B381ED89FE89E25AFF4F80839183A28346
:10F3D000B3830F89188D298D3A8D011511052105EB
:10F3E000310509F4A5C08E010F5F1F4F83ED282E54
:10F3F00085E1382E95E0C92E412C512C21E0622E5A
:10F40000712C58010C2DD5013C9111962C9111971E
:10F4100012969C91129713968C911397E4E0F0E06A
:10F42000AE0EBF1EC32ED22EE92EF82EF7FE08C058
:10F43000F094E094D094C094C11CD11CE11CF11C48
:10F44000D1016D917D918D919C9113976C157D05E6
:10F450008E059F05B4F4A70196010E94C2DEDC016F
:10F46000CB01481659066A067B065CF0F101608103
:10F47000718182819381A70196010E94C2DE2B01D6
:10F480003C01015024E030E0220E331E002309F03D
:10F49000BACFEBA1FCA180819181A281B3810D89BA
:10F4A0001E89025A1F4F8030F0E89F07F0E0AF0737
:10F4B000F0E0BF0730F1F80180819181A281B38132
:10F4C00024E0B695A795979587952A95D1F78083DF
:10F4D0009183A283B38377276627A30192010E94B9
:10F4E00044DEDC01CB01CD01BB2797FDB095AB2FEE
:10F4F000689413F8880F991FAA1FBB1F1694D1F7A1
:10F5000012C0F80180819181A281B381772766279B
:10F51000A30192010E9444DEDC01CB01CD01BB2797
:10F5200097FDB095AB2FF80180839183A283B383BD
:10F53000AD89BE899C961D921D921D921C929F972B
:10F54000FD0184899589A689B7890196A11DB11D00
:10F5500080AB91ABA2ABB3ABE25AFF4F20813181BC
:10F56000428153810D891E890E591F4FCA01B9016D
:10F570000E9424E2DC01CB01F80180839183A28305
:10F58000B383FCA5F093CA0D2FB7F89480913C1576
:10F5900090913D15A0913E15B0913F158093501567
:10F5A00090935115A0935215B09353158091401527
:10F5B00090914115A0914215B09143158093541537
:10F5C00090935515A0935615B093571580914415F7
:10F5D00090914515A0914615B09147158093581507
:10F5E00090935915A0935A15B0935B1580914815C7
:10F5F00090914915A0914A15B0914B1580935C15D7
:10F6000090935D15A0935E15B0935F1580914C1596
:10F6100090914D15A0914E15B0914F1580936015A6
:10F6200090936115A0936215B09363152FBF7EC5AB
:10F630000FA1002309F078C02B8D3C8D21153105D9
:10F6400009F072C08091641590916515A0916615BE
:10F65000B0916715181619061A061B060CF064C03F
:10F660000D891E890C5A1F4FD8016D917D918D9186
:10F670009C91139716161706180619060CF054C01D
:10F680002F89388D498D5A8D1216130614061506CA
:10F690000CF04AC00E94C2DEDC01CB01209164154F
:10F6A0003091651540916615509167158217930743
:10F6B000A407B507CCF5D8016D917D918D919C91F2
:10F6C0000E94C2DE062FC72E882E292EED88FE88C6
:10F6D000EEE5F0E0EE0EFF1EF70180819181A28140
:10F6E000B3813C0155244424602F7C2D882D922D1C
:10F6F0002F89388D498D5A8D0E94C2DE9B01AC0145
:10F70000C301B2010E9444DEDC01CB01CD01BB2765
:10F7100097FDB095AB2FF70180839183A283B383CC
:10F720000F8BC88E898E2A8EED89FE89E25AFF4F93
:10F7300020813181428153810D891E890E591F4FCD
:10F74000CA01B9010E9424E2DC01CB01F8018083E7
:10F750009183A283B383ED89FE89E85BFF4F0F8914
:10F76000188D298D3A8D0083118322833383ED898F
:10F77000FE8984899589A689B7898030F0E89F073A
:10F78000F0E0AF07F0E0BF0778F0B595A795979543
:10F790008795772766272F8D38A149A15AA1220F77
:10F7A000331F441F551F06C0772766272F8D38A1AA
:10F7B00049A15AA10E9444DE6F8B788F898F9A8F5E
:10F7C0000D891E8902591F4F2F89388D498D5A8DF9
:10F7D000BA01992777FD9095892F3FA1332391F0A6
:10F7E0002091EB153091EC154091ED155091EE15EF
:10F7F0000E9424E2DC01CB01F80180839183A28383
:10F80000B3830DC12091EF153091F0154091F115A2
:10F810005091F2150E9424E2DC01CB01F8018083B3
:10F820009183A283B3832D893E8938AF2FAB49EBF7
:10F8300055E158A34F8F68E675E17EAB6DAB1DA611
:10F8400019A708A7AFA9B8ADCD90DD90ED90FD90B8
:10F85000B8AFAFABC114D104E104F10409F4CEC0D8
:10F86000AD89BE8954960D911D912D913C9157976C
:10F8700009AB1AAB2BAB3CABEDA9FEA98081918102
:10F88000A281B38180179107A207B30750F1AF8D12
:10F89000B8A18D909D90AD90BC90E8A5F9A5208170
:10F8A000318142815381C701B6010E9424E26B017C
:10F8B0007C01C501B40129A93AA94BA95CA90E9400
:10F8C00024E2DC01CB018C159D05AE05BF0508F0D7
:10F8D00095C0A8A5B9A58D929D92AD92BC921397A3
:10F8E0008DC0AF8DB8A10D911D912D913C9109AFA7
:10F8F0001AAF2BAF3CAF97018601330F000B102FCF
:10F9000098010BA31CA32DA33EA3E8A5F9A5808114
:10F910009181A281B3811C012D019601A7016BA1E8
:10F92000762F862F962F51016201EE24FF2400E0EE
:10F9300010E00E94AA2224962FAF24973BA34DAF3C
:10F940005EAF6FAF21967FAF219722968FAF229740
:10F9500023969FAF239729AD3AAD4BAD5CAD5901CE
:10F960006A0149A95AA96BA97CA91A012B01950121
:10F97000A60160E070E080E090E051016201EE24B9
:10F98000FF2400E010E00E94AA222396AFAD239747
:10F990009A1748F1A91791F52296BFAD22978B17B8
:10F9A00010F1B81759F52196EFAD21977E17D8F0D1
:10F9B000E71721F5FFAD6F17B0F0F617F9F40EADAC
:10F9C000501788F00517D1F41DAD411760F01417DA
:10F9D000A9F44BA1341738F0431781F424965FAD96
:10F9E0002497251758F469AD7AAD8BAD9CADA8A5C9
:10F9F000B9A56D937D938D939C931397BDA5BF5F20
:10FA0000BDA7EF8DF8A13496F8A3EF8F0DA91EA91D
:10FA10000C5F1F4F1EAB0DABB53009F013CFED8956
:10FA2000FE89E259FF4F80819181A281B3818030AC
:10FA300010E8910710E0A10710E0B10738F477272C
:10FA400066272F89388D498D5A8D1CC0803020E063
:10FA5000920722E0A20720E0B207E8F4F2E0B595B1
:10FA6000A79597958795FA95D1F7772766272F89D8
:10FA7000388D498D5A8D02E05595479537952795D4
:10FA80000A95D1F70E94C2DEDC01CB01ED89FE8927
:10FA9000E85AFF4F3AC00D891E89085A1F4F80301F
:10FAA00030E0930738E0A30730E0B307A8F4F4E0B0
:10FAB000B595A79597958795FA95D1F777276627F6
:10FAC0002F89388D498D5A8DE4E0559547953795A6
:10FAD0002795EA95D1F714C025E0B595A795979598
:10FAE00087952A95D1F7772766272F89388D498DF5
:10FAF0005A8DE5E05595479537952795EA95D1F7C5
:10FB00000E94C2DEDC01CB01F80180839183A283D5
:10FB1000B383ED89FE89E259FF4F80809180A280F6
:10FB2000B3809401A50160E070E080E090E01FEDFB
:10FB3000A12E08E1B02E12E0C12EDD24EE24FF2418
:10FB400000E010E00E94AA220EE00E947D23AD8911
:10FB5000BE89D4962C93D497D5963C93D597D696B8
:10FB60004C93D697D7965C93D797FD01E85BFF4FF0
:10FB70000B8D1C8D01151105C9F46091CF15709185
:10FB8000D0158091D1159091D21560937C1570930A
:10FB90007D1580937E1590937F1520813181428160
:10FBA00053810E94C2DEDC01CB01E7C080819181DC
:10FBB000A281B3814091E7155091E8156091E91554
:10FBC0007091EA15481759076A077B076CF0809314
:10FBD0007C1590937D15A0937E15B0937F1580E0E2
:10FBE00090E0A1E0B0E0C9C03E010894611C711C26
:10FBF00007E016E11C8F0B8FB3ED4B2EB5E15B2EAA
:10FC000078011301CC2400E010E021E030E00F8BFC
:10FC1000188F298F3A8FAC2C4701D101CD90DD9000
:10FC2000ED90FD901D01F40141915191619171910F
:10FC30004F01C114D104E104F10409F441C0D2011F
:10FC40000D911D912D913C91D701C601841B950BFF
:10FC5000A60BB70BB7FF07C0B095A09590958195FF
:10FC60009F4FAF4FBF4F081719072A073B0744F5AF
:10FC70004C155D056E057F052CF4400F511F621F6A
:10FC8000731F04C0401B510B620B730BCB01BA01F5
:10FC9000A70196010E94C2DEDC01CB0118161906ED
:10FCA0001A061B061CF50F89188D298D3A8D8017B1
:10FCB0009107A207B30724F48F8B988FA98FBA8F6F
:10FCC000A39424E030E0420E531E35E0A31609F061
:10FCD000A4CF8F89988DA98DBA8D803040E094078C
:10FCE00041E0A40740E0B407C1F104C01F8A188EA8
:10FCF000198E1A8EED89FE89E85BFF4F6081718154
:10FD0000828193812F89388D498D5A8D0E9444DEDE
:10FD1000DC01CB0180937C1590937D15A0937E151B
:10FD2000B0937F1500E0D3016D917D918D919D91F0
:10FD30003D012F89388D498D5A8D0E9444DEDC01AA
:10FD4000CB01EB8DFC8D81939193A193B193FC8FAB
:10FD5000EB8F0F5F053039F750C0ED89FE89E85B06
:10FD6000FF4F408151816281738140937C15509394
:10FD70007D1560937E1570937F1549815A816B8143
:10FD80007C81409307165093081660930916709370
:10FD90000A164D815E816F81788540930B165093D2
:10FDA0000C1660930D1670930E1649855A856B8557
:10FDB0007C8540930F165093101660931116709324
:10FDC00012164D855E856F85788940931316509382
:10FDD0001416609315167093161649895A896B8903
:10FDE0007C894093171650931816609319167093D8
:10FDF0001A168F8B988FA98FBA8F0091CF151091FB
:10FE0000D0152091D1153091D2156CE035952795FC
:10FE1000179507956A95D1F7ED89FE89E85AFF4F46
:10FE2000C080D180E280F38076E0F594E794D794A7
:10FE3000C7947A95D1F7ED89FE89EC5AFF4F8080FF
:10FE40009180A280B380A5E0B594A79497948794FD
:10FE5000AA95D1F7C901B801A90198010E9444DE11
:10FE60002B013C01C501B401A70196010E9444DEAB
:10FE7000DC01CB01840D951DA61DB71D00E0009788
:10FE8000A105B10509F44BC0AC01BD014070507033
:10FE90006070707E411551056105710549F452E0AD
:10FEA000880F991FAA1FBB1F5A95D1F70F5FE7CF85
:10FEB000181619061A061B0694F5CD01BB2797FDE7
:10FEC000B095AB2F0730A8F00E94CB6E4C01AA244E
:10FED00097FCA094BA2C54019924882410E0065071
:10FEE000104004C0B594A794979487940A95D2F7CC
:10FEF00019C00E94CB6E4C01AA2497FCA094BA2C86
:10FF000054019924882486E090E0801B910904C064
:10FF1000880C991CAA1CBB1C8A95D2F703C08824A4
:10FF20009924540140917C1550917D1560917E1566
:10FF300070917F158091CF159091D015A091D1151A
:10FF4000B091D215ED89FE89E45BFF4F2D893E8982
:10FF5000205B3F4F481759076A077B0754F480839B
:10FF60009183A283B383F90180839183A283B383B6
:10FF70000AC04083518362837383D9014D935D939B
:10FF80006D937C931397ED89FE89E85BFF4F808129
:10FF90009181A281B381ED89FE89E35AFF4F8816D2
:10FFA0009906AA06BB061CF081E0808301C010827E
:10FFB000ED89FE89E45AFF4F81E08083ED89FE8957
:10FFC000ED58FF4F1082ED89FE89E05CFF4F1082F3
:10FFD000118212821382ED89FE8984859585A6851A
:10FFE000B7850097A105B10541F480899189A2895F
:10FFF000B3890097A105B105D9F0FFA1FF23C1F492
:020000021000EC
:100000008091B5159091B615A091B715B091B8151E
:100010000097A105B10521F58091B1159091B21518
:10002000A091B315B091B4150097A105B105C1F425
:10003000AD89BE89DB961C92DB97DD961C921E92E1
:10004000DC97DF961C921E92DE97FD01EC5BFF4F62
:1000500011821082FD01EA5BFF4F1182108204C001
:1000600081E0ED89FE8983AF8D899E894F89588D06
:10007000698D7A8D8A019B010E94DF6EFCA5F09349
:10008000CA0D2FB7F89480913C1590913D15A09121
:100090003E15B0913F158093501590935115A09344
:1000A0005215B09353158091401590914115A09130
:1000B0004215B09143158093541590935515A09314
:1000C0005615B09357158091441590914515A09100
:1000D0004615B09147158093581590935915A093E4
:1000E0005A15B0935B158091481590914915A091D0
:1000F0004A15B0914B1580935C1590935D15A093B4
:100100005E15B0935F1580914C1590914D15A0919F
:100110004E15B0914F158093601590936115A09383
:100120006215B09363152FBF0E948176CD5BDF4FC0
:100130000FB6F894DEBF0FBECDBFDF91CF911F91F8
:100140000F91FF90EF90DF90CF90BF90AF909F9076
:100150008F907F906F905F904F903F902F90089579
:10016000FF920F931F93CF93DF93F801FFB6F8949C
:10017000EC0188819981AA81BB818093501590936D
:100180005115A0935215B0935315EB0188819981B5
:10019000AA81BB818093541590935515A093561551
:1001A000B0935715EA0188819981AA81BB81809318
:1001B000581590935915A0935A15B0935B15E90102
:1001C00088819981AA81BB8180935C1590935D158C
:1001D000A0935E15B0935F1580819181A281B38158
:1001E0008093601590936115A0936215B093631589
:1001F0008091CA0D9091C90D891B8F7061F480E5C3
:1002000095E164E575E148E555E12CE535E100E669
:1002100015E10E94936DFFBEDF91CF911F910F9169
:10022000FF9008958BE196E16DE97AE140E00E944C
:100230002EDA08952F923F924F925F926F927F92A3
:100240008F929F92AF92BF92CF92DF92EF92FF92E6
:100250000F931F93CF93DF93CDB7DEB72F970FB6D2
:10026000F894DEBF0FBECDBF8B878823B1F082E04C
:1002700090E060E00E9477A9082F84E090E060E0C1
:100280000E9477A9682E8EE092E060E00E9477A934
:10029000813729F00E944A3F02C0662400E090E4C2
:1002A000A92E96E1B92E21E6822E23E0922E94010A
:1002B000275E3F4F3C832B83A4014E5E5F4F5E83DE
:1002C0004D83C40180969A838983A1E7B4E0BA87FD
:1002D000A987E6E4F2E0F887EF834424552422243A
:1002E0003324202F30E03D872C87462D50E05F8758
:1002F0004E87722C5B85552309F494C167FE0AC0B2
:100300008E859F85022C02C0959587950A94E2F709
:10031000817001C081E0D5018C938C859D85022C74
:1003200002C0959587950A94E2F7817090701196B6
:100330008C93F201E35AFB4F4081518162817381BA
:10034000C2018C559E4F0E94BBA90E94BBE020E0D9
:1003500034E244E759E40E94E8DFDC01CB01F50117
:1003600082839383A483B583A985BA856D917C919B
:100370008F8198850E9495A9BC0180E090E00E9441
:10038000BBE0DC01CB01F50186839783A087B187B1
:10039000F201E558FB4F4081518162817381C201B6
:1003A000805F9D4F0E94BBA90E94BDE0D5011296BF
:1003B0002D913D914D915C9115970E94C1E120E0F6
:1003C00030E04AE754E40E94C1E10E948AE028EE4E
:1003D00033E040E050E00E9498E269017A01B2E027
:1003E0007B1601F17B1620F0E4E0E71508F042C02F
:1003F000C701B60122E030E040E050E00E9498E200
:1004000089019A01D50150960D931D932D933C932C
:10041000539788279927DC01801B910BA20BB30B04
:10042000F50134C0C2018C5D9D4F40E050E060E0BA
:1004300070E00E94BBA90E94BBE0D50112962D91ED
:100440003D914D915C9115970E94C1E10E948AE017
:10045000DC01CB01A7019601281B390B4A0B5B0B72
:10046000F501208B318B428B538B148615861686B3
:10047000178610C0F501208B318B428B538B882758
:100480009927DC01821B930BA40BB50B84879587FE
:10049000A687B787D4011C96ED91FC911D9720810A
:1004A00081E090E01B960C901B9702C0880F991F6B
:1004B0000A94E2F7282B20831596ED91FC9116976C
:1004C000208181E090E014960C90149702C0880F70
:1004D000991F0A94E2F7282B20831E96ED91FC9138
:1004E0001F97208181E090E0AD81BE810C9002C019
:1004F000880F991F0A94E2F7282B2083D401539682
:10050000ED91FC915497208181E090E0AD81BE8116
:100510000C9002C0880F991F0A94E2F7282B2083C1
:10052000F401848D958D0097A9F101A0F2A1E02D31
:10053000208181E090E0A981BA810C9002C0880FEF
:10054000991F0A94E2F7809582238083F5018081C8
:10055000D4015C96ED91FC915D972081882369F030
:1005600081E090E0A981BA810C9002C0880F991FA8
:100570000A94E2F7282B20830DC081E090E0A98146
:10058000BA810C9002C0880F991F0A94E2F78095F7
:1005900082238083F401858996890097A9F1028CD2
:1005A000F38DE02D208181E090E0AB81BC810C9047
:1005B00002C0880F991F0A94E2F7809582238083F6
:1005C000F5018081D4015596ED91FC9156972081DB
:1005D000882369F081E090E0AB81BC810C9002C07F
:1005E000880F991F0A94E2F7282B20830DC081E021
:1005F00090E0AB81BC810C9002C0880F991F0A94D7
:10060000E2F7809582238083F101EE0FFF1FEE0F4A
:10061000FF1FE45DF94E1082118212821382F501F0
:1006200012861386F101E95DF94E108281E0F2E055
:10063000F71508F080E0D50159968C935997F5018C
:10064000158E168E178E10A221E0228F138E148A1B
:1006500055961D921D921D921C92589711A212A29E
:1006600013A214A295961D921D921D921C9298970A
:100670000894211C311CE9E2F0E0AE0EBF1E23E21B
:1006800030E0820E931E4B815C814D5D5F4F5C8339
:100690004B838D819E8183969E838D83A981BA81B0
:1006A0009396BA83A983E4E0F0E04E0E5F1E29859D
:1006B0003A852E5F3F4F3A8729874F8158854E5F95
:1006C0005F4F58874F8355E02516310409F011CE4E
:1006D0008B85882321F010922216109221161092F9
:1006E00024161092231610922616109225162F9675
:1006F0000FB6F894DEBF0FBECDBFDF91CF911F9133
:100700000F91FF90EF90DF90CF90BF90AF909F90B0
:100710008F907F906F905F904F903F902F900895B3
:1007200090E029E230E0829FF001839FF00D929FDC
:10073000F00D1124E05CF94EDF0112965281119602
:100740004C91119712963C91129713962C91852FEC
:10075000942FA32FB22FBC01CD0108950F931F93A7
:10076000CF93DF930F92CDB7DEB749830E94BDE0F0
:100770008B019C01498150E089E290E0489FF001A3
:10078000499FF00D589FF00D1124E05CF94EC9010E
:10079000B80122813381448155810E94E8DF462FD0
:1007A000572F682F792FCB01BA010F90DF91CF918E
:1007B0001F910F9108954F925F926F927F928F9247
:1007C0009F92AF92BF92CF92DF92EF92FF920F93E0
:1007D0001F93CF93DF93142F20E030E04AE754E4D7
:1007E0000E94C1E10E9450E0E901942E852E762EF0
:1007F000672E582E492E212F30E089E290E0289F65
:10080000F001299FF00D389FF00D1124E05CF94EA6
:1008100062817381848195810E9450E059016A014F
:100820007B018C019E01492D582D672D762D852D3C
:10083000942D0E94AA22A8EEAA2EB3E0BB2ECC24AF
:10084000DD24EE24FF2400E010E00E94EB23952F2E
:10085000B901842FDF91CF911F910F91FF90EF90FD
:10086000DF90CF90BF90AF909F908F907F906F90D0
:100870005F904F9008958DE097E16DE97AE140E057
:100880000E942EDA08950F931F93CF93DF93C0E059
:10089000D0E00BE010E0C09FC001C19F900DD09F41
:1008A000900D1124885A984E6C2F0E94F5A821961D
:1008B000C530D10581F7DF91CF911F910F91089538
:1008C00080915717882319F480915617089581E075
:1008D00008954F925F927F928F929F92AF92BF92B4
:1008E000CF92DF92EF92FF920F931F93CF93DF93FC
:1008F0007FB6F89408E312E0C0E0D0E0C80140E021
:1009000050E060E070E00E94BBA96B017C018C2F7D
:100910000E9490834B015C0186E197E1BE010E9439
:100920006F562C01C701B6010E94BDE0A5019401DC
:100930000E94C1E120E030E04AE754E40E94E8DF91
:100940000E948AE0DC01CB01F20180839183A283C3
:10095000B38321960C5F1F4FC330D10579F6C2E0F7
:10096000D0E086E197E1BE010E946F56FC01108243
:100970001182128213822196C530D10591F7C0E011
:10098000D0E08AE297E1BE010E946F56FC0110821E
:100990001182128213822196C530D10591F77FBE54
:1009A000DF91CF911F910F91FF90EF90DF90CF904B
:1009B000BF90AF909F908F907F905F904F900895E1
:1009C000109257171092561781E00E941A810E94C8
:1009D000438488E392E04FEF5FEF6FEF7FEF0E9479
:1009E000BBA9DC01CB018F3F2FEF92072FEFA207AE
:1009F0002FEFB20711F40E94B03E08957F928F92BC
:100A00009F92AF92BF92CF92DF92EF92FF920F939D
:100A10001F93CF93DF93CDB7DEB764970FB6F894EB
:100A2000DEBF0FBECDBFDE011196FC0184E1019057
:100A30000D928150E1F78BE4E82E86E1F82E00E07C
:100A400010E077247394F7017082CE010196B8010B
:100A50000E946F566C01FC0180809180A280B3805F
:100A60008091141790911517B8010E946F56FC01E0
:100A700080819181A281B381880D991DAA1DBB1D22
:100A8000F60180839183A283B3830F5F1F4F89E2B6
:100A900090E0E80EF91E05301105A9F6CE01019689
:100AA00060E070E00E946F567C01CE01019661E02B
:100AB00070E00E946F564C01CE01019662E070E03A
:100AC0000E946F566C01CE01019663E070E00E94B7
:100AD0006F565C01CE01019664E070E00E946F5693
:100AE0008C01C701B401A60195010E94B0806496F3
:100AF0000FB6F894DEBF0FBECDBFDF91CF911F912F
:100B00000F91FF90EF90DF90CF90BF90AF909F90AC
:100B10008F907F9008958F929F92AF92BF92CF92C5
:100B2000DF92EF92FF920F931F93CF93DF93CDB796
:100B3000DEB764970FB6F894DEBF0FBECDBFDE01FF
:100B40001196FC0184E101900D928150E1F781E062
:100B500080934B168093741680939D168093C616CF
:100B60008093EF16CE01019660E070E00E946F5610
:100B70007C01CE01019661E070E00E946F566C012D
:100B8000CE01019662E070E00E946F565C01CE01DA
:100B9000019663E070E00E946F564C01CE01019611
:100BA00064E070E00E946F568C01C701B601A50198
:100BB00094010E94B08064960FB6F894DEBF0FBE19
:100BC000CDBFDF91CF911F910F91FF90EF90DF90FC
:100BD000CF90BF90AF909F908F9008955F926F924B
:100BE0007F928F929F92AF92BF92CF92DF92EF92BD
:100BF000FF920F931F93CF93DF93CDB7DEB7649728
:100C00000FB6F894DEBF0FBECDBF782E692E0E94BE
:100C100032565FB6F89400D000D0409150155091F4
:100C20005115609152157091531500915415109102
:100C300055152091561530915715C0905815D090E4
:100C40005915E0905A15F0905B1580905C159090C6
:100C50005D15A0905E15B0905F1580916015909124
:100C60006115A0916215B0916315EDB7FEB7818350
:100C70009283A383B483CE0101960E943356E72D5D
:100C8000F62DDE01119684E10D9001928150E1F77D
:100C90000F900F900F900F9000E010E0872D962D91
:100CA000B8010E946F564C01FC01C080D180E280E7
:100CB000F3808091141790911517B8010E946F5618
:100CC000FC0180819181A281B381C81AD90AEA0A04
:100CD000FB0AF401C082D182E282F3820F5F1F4FD0
:100CE00005301105D9F65FBE872D962D64960FB697
:100CF000F894DEBF0FBECDBFDF91CF911F910F9152
:100D0000FF90EF90DF90CF90BF90AF909F908F902B
:100D10007F906F905F9008956F927F928F929F92D5
:100D2000AF92BF92CF92DF92EF92FF920F931F93F9
:100D3000CF93DF93CDB7DEB765970FB6F894DEBFDC
:100D40000FBECDBF3C01CE010296BE016A5F7F4F50
:100D5000AE01465F5F4F9E01225F3F4F8E010E5EE8
:100D60001F4F7E010894E11CF11C0E94E86D8981EF
:100D700081708983813029F436E1E32E37E1F32E47
:100D800004C02AE2E22E27E1F22E92E0C92ED12CF5
:100D9000CC0EDD1E00E010E0F60180809180A28084
:100DA000B380C701B8010E946F56FC018081918118
:100DB000A281B381A5019401281B390B4A0B5B0B5F
:100DC000F60121933193419351936F010F5F1F4FB0
:100DD0000530110509F700D000D04A815B816C8194
:100DE0007D810E811F8128853985CA84DB84EC844E
:100DF000FD848E849F84A888B9888A899B89AC8960
:100E0000BD89EDB7FEB781839283A383B483C30109
:100E10000E9433560F900F900F900F90C30165966C
:100E20000FB6F894DEBF0FBECDBFDF91CF911F91FB
:100E30000F91FF90EF90DF90CF90BF90AF909F9079
:100E40008F907F906F9008958093401708952F9210
:100E50003F924F925F926F927F928F929F92AF924A
:100E6000BF92CF92DF92EF92FF920F931F93CF9397
:100E7000DF9300D000D0CDB7DEB73C011A012B01C3
:100E8000ECE38E2EE5E19E2E540100E010E0C3015C
:100E9000B8010E946756FC01C080D180E280F380D7
:100EA0008091141790911517B8010E946F56FC019C
:100EB00080819181A281B3818C0D9D1DAE1DBF1DCE
:100EC000F50181939193A193B1935F010F5F1F4F40
:100ED00005301105E1F6409144155091451560919A
:100EE0004615709147158091A2169091A316A09176
:100EF000A416B091A516481759076A077B0714F482
:100F0000DB01CA018093441590934515A0934615C3
:100F1000B093471540E5642E45E1742E50E8E52E68
:100F200055E1F52ECC24AA2480E090E0A0E0B0E0CA
:100F3000F40101911191219131914F01F3014191FE
:100F40005191619171913F01041B150B260B370BD9
:100F500037FF07C030952095109501951F4F2F4FF3
:100F60003F4FF70101931193219331937F01801734
:100F70009107A207B3071CF4AC2CD901C801C39494
:100F8000F5E0CF16A9F6A09294158093951590934D
:100F90009615A0939715B09398150097A105B105E4
:100FA00051F160E472E48FE090E0A20191010E94AF
:100FB00098E229833A834B835C8360E070E080E0B1
:100FC00090E0AE014F5F5F4F23E137E100E0E0903A
:100FD00013170E94CE768091CA0D9091C90D891B7E
:100FE0008F7090915517891720F081E080935717E3
:100FF00002C0109257170F900F900F900F90DF9133
:10100000CF911F910F91FF90EF90DF90CF90BF9005
:10101000AF909F908F907F906F905F904F903F9098
:101020002F9008952F923F924F925F926F927F92EE
:101030008F929F92AF92BF92CF92DF92EF92FF92E8
:101040000F931F93CF93DF93CDB7DEB72A970FB6D9
:10105000F894DEBF0FBECDBF3C014D835E836F832E
:101060007887A0E54A2EA5E15A2EBCE32B2EB5E1E8
:101070003B2E7101620100E010E0822F90E09A8720
:10108000898789859A85002E02C0959587950A944F
:10109000E2F780FF0AC0D6018D909D90AD90BC9084
:1010A000C301B8010E94675610C0C301B8010E9475
:1010B0006756DC018D909D90AD90BC908091141787
:1010C00090911517B8010E946F56FC0180819181A3
:1010D000A281B381880D991DAA1DBB1DF7018083D4
:1010E0009183A283B3830F5F1F4F84E090E0C80E0B
:1010F000D91EE80EF91E0530110519F64091441568
:101100005091451560914615709147158091A21632
:101110009091A316A091A416B091A516481759074F
:101120006A077B0714F4DB01CA018093441590938E
:101130004515A0934615B0934715F0E88F2EF5E1BD
:101140009F2EEE24CC2400E010E020E030E0D1011E
:101150004D915D916D917D911D01F2018191919172
:10116000A191B1912F01481B590B6A0B7B0B77FFA3
:1011700007C070956095509541955F4F6F4F7F4FB9
:10118000D4014D935D936D937D934D010417150725
:10119000260737071CF4CE2C8A019B01E394B5E0A7
:1011A000EB16A9F6C0929415009395151093961519
:1011B00020939715309398150115110521053105D8
:1011C00081F16D817E818F819885A90198010E94AE
:1011D00098E260E472E48FE090E00E9498E2298354
:1011E0003A834B835C8360E070E080E090E0AE0186
:1011F0004F5F5F4F23E137E100E0E09013170E945B
:10120000CE768091CA0D9091C90D891B8F709091F7
:101210005517891720F081E08093571702C010926C
:1012200057172A960FB6F894DEBF0FBECDBFDF91D9
:10123000CF911F910F91FF90EF90DF90CF90BF90D3
:10124000AF909F908F907F906F905F904F903F9066
:101250002F9008952F923F924F925F926F927F92BC
:101260008F929F92AF92BF92CF92DF92EF92FF92B6
:101270000F931F93CF93DF93CDB7DEB766970FB66B
:10128000F894DEBF0FBECDBF1C01498B5A8B6B8B10
:101290007C8BED86FE860F87188BDE8ACD8A40E533
:1012A00055E15C874B876CE375E17A8769878B0131
:1012B0002A01CC24DD24E22EFF24C7010C2C02C01D
:1012C000959587950A94E2F780FF0AC0F201808025
:1012D0009180A280B380C101B6010E94675610C000
:1012E000C101B6010E946756FC0180809180A280F6
:1012F000B3808091141790911517B6010E946F5614
:10130000FC0180819181A281B381880D991DAA1D64
:10131000BB1DF80180839183A283B3830894C11C11
:10132000D11C44E050E0440E551E0C5F1F4F55E0A9
:10133000C516D10411F640914415509145156091A0
:101340004615709147158091A2169091A316A09111
:10135000A416B091A516481759076A077B0714F41D
:10136000DB01CA018093441590934515A09346155F
:10137000B09347151092941520E8222E25E1322EC5
:1013800061E477E17E836D838DE995E198878F83B2
:1013900010E0882499245401E985FA8541915191FE
:1013A00061917191FA87E987EB85FC858191919133
:1013B000A191B191FC87EB87481B590B6A0B7B0B02
:1013C000F10140835183628373836A017B0177FF5C
:1013D00007C0CC24DD247601C41AD50AE60AF70A30
:1013E000F0E0CF16F0E8DF06F0E0EF06F0E0FF06F1
:1013F00064F4CA0177276627ED81FE81208131815F
:10140000428153810E9444DE22C0CB01BA010E9476
:10141000BDE02B013C01ED81FE8160817181828103
:1014200093810E94BDE020E030E040E857E30E9455
:10143000C1E19B01AC01C301B2010E94C1E120E006
:1014400030E040E857E40E94C1E10E948AE0DC01FC
:10145000CB01EF81F88580839183A283B383F1016F
:10146000C082D182E282F3828C149D04AE04BF0458
:1014700024F4109394154601570144E050E0240EE3
:10148000351E1F5F6D817E816C5F7F4F7E836D8314
:101490008F819885049698878F83153009F07CCFCB
:1014A0008092951590929615A0929715B0929815E6
:1014B00081149104A104B10409F463C06D857E8593
:1014C0008F85988920E030E040E050E00E94E4DF22
:1014D000882309F456C06D857E858F85988920E024
:1014E00030E040E857E40E94C1E10E948AE0DC015C
:1014F000CB018093991590939A15A0939B15B09367
:101500009C1520911004222379F0ED89FE89CF01EA
:10151000AA2797FDA095BA2F1AE0880F991FAA1F36
:10152000BB1F1A95D1F704C080E090E0A0E0B0E0C6
:1015300049895A896B897C8949835A836B837C8367
:10154000222319F00091110401C000E0BC01CD017B
:10155000AE014F5F5F4F23E137E1E09013170E9428
:10156000CE768091CA0D9091C90D891B8F70909194
:101570005517891720F081E08093571702C0109209
:10158000571766960FB6F894DEBF0FBECDBFDF913A
:10159000CF911F910F91FF90EF90DF90CF90BF9070
:1015A000AF909F908F907F906F905F904F903F9003
:1015B0002F9008952F923F924F925F926F927F9259
:1015C0008F929F92AF92BF92CF92DF92EF92FF9253
:1015D0000F931F93CF93DF93CDB7DEB765970FB609
:1015E000F894DEBF0FBECDBF882E29013A011092BC
:1015F00011047E010894E11CF11CC7016D8B0E944F
:101600008C866AE4C62E66E1D62E00E010E06D8975
:10161000262E33249E2CEF2CFF24F394C101002EA0
:1016200002C0959587950A94E2F737E2A32E36E13A
:10163000B32EA00EB11E80FD03C0F50110821DC0A7
:10164000892D9E2DB8010E946F56FC01882029F03B
:101650008FEF9FEFAFEFBFE304C080E090E0A0E02A
:10166000B0EC80839183A283B383F501F0820230D2
:1016700011F4F0923F17F601F0820F5F1F4F89E2DD
:1016800090E0C80ED91E0530110541F6CE01019635
:10169000B301A2010E94278781E0809356176596C7
:1016A0000FB6F894DEBF0FBECDBFDF91CF911F9173
:1016B0000F91FF90EF90DF90CF90BF90AF909F90F1
:1016C0008F907F906F905F904F903F902F900895F4
:1016D000853098F49091221621E030E002C0220F6C
:1016E000331F8A95E2F7662321F0922B90932216FE
:1016F000089520952923209322160895809122167B
:101700000895853078F4482F50E02BE030E0429F78
:10171000C001439F900D529F900D1124885A984EFE
:101720000E94FBA80895809311040895817080930E
:101730001317813019F486E197E102C08AE297E13C
:10174000909315178093141708958091C303909177
:10175000C4030097A1F0E091C503F091C603808116
:1017600090E00090C70302C0959587950A94E2F730
:101770008170907091E020919216281709F490E002
:10178000292F2295220F207E8091BC039091BD03CA
:101790000097A1F0E091BE03F091BF03808190E03B
:1017A0000090C00302C0959587950A94E2F7817076
:1017B000907031E090919216981709F430E03295CC
:1017C000307F322B8091A0039091A1030097A1F06C
:1017D000E091A203F091A303808190E00090A40324
:1017E00002C0959587950A94E2F78170907021E088
:1017F00090916916981709F420E0220F220F220F0A
:10180000232B8091990390919A030097A1F0E09186
:101810009B03F0919C03808190E000909D0302C0A7
:10182000959587950A94E2F78170907041E09091C8
:101830006916981709F440E0440F440F422B809139
:101840007D0390917E030097A1F0E0917F03F091DA
:101850008003208130E00090810302C035952795F8
:101860000A94E2F72170307081E09091401692174F
:1018700009F480E0880F842B209176033091770360
:1018800021153105A1F0E0917803F09179032081D1
:1018900030E000907A0302C0359527950A94E2F76C
:1018A0002170307091E030914016321709F490E0C9
:1018B000892B089590911004992309F480E00E94E7
:1018C000BB6E08950E94436E1092571710925617E0
:1018D00080E00E941A81809110048093110481E0BD
:1018E0000E945A8C08952F923F924F925F926F926E
:1018F0007F928F929F92AF92BF92CF92DF92EF92A0
:10190000FF920F931F93CF93DF9380E00E941A8181
:101910000E94438410923E1710923F170E946984E0
:1019200080E00E94968B88E891E06FEF0E9477A993
:10193000803811F00E94123D8EE691E060E00E9436
:1019400077A98170809310048093110481E00E9434
:101950005A8C01E417E1C0E08C2F0E9490839B0118
:10196000AC0160E070E080E89FE30E94E8DF20E0E7
:1019700030E040E857E40E94C1E10E948AE0DC01C7
:10198000CB01F80181939193A193B1938F01CF5F24
:10199000C53011F782E791E068EE73E00E9495A9E7
:1019A000A0E0B0E08093F3159093F415A093F515A3
:1019B000B093F61584E791E068EE73E00E9495A974
:1019C000A0E0B0E08093F7159093F815A093F91577
:1019D000B093FA1586E791E066E970E00E9495A958
:1019E000A0E0B0E08093FB159093FC15A093FD154B
:1019F000B093FE1588E791E060EA7FE00E9495A928
:101A0000A0E0B0E08093FF1590930016A09301161C
:101A1000B09302168AE791E060EA7FE00E9495A900
:101A2000A0E0B0E08093031690930416A0930516EF
:101A3000B093061603EF15E1E9EB6E2EE5E17E2E7D
:101A4000F8E64F2EF5E15F2EC0E088248A94982CAA
:101A500054011801F801C080D180E280F3808C2FFE
:101A60000E9490839B01AC0160EF7FEF8FE799E4C8
:101A70000E94E8DF0E948FE0DC01CB018C159D0500
:101A8000AE05BF05A0F48C2F0E9490839B01AC0192
:101A900060EF7FEF8FE799E40E94E8DF0E948FE01C
:101AA000DC01CB01F80180839183A283B3830C5FB7
:101AB0001F4FF10160817181828193810E94BBE09F
:101AC0006B017C018C2F0E9490839B01AC01C701AC
:101AD000B6010E94C1E10E948FE09B01AC01F301BD
:101AE00061937193819391933F01C501B4010E9469
:101AF00076E2F20121933193419351932F01CF5F0D
:101B0000C53009F0A6CF80E791E060ED77E00E9454
:101B100095A9A0E0B0E08093EF159093F015A09305
:101B2000F115B093F2158131F7E29F07F0E0AF07AE
:101B3000F0E0BF0760F080E197E2A0E0B0E08093C2
:101B4000EF159093F015A093F115B093F21586E878
:101B500091E060EA7FE00E9495A9A0E0B0E0809368
:101B6000EB159093EC15A093ED15B093EE15813124
:101B700027E2920720E0A20720E0B20760F080E1B0
:101B800097E2A0E0B0E08093EB159093EC15A09362
:101B9000ED15B093EE1580EE91E060E070E00E94EC
:101BA00095A990939D0D80939C0D82EE91E060E04D
:101BB00070E00E9495A990939F0D80939E0D8CE7F5
:101BC00091E06AE070E00E9495A9BC0180E090E09D
:101BD0000E94BBE020E030E040E857E40E94C1E111
:101BE0000E948AE0DC01CB018093D3159093D41539
:101BF000A093D515B093D6158EE791E06AE070E01A
:101C00000E9495A9BC0180E090E00E94BBE020E02A
